:020000040800F2
:1000000000060020A1020008FD0F00087D0F000877
:10001000D50F00087D0F0008A90F0008A3020008F3
:10002000A3020008A3020008A3020008512300084D
:10003000A3020008A3020008A3020008A30200080C
:10004000A3020008A3020008A3020008A3020008FC
:10005000A3020008A3020008D937000805380008E9
:10006000313800085D38000889380008A30200080C
:10007000A3020008A3020008A3020008A3020008CC
:10008000A3020008A3020008A3020008A3020008BC
:10009000A3020008A3020008A3020008B538000864
:1000A000A3020008A3020008A3020008A30200089C
:1000B000A3020008A3020008A3020008A30200088C
:1000C000A3020008A3020008A3020008A30200087C
:1000D000A3020008A3020008A3020008A30200086C
:1000E00019390008A3020008A3020008A3020008AF
:1000F000A3020008A3020008A3020008A30200084C
:10010000A3020008A30200088D390008A30200081A
:10011000A3020008A3020008A3020008A30200082B
:10012000A3020008A3020008A3020008A30200081B
:10013000A3020008A3020008A3020008A30200080B
:10014000A3020008A3020008A3020008A3020008FB
:10015000A3020008A3020008A3020008A3020008EB
:10016000A3020008A3020008A3020008A3020008DB
:10017000A3020008BD2E0008A3020008A302000885
:10018000A3020008A3020008A3020008A3020008BB
:10019000A3020008A3020008A3020008A3020008AB
:1001A000A3020008A3020008A3020008A30200089B
:1001B000A3020008A3020008A3020008A30200088B
:1001C000A3020008A3020008A3020008A30200087B
:1001D000A3020008A92E0008A3020008A302000839
:1001E000A3020008A3020008A3020008A30200085B
:1001F000A3020008A3020008A3020008A30200084B
:10020000A3020008A3020008A3020008A30200083A
:10021000A3020008A3020008A3020008A30200082A
:10022000A3020008A3020008A3020008A30200081A
:10023000A3020008A3020008A3020008A30200080A
:10024000A3020008A3020008A3020008A3020008FA
:10025000A3020008A3020008A3020008A3020008EA
:10026000A3020008A3020008A3020008A3020008DA
:10027000A3020008A3020008A3020008A3020008CA
:10028000A3020008A3020008A3020008A3020008BA
:10029000A3020008A3020008A3020008A3020008AA
:1002A00002E000F000F8FEE772B63A4880F30888F2
:1002B000394880F3098839484EF60851CEF20001DA
:1002C000086040F20000CCF200004EF63471CEF22D
:1002D00000010860BFF34F8FBFF36F8F40F2000043
:1002E000C0F2F0004EF68851CEF200010860BFF374
:1002F0004F8FBFF36F8F4FF00000E1EE100A4EF604
:100300003C71CEF200010860062080F31488BFF330
:100310006F8F02F0DBF802F07DF803F017F84FF072
:1003200055301F491B4A91423CBF41F8040BFAE784
:100330001C49194A91423CBF41F8040BFAE71A499B
:100340001A4A1B4B9A423EBF51F8040B42F8040B69
:10035000F8E700201749184A91423CBF41F8040BC6
:10036000FAE702F095F803F075F8144C144DAC421E
:1003700003DA54F8041B8847F9E700F041F8114C00
:10038000114DAC4203DA54F8041B8847F9E702F038
:100390007DB80000000600200022002000000008B8
:1003A0000000002000060020583D00080022002028
:1003B0005C220020602200207C420020A002000875
:1003C000A0020008A0020008A00200082DE9F04FDA
:1003D0002DED108AC1F80CD0D0F80CD0BDEC108AED
:1003E000BDE8F08F002383F311882846A047002042
:1003F00001F090FBFEE701F00BFB00DFFEE70000E1
:1004000038B501F08DFF30B1164B00220A211A7267
:100410005A729972DA7201F059FF054601F08EFFA7
:100420000446D0B9104B9D4219D001339D4241F290
:10043000883512BF044600250124002001F050FF3A
:100440000CB100F079F800F06DFD00F015FC2846C5
:1004500000F020F900F070F8F9E70025EDE7054617
:10046000EBE700BF00220020010007B008B500F054
:10047000D5FBA0F120035842584108BD07B541F211
:100480001203022101A8ADF8043000F0E5FB03B02F
:100490005DF804FB38B5202383F311881748C3683F
:1004A0000BB101F0BDFB0023154A4FF47A711348DC
:1004B00001F07AFB002383F31188124C236813B1F7
:1004C0002368013B2360636813B16368013B636089
:1004D0000D4D2B7833B963687BB9022000F09CFC8A
:1004E000322363602B78032B07D163682BB902207A
:1004F00000F092FC4FF47A73636038BD60220020F4
:10050000950400087C23002074220020084B1870FA
:1005100003280CD8DFE800F008050208022000F0EC
:1005200071BC022000F064BC024B00225A6070478C
:10053000742200207C230020F8B5504B504A1C4602
:100540001968013100F0998004339342F8D1626850
:100550004C4B9A4240F291804B4B9B6803F10063F5
:1005600003F5C0239A4280F08880002000F09EFBB3
:100570000220FFF7CBFF454B0021D3F8E820C3F85A
:10058000E810D3F81021C3F81011D3F81021D3F8D4
:10059000EC20C3F8EC10D3F81421C3F81411D3F8ED
:1005A0001421D3F8F020C3F8F010D3F81821C3F8C1
:1005B0001811D3F81821D3F8802042F00062C3F854
:1005C0008020D3F8802022F00062C3F88020D3F886
:1005D0008020D3F8802042F00072C3F88020D3F846
:1005E000802022F00072C3F88020D3F8803072B6E9
:1005F0004FF0E023C3F8084DD4E90004BFF34F8F58
:10060000BFF36F8F224AC2F88410BFF34F8F536934
:1006100023F480335361BFF34F8FD2F8803043F619
:10062000E076C3F3C905C3F34E335B0103EA060C5E
:1006300029464CEA81770139C2F87472F9D2203B1D
:1006400013F1200FF2D1BFF34F8FBFF36F8FBFF3C2
:100650004F8FBFF36F8F536923F40033536100232F
:10066000C2F85032BFF34F8FBFF36F8F202383F355
:100670001188854680F308882047F8BD00000608E9
:1006800020000608FFFF0508002200200044025851
:1006900000ED00E02DE9F04F93B0B44B2022FF2194
:1006A00000900AA89D6800F0E7FBB14A1378A3B94F
:1006B0000121B0481170C360202383F31188C368FF
:1006C0000BB101F0ADFA0023AB4A4FF47A71A9489F
:1006D00001F06AFA002383F31188009B13B1A74B42
:1006E000009A1A60A64A1378032B03D000231370D4
:1006F000A24A53604FF0000A009CD3465646D146AA
:10070000012000F07FFB24B19C4B1B68002B00F004
:100710002682002000F082FA0390039B002BF2DB7C
:10072000012000F065FB039B213B1F2BE8D801A2B1
:1007300052F823F0B5070008DD070008710800082B
:100740000107000801070008010700080309000865
:10075000D30A0008ED0900084F0A0008770A0008CC
:100760009D0A000801070008AF0A000801070008F9
:10077000210B00085508000801070008650B000858
:10078000C107000855080008010700084F0A0008C3
:100790000107000801070008010700080107000819
:1007A0000107000801070008010700080107000809
:1007B000710800080220FFF759FE002840F0F98177
:1007C000009B022105A8BAF1000F08BF1C4641F2A8
:1007D0001233ADF8143000F03FFA91E74FF47A701D
:1007E00000F01CFA071EEBDB0220FFF73FFE00289B
:1007F000E6D0013F052F00F2DE81DFE807F0030AB3
:100800000D1013360523042105A8059300F024FAE2
:1008100017E004215548F9E704215A48F6E7042176
:100820005948F3E74FF01C08404608F1040800F06F
:100830003FFA0421059005A800F00EFAB8F12C0F3C
:10084000F2D101204FF0000900FA07F747EA0B0B3D
:100850005FFA8BFB00F05CFB26B10BF00B030B2B5C
:1008600008BF0024FFF70AFE4AE704214748CDE706
:10087000002EA5D00BF00B030B2BA1D10220FFF70C
:10088000F5FD074600289BD00120002600F00EFA57
:100890000220FFF73BFE5FFA86F8404600F016FAAA
:1008A0000446B0B1039940460136A1F140025142DD
:1008B000514100F01BFA0028EDD1BA46044641F23E
:1008C0001213022105A83E46ADF8143000F0C4F919
:1008D00016E725460120FFF719FE244B9B68AB4223
:1008E00007D9284600F0E4F9013040F0678104356B
:1008F000F3E70025224BBA463E461D701F4B5D6054
:10090000A8E7002E3FF45CAF0BF00B030B2B7FF43A
:1009100057AF0220FFF7FAFD322000F07FF9B0F167
:100920000008FFF64DAF18F003077FF449AF0F4AF8
:1009300008EB0503926893423FF642AFB8F5807F1B
:100940003FF73EAF124BB845019323DD4FF47A7069
:1009500000F064F90390039A002AFFF631AF039A7E
:100960000137019B03F8012BEDE700BF00220020B7
:100970007823002060220020950400087C230020BA
:100980007422002004220020082200200C220020D3
:1009900078220020C820FFF769FD074600283FF4B1
:1009A0000FAF1F2D11D8C5F120020AAB25F00300AF
:1009B00084494245184428BF4246019200F036FA65
:1009C000019AFF217F4800F057FA4FEAA803C8F3C5
:1009D00087027C492846019300F056FA0646002813
:1009E0003FF46DAF019B05EB830533E70220FFF772
:1009F0003DFD00283FF4E4AE00F096F900283FF4F6
:100A0000DFAE0027B846704B9B68BB4218D91F2F3A
:100A100011D80A9B01330ED027F0030312AA134406
:100A200053F8203C05934046042205A9043700F002
:100A3000E7FA8046E7E7384600F03AF90590F2E732
:100A4000CDF81480042105A800F006F902E7002380
:100A5000642104A8049300F0F5F800287FF4B0AEF8
:100A60000220FFF703FD00283FF4AAAE049800F02F
:100A700051F90590E6E70023642104A8049300F0EF
:100A8000E1F800287FF49CAE0220FFF7EFFC00287D
:100A90003FF496AE049800F03FF9EAE70220FFF732
:100AA000E5FC00283FF48CAE00F04EF9E1E70220AF
:100AB000FFF7DCFC00283FF483AE05A9142000F00A
:100AC00049F907460421049004A800F0C5F8394606
:100AD000B9E7322000F0A2F8071EFFF671AEBB079F
:100AE0007FF46EAE384A07EB0903926893423FF6F3
:100AF00067AE0220FFF7BAFC00283FF461AE27F092
:100B000003074F44B9453FF4A5AE484609F104092F
:100B100000F0CEF80421059005A800F09DF8F1E75B
:100B20004FF47A70FFF7A2FC00283FF449AE00F0C2
:100B3000FBF8002844D00A9B01330BD008220AA9F5
:100B4000002000F0A1F900283AD02022FF210AA8B5
:100B500000F092F9FFF792FC1C4800F0E1FF13B09F
:100B6000BDE8F08F002E3FF42BAE0BF00B030B2BE8
:100B70007FF426AE0023642105A8059300F062F8F7
:100B8000074600287FF41CAE0220FFF76FFC80466A
:100B900000283FF415AEFFF771FC41F2883000F0F9
:100BA000BFFF059800F0E8F946463C4600F0B0F972
:100BB000A6E506464EE64FF0000901E6BA467EE697
:100BC00037467CE67822002000220020A086010023
:100BD0000F4B70B51B780C460133DBB2012B11D8DB
:100BE0000C4D4FF47A732968A2FB033222460E6A39
:100BF00001462846B047844204D1074B0022012019
:100C00001A7070BD4FF4FA7000F08AFF0020F8E708
:100C10001022002070250020B0230020002307B5FB
:100C2000024601210DF107008DF80730FFF7D0FFD4
:100C300020B19DF8070003B05DF804FB4FF0FF30D2
:100C4000F9E700000A46042108B5FFF7C1FF80F06C
:100C50000100C0B2404208BD30B4054C0A4601460E
:100C600023682046DD69034BAC4630BC604700BFBB
:100C700070250020A086010070B50A4E00240A4DA0
:100C800001F0FCF9308028683388834208D901F0EC
:100C9000F1F92B6804440133B4F5C02F2B60F2D373
:100CA00070BD00BFB22300208423002001F0C4BA2D
:100CB00000F1006000F5C0200068704700F100609E
:100CC000920000F5C02001F03BBA0000054B1A6805
:100CD000054B1B889B1A834202D9104401F0CAB904
:100CE0000020704784230020B223002038B504463A
:100CF000074D29B128682044BDE8384001F0D2B939
:100D00002868204401F0BCF90028F3D038BD00BFAA
:100D1000842300200020704700F1FF5000F58F1061
:100D2000D0F8000870470000064991F8243033B12C
:100D300000230822086A81F82430FFF7BFBF012092
:100D4000704700BF88230020014B1868704700BF20
:100D50000010005C244BF0B51A680446234BC2F324
:100D60000B06120C1F885868BE4293F9085028D011
:100D70009F89BE4206D101200C2505FB003358682F
:100D800093F9085041F201039A421CD041F2030347
:100D90009A421AD042F201039A4218D042F2030357
:100DA0009A4208BF5625621E0B46441E0A449342CF
:100DB0000FD214F9016F581C6EB1034600F8016C94
:100DC000F5E70020D8E75A25EDE75925EBE7582548
:100DD000E9E7184605E02C2482421C7001D9981CD2
:100DE0005D70401AF0BD00BF0010005C14220020AE
:100DF000022803D1024B4FF080729A61704700BF06
:100E000000000258022803D1024B4FF480729A610D
:100E1000704700BF00000258022804D1024A5369FB
:100E200083F480735361704700000258002310B5AB
:100E3000934203D0CC5CC4540133F9E710BD0000E9
:100E4000013810B510F9013F3BB191F900409C42C7
:100E500003D11AB10131013AF4E71AB191F9002036
:100E6000981A10BD1046FCE703460246D01A12F944
:100E7000011B0029FAD1704702440346934202D075
:100E800003F8011BFAE770472DE9F8431F4D14469C
:100E90000746884695F8242052BBDFF870909CB333
:100EA00095F824302BB92022FF2148462F62FFF706
:100EB000E3FF95F824004146C0F1080205EB8000ED
:100EC000A24228BF2246D6B29200FFF7AFFF95F8A4
:100ED0002430A41B17441E449044E4B2F6B2082EFA
:100EE00085F82460DBD1FFF71FFF0028D7D108E089
:100EF0002B6A03EB82038342CFD0FFF715FF002854
:100F0000CBD10020BDE8F8830120FBE78823002037
:100F1000024B1A78024B1A70704700BFB0230020B2
:100F20001022002010B5104C104800F0FBF82146AC
:100F30000E4800F023F924680D48D4F89020D2F828
:100F4000043843F00203C2F8043800F0E9FD09490F
:100F5000204600F021FAD4F89020D2F8043823F08B
:100F60000203C2F8043810BD383B00087025002089
:100F700040420F00403B00087047000000B59BB0A6
:100F8000EFF3098168226846FFF750FFEFF305830E
:100F9000044B9A6BDA6A9A6A9A6A9A6A9A6A9A6AA5
:100FA0009B6AFEE700ED00E000B59BB0EFF309811E
:100FB00068226846FFF73AFFEFF30583044B9A6B0C
:100FC0009A6A9A6A9A6A9A6A9A6A9B6AFEE700BF64
:100FD00000ED00E000B59BB0EFF3098168226846A0
:100FE000FFF724FFEFF30583034B5A6B9A6A9A6A63
:100FF0009A6A9A6A9B6AFEE700ED00E0FEE700004D
:1010000030B50A44084D91420DD011F8013B5840CB
:10101000082340F30004013B2C4013F0FF0384EA53
:101020005000F6D1EFE730BD2083B8ED0268436889
:101030001143016003B118477047000013B5406BBE
:1010400000F58054D4F8A4381A681178042914D112
:10105000017C022911D11979012312898B40134295
:101060000BD101A94C3002F071F8D4F8A448024623
:10107000019B2179206800F0DFF902B010BD00006B
:10108000143001F0F3BF00004FF0FF33143001F0D3
:10109000EDBF00004C3002F0C5B800004FF0FF3348
:1010A0004C3002F0BFB80000143001F0C1BF0000A6
:1010B0004FF0FF31143001F0BBBF00004C3002F0A4
:1010C00091B800004FF0FF324C3002F08BB80000B6
:1010D0000020704710B500F58054D4F8A4381A6881
:1010E0001178042917D1017C022914D159790123DF
:1010F00052898B4013420ED1143001F053FF024647
:1011000048B1D4F8A4484FF4407361792068BDE831
:10111000104000F07FB910BD406BFFF7DBBF00004F
:10112000704700007FB5124B01250426044603607A
:101130000023057400F1840243602946C0E90233AC
:101140000C4B0290143001934FF44073009601F061
:1011500005FF094B04F69442294604F14C00029421
:10116000CDE900634FF4407301F0CCFF04B070BDD3
:10117000743A0008191100083D1000080A6820237D
:1011800083F311880B790B3342F823004B79133327
:1011900042F823008B7913B10B3342F8230000F59A
:1011A0008053C3F8A41802230374002383F3118827
:1011B0007047000038B5037F044613B190F85430EF
:1011C000ABB90125201D0221FFF730FF04F1140007
:1011D0006FF00101257700F0CBFC04F14C0084F89E
:1011E00054506FF00101BDE8384000F0C1BC38BD7B
:1011F00010B5012104460430FFF718FF00232377C0
:1012000084F8543010BD000038B504460025143071
:1012100001F0BCFE04F14C00257701F08BFF201D8E
:1012200084F854500121FFF701FF2046BDE8384003
:10123000FFF750BF90F8803003F06003202B06D1F9
:1012400090F881200023212A03D81F2A06D80020E5
:101250007047222AFBD1C0E91D3303E0034A4267ED
:1012600007228267C3670120704700BF2C2200203D
:1012700037B500F58055D5F8A4381A6811780429D7
:101280001AD1017C022917D11979012312898B40C7
:10129000134211D100F14C04204602F00BF858B172
:1012A00001A9204601F052FFD5F8A4480246019B4F
:1012B0002179206800F0C0F803B030BD01F10B03C4
:1012C000F0B550F8236085B004460D46FEB12023EA
:1012D00083F3118804EB8507301D0821FFF7A6FE74
:1012E000FB6806F14C005B691B681BB1019001F0C3
:1012F0003BFF019803A901F029FF024648B1039B77
:101300002946204600F098F8002383F3118805B0A1
:10131000F0BDFB685A691268002AF5D01B8A013BB0
:101320001340F1D104F18002EAE70000133138B52F
:1013300050F82140ECB1202383F3118804F5805349
:10134000D3F8A4281368527903EB8203DB689B6906
:101350005D6845B104216018FFF768FE294604F175
:10136000140001F029FE2046FFF7B4FE002383F3AA
:10137000118838BD7047000001F01CB901234022DC
:10138000002110B5044600F8303BFFF775FD00233F
:10139000C4E9013310BD000010B52023044683F3D7
:1013A00011882422416000210C30FFF765FD2046A2
:1013B00001F022F902232370002383F3118810BD6A
:1013C00070B500EB8103054650690E461446DA609D
:1013D00018B110220021FFF74FFDA06918B11022AB
:1013E0000021FFF749FD31462846BDE8704001F075
:1013F00015BA000083682022002103F0011310B504
:10140000044683601030FFF737FD2046BDE81040EA
:1014100001F090BAF0B4012500EB810447898D40BA
:10142000E4683D43A469458123600023A2606360B2
:10143000F0BC01F0ADBA0000F0B4012500EB81046E
:1014400007898D40E4683D4364690581236000237A
:10145000A2606360F0BC01F023BB000070B5022302
:1014600000250446242203702946C0F888500C3019
:1014700040F8045CFFF700FD204684F8705001F04E
:1014800061F963681B6823B129462046BDE87040B6
:10149000184770BD037880F88C30052303704368CB
:1014A0001B6810B504460BB1042198470023A360C4
:1014B00010BD000090F88C20436802701B680BB1CF
:1014C000052118477047000070B590F87030044649
:1014D00013B1002380F8703004F18002204601F03F
:1014E0004DFA63689B68B3B994F8803013F06005D7
:1014F00035D00021204601F0F7FC0021204601F004
:10150000E7FC63681B6813B1062120469847062351
:1015100084F8703070BD204698470028E4D0B4F8B5
:101520008630A26F9A4288BFA36794F98030A56F76
:10153000002B4FF0200380F20381002D00F0F28099
:10154000092284F8702083F3118800212046D4E911
:101550001D23FFF771FF002383F31188DAE794F866
:10156000812003F07F0343EA022340F202329342D8
:1015700000F0C58021D8B3F5807F48D00DD8012B6D
:101580003FD0022B00F09380002BB2D104F18802EF
:1015900062670222A267E367C1E7B3F5817F00F0CB
:1015A0009B80B3F5407FA4D194F88230012BA0D169
:1015B000B4F8883043F0020332E0B3F5006F4DD049
:1015C00017D8B3F5A06F31D0A3F5C063012B90D825
:1015D0006368204694F882205E6894F88310B4F81B
:1015E0008430B047002884D0436863670368A367EA
:1015F0001AE0B3F5106F36D040F6024293427FF402
:1016000078AF5C4B63670223A3670023C3E794F8BA
:101610008230012B7FF46DAFB4F8883023F00203E1
:10162000A4F88830C4E91D55E56778E7B4F8803040
:10163000B3F5A06F0ED194F88230204684F88A303A
:1016400001F0DEF863681B6813B10121204698475A
:10165000032323700023C4E91D339CE704F18B03AB
:1016600063670123C3E72378042B10D1202383F37E
:1016700011882046FFF7BEFE85F3118803216368B9
:1016800084F88B5021701B680BB12046984794F862
:101690008230002BDED084F88B3004232370636803
:1016A0001B68002BD6D0022120469847D2E794F839
:1016B000843020461D0603F00F010AD501F050F9D1
:1016C000012804D002287FF414AF2B4B9AE72B4B50
:1016D00098E701F037F9F3E794F88230002B7FF4B4
:1016E00008AF94F8843013F00F01B3D01A062046E7
:1016F00002D501F011FCADE701F002FCAAE794F875
:101700008230002B7FF4F5AE94F8843013F00F0193
:10171000A0D01B06204602D501F0E6FB9AE701F0B7
:10172000D7FB97E7142284F8702083F311882B46A7
:101730002A4629462046FFF76DFE85F31188E9E623
:101740005DB1152284F8702083F3118800212046B2
:10175000D4E91D23FFF75EFEFDE60B2284F870201E
:1017600083F311882B462A4629462046FFF764FE5C
:10177000E3E700BFA43A00089C3A0008A03A00083A
:1017800038B590F870300446002B3ED0063BDAB2F4
:101790000F2A34D80F2B32D8DFE803F03731310865
:1017A000223231313131313131313737856FB0F853
:1017B00086309D4214D2C3681B8AB5FBF3F203FB4B
:1017C00012556DB9202383F311882B462A462946EA
:1017D000FFF732FE85F311880A2384F870300EE09B
:1017E000142384F87030202383F3118800232046CB
:1017F0001A461946FFF70EFE002383F3118838BD01
:10180000C36F03B198470023E7E70021204601F0AA
:101810006BFB0021204601F05BFB63681B6813B182
:101820000621204698470623D7E7000010B590F818
:1018300070300446142B29D017D8062B05D001D8B8
:101840001BB110BD093B022BFBD80021204601F043
:101850004BFB0021204601F03BFB63681B6813B182
:10186000062120469847062319E0152BE9D10B23C2
:1018700080F87030202383F3118800231A4619461C
:10188000FFF7DAFD002383F31188DAE7C3689B6969
:101890005B68002BD5D1C36F03B19847002384F850
:1018A0007030CEE7024B0022C3E900339A607047E4
:1018B000B4230020002382680374054B1B689968D9
:1018C0009142FBD25A6803604260106058607047D2
:1018D000B423002008B5202383F31188037C032B55
:1018E00005D0042B0DD02BB983F3118808BD4369B3
:1018F00000221A604FF0FF334361FFF7DBFF002344
:10190000F2E7D0E9003213605A60F3E700238268FF
:101910000374054B1B6899689142FBD85A680360B1
:101920004260106058607047B4230020054B19696D
:1019300008741868026853601A6018610123037400
:10194000FEF744BDB42300204B1C30B5044687B0DD
:101950000A4D10D02B6901A8094A00F025F920464C
:10196000FFF7E4FF049B13B101A800F059F92B69BC
:10197000586907B030BDFFF7D9FFF8E7B42300205E
:10198000D518000838B50C4D044641612B698168B3
:101990009A68914203D8BDE83840FFF78BBF1846DC
:1019A000FFF7B4FF01232C61014623742046BDE8F4
:1019B0003840FEF70BBD00BFB4230020044B1A686B
:1019C0001B6990689B68984294BF00200120704773
:1019D000B423002010B5084C236820691A685460AD
:1019E0002260012223611A74FFF790FF01462069EB
:1019F000BDE81040FEF7EABCB423002008B5FFF7AD
:101A0000DDFF18B1BDE80840FFF7E4BF08BD0000E6
:101A1000FFF7E0BFFEE7000010B50C4CFFF742FFF8
:101A200000F0B4F880220A49204600F03BF8012378
:101A300044F8180C037400F09BFC002383F3118816
:101A400062B60448BDE8104000F04CB8DC2300202A
:101A5000A83A0008B83A000800F01CB9EFF311806A
:101A600020B9EFF30583202282F31188704700002C
:101A700010B530B9EFF30584C4F3080414B180F352
:101A8000118810BDFFF7BAFF84F31188F9E7000051
:101A9000034A516853685B1A9842FBD8704700BFED
:101AA000001000E082600222028270478368A3F186
:101AB0007C0243F80C2C026943F83C2C426943F841
:101AC000382C074A43F81C2CC268A3F1180043F8CD
:101AD000102C022203F8082C002203F8072C704770
:101AE000E503000810B5202383F31188FFF7DEFF1C
:101AF00000210446FFF746FF002383F311882046A8
:101B000010BD0000024B1B6958610F20FFF70EBF8C
:101B1000B4230020202383F31188FFF7F3BF0000D4
:101B200008B50146202383F311880820FFF70CFF36
:101B3000002383F3118808BD49B1064B42681B6935
:101B400018605A60136043600420FFF7FDBE4FF039
:101B5000FF307047B42300200368984206D01A680B
:101B60000260506018465961FFF7A4BE704700003C
:101B700038B504460D462068844200D138BD03685C
:101B800023605C604561FFF795FEF4E7054B4FF07D
:101B9000FF3103F11402C3E905220022C3E9071251
:101BA000704700BFB423002070B51C4E05460C469C
:101BB000C0E9032301F0B4FB334653F8142F9A42D3
:101BC0000DD130620A2C2CBF00190A302A60C5E9F9
:101BD0000124C6E90555BDE8704001F08BBB316AB0
:101BE000431AE31838BF1C469368A34202D9081968
:101BF00001F090FB73699A6894420CD85A68AC6003
:101C00002B606A6015609A685D60121B9A604FF0E5
:101C1000FF33F36170BDA41A1B68ECE7B423002006
:101C200038B51B4C636998420DD08168D0E9003209
:101C300013605A600022C2609A680A449A604FF0AA
:101C4000FF33E36138BD03682246002142F8143FA8
:101C500093425A60C16003D1BDE8384001F054BBE3
:101C60009A688168256A0A449A6001F059FB6369A1
:101C7000411B9A688A42E5D9AB181D1A206A092DC2
:101C800098BF01F10A02BDE83840104401F042BBA0
:101C9000B42300202DE9F041184C002704F114066C
:101CA000656901F03DFB236AAA68C11A8A4215D80A
:101CB0001344D5F80C802362D5E9003213605A60D2
:101CC0006369EF60B34201D101F01EFB87F3118815
:101CD0002869C047202383F31188E1E76169B14295
:101CE00009D013441B1ABDE8F0410A2B2CBFC018C1
:101CF0000A3001F00FBBBDE8F08100BFB423002023
:101D000000207047FEE70000704700004FF0FF30F2
:101D10007047000002290CD0032904D0012907488C
:101D200018BF00207047032A05D8054800EBC20001
:101D30007047044870470020704700BF9C3B000874
:101D40003C220020503B000870B59AB0054608467A
:101D5000144601A900F0C2F801A8FFF785F8431C5A
:101D60000022C6B25B001046C5E90034237003238D
:101D7000023404F8013C01ABD1B202348E4201D8E6
:101D80001AB070BD13F8011B013204F8010C04F8FD
:101D9000021CF1E708B5202383F311880348FFF7FD
:101DA00067FA002383F3118808BD00BF7025002067
:101DB00090F8803003F01F02012A07D190F88120AB
:101DC0000B2A03D10023C0E91D3315E003F06003A3
:101DD000202B08D1B0F884302BB990F88120212A2B
:101DE00003D81F2A04D8FFF725BA222AEBD0FAE736
:101DF000034A426707228267C3670120704700BF1A
:101E00003322002007B5052917D8DFE801F019169D
:101E100003191920202383F31188104A012101900E
:101E2000FFF7CEFA019802210D4AFFF7C9FA0D48D3
:101E3000FFF7EAF9002383F3118803B05DF804FB90
:101E4000202383F311880748FFF7B4F9F2E7202332
:101E500083F311880348FFF7CBF9EBE7F03A00086A
:101E6000143B00087025002038B50C4D0C4C2A4658
:101E70000C4904F10800FFF767FF05F1CA0204F1FD
:101E800010000949FFF760FF05F5CA7204F1180058
:101E90000649BDE83840FFF757BF00BF483E002065
:101EA0003C220020D03A0008DA3A0008E53A00085F
:101EB00070B5044608460D46FEF7D6FFC6B220466A
:101EC000013403780BB9184670BD32462946FEF737
:101ED000B7FF0028F3D10120F6E700002DE9F84F05
:101EE00005460C46FEF7C0FF2C49C6B22846FFF750
:101EF000DFFF08B10536F6B229492846FFF7D8FFBB
:101F000008B11036F6B2632E0DD8DFF89080DFF8F6
:101F10009090244FDFF894A0DFF894B02E7846B963
:101F20002670BDE8F88F29462046BDE8F84F01F03D
:101F30008BBD252E2ED1072241462846FEF780FF75
:101F400070B9DBF8003007350C3444F80C3CDBF892
:101F5000043044F8083CDBF8083044F8043CDDE782
:101F6000082249462846FEF76BFF98B9A21C0E4B83
:101F7000197802320909C95D02F8041C13F8011B23
:101F800001F00F015345C95D02F8031CF0D118346C
:101F90000835C3E7013504F8016BBFE7BC3B000817
:101FA000E53A0008D13B000800E8F11F0CE8F11FFA
:101FB000C43B0008BFF34F8F044B1A695107FCD193
:101FC000D3F810215207F8D1704700BF002000520B
:101FD00008B50D4B1B78ABB9FFF7ECFF0B4BDA687C
:101FE000D10704D50A4A5A6002F188325A60D3F800
:101FF0000C21D20706D5064AC3F8042102F1883223
:10200000C3F8042108BD00BFA640002000200052F4
:102010002301674508B5114B1B78F3B9104B1A69BA
:10202000510703D5DA6842F04002DA60D3F8102194
:10203000520705D5D3F80C2142F04002C3F80C2119
:10204000FFF7B8FF064BDA6842F00102DA60D3F816
:102050000C2142F00102C3F80C2108BDA64000206B
:10206000002000520F289ABF00F580604004002035
:10207000704700004FF40030704700001020704798
:102080000F2808B50BD8FFF7EDFF00F50033026805
:10209000013204D104308342F9D1012008BD00206F
:1020A000FCE700000F2870B5054645D8FFF7D6FCC1
:1020B000224CFFF77FFF0646FFF78AFF4FF0FF3302
:1020C000072D6361C4F8143120D82361FFF772FF34
:1020D0002B0243F02403E360E36843F08003E360F2
:1020E00023695A07FCD42846FFF764FF4FF40031F8
:1020F000FFF7B8FF00F002F93046FFF78BFFFFF75C
:10210000B7FC2846BDE87040FFF7BABFC4F81031ED
:10211000FFF750FFA5F108031B0243F02403C4F8A6
:102120000C31D4F80C3143F08003C4F80C31D4F8EE
:1021300010315B07FBD4D6E7002070BD00200052B1
:102140002DE9F84F40EA020305460C461746D8062B
:1021500002D00020BDE8F88F27F01F07DFF8D4B0C9
:10216000FFF736FF2744BC4203D10120FFF752FF9F
:10217000F0E720222946204601F056FC10B9203510
:102180002034F0E72B4605F120021E68711CE0D1D7
:1021900004339A42F9D1FFF761FC05F17843234AF1
:1021A000B3F5801F224B28BF9A4603F1040338BFC2
:1021B0009046A2F1080228BF9846A3F108033ABF4F
:1021C0009146DA469946FFF7F5FEC8F80060A5EBA0
:1021D000040CD9F8002004F11C0142F00202C9F8F5
:1021E0000020221FDAF8006016F00506FAD152F836
:1021F000043F8A424CF80230F4D1BFF34F8FFFF70F
:10220000D9FE4FF0FF32C8F80020D9F8002022F0A4
:102210000202C9F80020FFF72BFC202221462846A5
:1022200001F002FC0028AAD030469FE7142000529B
:10223000102100521020005210B5084C237828B10C
:102240001BB9FFF7C5FE0123237010BD002BFCD086
:102250002070BDE81040FFF7DDBE00BFA6400020A3
:102260000244074BD2B210B5904200D110BD441CBD
:1022700000B253F8200041F8040BE0B2F4E700BFCD
:10228000504000580E4B30B51C6F240405D41C6F11
:102290001C671C6F44F400441C670A4C024423680A
:1022A000D2B243F480732360074B904200D130BD1B
:1022B000441C51F8045B00B243F82050E0B2F4E74C
:1022C00000440258004802585040005807B5012207
:1022D00001A90020FFF7C4FF019803B05DF804FBDB
:1022E00013B50446FFF7F2FFA04205D0012201A971
:1022F00000200194FFF7C6FF02B010BD0144BFF3F8
:102300004F8F064B884204D3BFF34F8FBFF36F8FBD
:102310007047C3F85C022030F4E700BF00ED00E036
:1023200000207047034B1A681AB9034AD2F8D02428
:102330001A607047A84000200040025808B5FFF717
:10234000F1FF024B1868C0F3806008BDA840002070
:10235000EFF30983054968334A6B22F001024A63AF
:1023600083F30988002383F31188704700EF00E0AE
:10237000202080F3118862B60D4B0E4AD96821F4F3
:10238000E0610904090C0A430B49DA60D3F8FC2028
:1023900042F08072C3F8FC20084AC2F8B01F1168EE
:1023A00041F0010111601022DA7783F822007047B2
:1023B00000ED00E00003FA0555CEACC5001000E0CA
:1023C000202310B583F311880E4B5B6813F4006370
:1023D00014D0F1EE103AEFF309844FF08073683CAB
:1023E000E361094BDB6B236684F30988FFF7E6FAA8
:1023F00010B1064BA36110BD054BFBE783F31188B9
:10240000F9E700BF00ED00E000EF00E0F70300088F
:10241000FA03000870B5BFF34F8FBFF36F8F1A4AEE
:102420000021C2F85012BFF34F8FBFF36F8F536973
:1024300043F400335361BFF34F8FBFF36F8FC2F884
:102440008410BFF34F8FD2F8803043F6E074C3F3AB
:10245000C900C3F34E335B0103EA0406014646EAB2
:1024600081750139C2F86052F9D2203B13F1200F77
:10247000F2D1BFF34F8F536943F480335361BFF3FD
:102480004F8FBFF36F8F70BD00ED00E0FEE70000DF
:102490000A4B0B480B4A90420BD30B4BC11EDA1C64
:1024A000121A22F003028B4238BF00220021FEF7ED
:1024B000E3BC53F8041B40F8041BECE7B43D0008F0
:1024C0007C4200207C4200207C42002070470000BB
:1024D00070B5D0E9244300224FF0FF359E6804EB2D
:1024E00042135101D3F80009002805DAD3F8000996
:1024F00040F08040C3F80009D3F8000B002805DA4B
:10250000D3F8000B40F08040C3F8000B0132631891
:102510009642C3F80859C3F8085BE0D24FF00113A4
:10252000C4F81C3870BD000000EB8103D3F80CC068
:102530002DE9F043DCF814204E1CD0F89050D2F86E
:1025400000E005EB063605EB4118506870450AD3EC
:102550000122D5F8343802FA01F123EA0101C5F865
:102560003418BDE8F083AEEB0003BCF81040A34282
:1025700028BF2346D8F81849A4B2B3EB840FF0D88B
:102580009468A4F1040959F8047F3760A4EB0907A3
:102590001F44042FF7D81C44034494605360D4E7CD
:1025A000890141F02001016103699B06FCD41220DE
:1025B000FFF76EBA10B50A4C2046FEF7DFFE094B56
:1025C000C4F89030084BC4F89430084C2046FEF70D
:1025D000D5FE074BC4F89030064BC4F8943010BDBC
:1025E000AC40002000000840083C000848410020A2
:1025F00000000440143C000870B503780546012B28
:102600005DD1494BD0F89040984259D1474B0E21AB
:102610006520D3F8D82042F00062C3F8D820D3F860
:10262000002142F00062C3F80021D3F80021D3F862
:10263000802042F00062C3F88020D3F8802022F08E
:102640000062C3F88020D3F8803000F071FC384B72
:10265000E360384BC4F800380023D5F89060C4F824
:10266000003EC02323604FF40413A3633369002B9F
:10267000FCDA01230C203361FFF70AFA3369DB0728
:10268000FCD41220FFF704FA3369002BFCDA002691
:102690002846A660FFF71CFF6B68C4F81068DB686B
:1026A000C4F81468C4F81C68002B3AD1224BA3610B
:1026B0004FF0FF336361A36843F00103A36070BD73
:1026C0001E4B9842C8D1194B0E214D20D3F8D8206B
:1026D00042F00072C3F8D820D3F8002142F0007213
:1026E000C3F80021D3F80021D3F8802042F0007213
:1026F000C3F88020D3F8802022F00072C3F8802035
:10270000D3F88020D3F8D82022F08062C3F8D820F4
:10271000D3F8002122F08062C3F80021D3F8003101
:1027200093E7074BC3E700BFAC40002000440258CA
:102730004014004003002002003C30C0484100200B
:10274000083C30C0F8B5D0F89040054600214FF065
:1027500000662046FFF724FFD5F8941000234FF0C1
:1027600001128F684FF0FF30C4F83438C4F81C28C9
:1027700004EB431201339F42C2F80069C2F8006BB8
:10278000C2F80809C2F8080BF2D20B68D5F89020FD
:10279000C5F89830636210231361166916F01006AD
:1027A000FBD11220FFF774F9D4F8003823F4FE634C
:1027B000C4F80038A36943F4402343F01003A36135
:1027C0000923C4F81038C4F814380B4BEB604FF0F1
:1027D000C043C4F8103B094BC4F8003BC4F810696F
:1027E000C4F80039D5F8983003F1100243F480138F
:1027F000C5F89820A362F8BDE43B000840800010B3
:10280000D0F8902090F88A10D2F8003823F4FE63B4
:1028100043EA0113C2F80038704700002DE9F8437D
:1028200000EB8103D0F890500C468046DA680FFA2E
:1028300081F94801166806F00306731E022B05EBAA
:1028400041134FF0000194BFB604384EC3F8101B7B
:102850004FF0010104F1100398BF06F1805601FA10
:1028600003F3916998BF06F5004600293AD0578ACC
:1028700004F15801374349016F50D5F81C180B4338
:102880000021C5F81C382B180127C3F81019A740E0
:102890005369611E9BB3138A928B9B08012A88BFE0
:1028A0005343D8F89820981842EA034301F14002B4
:1028B0002146C8F89800284605EB82025360FFF7CE
:1028C0006FFE08EB8900C3681B8A43EA84534834CF
:1028D0001E4364012E51D5F81C381F43C5F81C78DF
:1028E000BDE8F88305EB4917D7F8001B21F4004138
:1028F000C7F8001BD5F81C1821EA0303C0E704F150
:102900003F030B4A2846214605EB83035A60FFF735
:1029100047FE05EB4910D0F8003923F40043C0F816
:102920000039D5F81C3823EA0707D7E700800010E4
:1029300000040002D0F894201268C0F89820FFF735
:10294000C7BD00005831D0F8903049015B5813F4EE
:10295000004004D013F4001F0CBF02200120704778
:102960004831D0F8903049015B5813F4004004D04E
:1029700013F4001F0CBF02200120704700EB8101FF
:10298000CB68196A0B6813604B685360704700008E
:1029900000EB810330B5DD68AA691368D36019B90B
:1029A000402B84BF402313606B8A1468D0F89020BA
:1029B0001C4402EB4110013C09B2B4FBF3F4634345
:1029C000033323F0030343EAC44343F0C043C0F896
:1029D000103B2B6803F00303012B0ED1D2F808380B
:1029E00002EB411013F4807FD0F8003B14BF43F09A
:1029F000805343F00053C0F8003B02EB4112D2F881
:102A0000003B43F00443C2F8003B30BD2DE9F041E8
:102A1000D0F8906005460C4606EB4113D3F8087BCE
:102A20003A07C3F8087B08D5D6F814381B0704D535
:102A300000EB8103DB685B689847FA071FD5D6F87F
:102A40001438DB071BD505EB8403D968CCB98B6937
:102A5000488A5A68B2FBF0F600FB16228AB9186859
:102A6000DA6890420DD2121AC3E90024202383F3BE
:102A7000118821462846FFF78BFF84F31188BDE8B3
:102A8000F081012303FA04F26B8923EA02036B81CC
:102A9000CB68002BF3D021462846BDE8F04118470B
:102AA00000EB81034A0170B5DD68D0F890306C69A5
:102AB0002668E66056BB1A444FF40020C2F810099D
:102AC0002A6802F00302012A0AB20ED1D3F80808DC
:102AD00003EB421410F4807FD4F8000914BF40F0D7
:102AE000805040F00050C4F8000903EB4212D2F8C5
:102AF000000940F00440C2F800090122D3F834086C
:102B000002FA01F10143C3F8341870BD19B9402E1F
:102B100084BF4020206020681A442E8A8419013C1A
:102B2000B4FBF6F440EAC44040F00050C6E70000B1
:102B30002DE9F041D0F8906004460D4606EB4113B4
:102B4000D3F80879C3F80879FB071CD5D6F81038F4
:102B5000DA0718D500EB8103D3F80CC0DCF8143089
:102B6000D3F800E0DA6896451BD2A2EB0E024FF0D4
:102B700000081A60C3F80480202383F31188FFF74C
:102B80008FFF88F311883B0618D50123D6F8342827
:102B9000AB40134212D029462046BDE8F041FFF772
:102BA000C3BC012303FA01F2038923EA0203038170
:102BB000DCF80830002BE6D09847E4E7BDE8F08168
:102BC0002DE9F84FD0F8905004466E69AB691E406D
:102BD00016F480586E6103D0BDE8F84FFEF73EBC96
:102BE000002E12DAD5F8003E9F0705D0D5F8003E3A
:102BF00023F00303C5F8003ED5F80438204623F03F
:102C00000103C5F80438FEF755FC300505D520460C
:102C1000FFF75EFC2046FEF73DFCB1040CD5D5F86D
:102C2000083813F0060FEB6823F470530CBF43F41D
:102C3000105343F4A053EB60320704D56368DB689C
:102C40000BB120469847F30200F1BA80B70226D5AF
:102C5000D4F8909000274FF0010A09EB4712D2F800
:102C6000003B03F44023B3F5802F11D1D2F8003B91
:102C7000002B0DDA62890AFA07F322EA0303638163
:102C800004EB8703DB68DB6813B1394620469847BD
:102C90000137D4F89430FFB29B689F42DDD9F0062B
:102CA00019D5D4F89000026AC2F30A1702F00F0394
:102CB00002F4F012B2F5802F00F0CC80B2F5402F74
:102CC00009D104EB8303002200F58050DB681B6A06
:102CD000974240F0B2803003D5F8185835D5E90353
:102CE00003D500212046FFF791FEAA0303D5012159
:102CF0002046FFF78BFE6B0303D502212046FFF72A
:102D000085FE2F0303D503212046FFF77FFEE8024F
:102D100003D504212046FFF779FEA90203D505213A
:102D20002046FFF773FE6A0203D506212046FFF70F
:102D30006DFE2B0203D507212046FFF767FEEF014A
:102D400003D508212046FFF761FE700340F1A980FA
:102D5000E90703D500212046FFF7EAFEAA0703D5BD
:102D600001212046FFF7E4FE6B0703D50221204630
:102D7000FFF7DEFE2F0703D503212046FFF7D8FE1D
:102D8000EE0603D504212046FFF7D2FEA80603D5A0
:102D900005212046FFF7CCFE690603D50621204613
:102DA000FFF7C6FE2A0603D507212046FFF7C0FE1F
:102DB000EB0576D520460821BDE8F84FFFF7B8BEF1
:102DC000D4F8909000274FF0010AD4F894305FFABD
:102DD00087FB9B689B453FF639AF09EB4B13D3F854
:102DE000002902F44022B2F5802F24D1D3F8002923
:102DF000002A20DAD3F8002942F09042C3F80029D3
:102E0000D3F80029002AFBDB5946D4F89000FFF7DD
:102E1000C7FB22890AFA0BF322EA0303238104EB9E
:102E20008B03DB689B6813B1594620469847594687
:102E30002046FFF779FB0137C7E7910701D1D0F8AA
:102E40000080072A02F101029CBF03F8018B4FEAC0
:102E500018283DE704EB830300F58050DA68D2F8C8
:102E600018C0DCF80820DCE9001CA1EB0C0C0021E8
:102E70008F4208D1DB689B699A683A449A605A6825
:102E80003A445A6027E711F0030F01D1D0F80080CF
:102E90008C4501F1010184BF02F8018B4FEA18282B
:102EA000E6E7BDE8F88F000008B50348FFF788FEA5
:102EB000BDE80840FFF784BAAC40002008B50348DD
:102EC000FFF77EFEBDE80840FFF77ABA48410020D0
:102ED000D0F8903003EB4111D1F8003B43F40013DC
:102EE000C1F8003B70470000D0F8903003EB41116F
:102EF000D1F8003943F40013C1F8003970470000DD
:102F0000D0F8903003EB4111D1F8003B23F40013CB
:102F1000C1F8003B70470000D0F8903003EB41113E
:102F2000D1F8003923F40013C1F8003970470000CC
:102F3000090100F16043012203F56143C9B283F83E
:102F4000001300F01F039A4043099B0003F1604304
:102F500003F56143C3F880211A60704730B504332C
:102F6000039C0172002104FB0325C160C0E90653E4
:102F7000049B0363059BC0E90000C0E90422C0E98B
:102F80000842C0E90A11436330BD00000022416AD3
:102F9000C260C0E90411C0E90A226FF00101FEF726
:102FA000E7BD0000D0E90432934201D1C2680AB9FA
:102FB000181D704700207047036919600021C2681E
:102FC0000132C260C269134482699342036124BF23
:102FD000436A0361FEF7C0BD38B504460D46E36899
:102FE0003BB162690020131D1268A3621344E362BF
:102FF00007E0237A33B929462046FEF79DFD0028D5
:10300000EDDA38BD6FF00100FBE70000C368C2696C
:10301000013BC3604369134482699342436124BF07
:10302000436A436100238362036B03B1184770470F
:1030300070B52023044683F31188866A3EB9FFF7F2
:10304000CBFF054618B186F31188284670BDA36AE8
:10305000E26A13F8015B9342A36202D32046FFF7B2
:10306000D5FF002383F31188EFE700002DE9F84F27
:1030700004460E46174698464FF0200989F31188FA
:103080000025AA46D4F828B0BBF1000F09D141466B
:103090002046FFF7A1FF20B18BF311882846BDE839
:1030A000F88FD4E90A12A7EB050B521A934528BFF3
:1030B0009346BBF1400F1BD9334601F1400251F852
:1030C000040B914243F8040BF9D1A36A4036403512
:1030D0004033A362D4E90A239A4202D32046FFF781
:1030E00095FF8AF31188BD42D8D289F31188C9E7C8
:1030F00030465A46FDF79AFEA36A5E445D445B443F
:10310000A362E7E710B5029C0433017204FB0321BC
:10311000C460C0E906130023C0E90A33039B0363BC
:10312000049BC0E90000C0E90422C0E908424363EF
:1031300010BD0000026A6FF00101C260426AC0E97E
:1031400004220022C0E90A22FEF712BDD0E90423BE
:103150009A4201D1C26822B9184650F8043B0B606C
:103160007047002070470000C3680021C269013326
:10317000C3604369134482699342436124BF436A35
:103180004361FEF7E9BC000038B504460D46E3682C
:103190003BB1236900201A1DA262E2691344E36275
:1031A00007E0237A33B929462046FEF7C5FC0028FC
:1031B000EDDA38BD6FF00100FBE70000036919602C
:1031C000C268013AC260C2691344826993420361D2
:1031D00024BF436A036100238362036B03B1184772
:1031E0007047000070B520230D460446114683F356
:1031F0001188866A2EB9FFF7C7FF10B186F31188D0
:1032000070BDA36A1D70A36AE26A01339342A36290
:1032100004D3E16920460439FFF7D0FF002080F392
:103220001188EDE72DE9F84F04460D469046994682
:103230004FF0200A8AF311880026B346A76A4FB9D7
:1032400049462046FFF7A0FF20B187F3118830469A
:10325000BDE8F88FD4E90A073A1AA8EB06079742A7
:1032600028BF1746402F1BD905F1400355F8042B02
:103270009D4240F8042BF9D1A36A40364033A36243
:10328000D4E90A239A4204D3E16920460439FFF7BE
:1032900095FF8BF311884645D9D28AF31188CDE783
:1032A00029463A46FDF7C2FDA36A3D443E443B44ED
:1032B000A362E5E7D0E904239A4217D1C3689BB122
:1032C000836A8BB1043B9B1A0ED01360C368013B29
:1032D000C360C3691A4483699A42026124BF436A86
:1032E0000361002383620123184670470023FBE734
:1032F00000F0DAB8034B002258631A610222DA6048
:10330000704700BF000C0040014B0022DA6070479C
:10331000000C0040014B5863704700BF000C004098
:10332000014B586A704700BF000C00404B68436077
:103330008B688360CB68C3600B6943614B69036230
:103340008B6943620B6803607047000008B53C4B13
:1033500040F2FF713B48D3F888200A43C3F8882025
:10336000D3F8882022F4FF6222F00702C3F88820F5
:10337000D3F88820D3F8E0200A43C3F8E020D3F83C
:1033800008210A43C3F808212F4AD3F8083111460F
:10339000FFF7CCFF00F5806002F11C01FFF7C6FFCC
:1033A00000F5806002F13801FFF7C0FF00F5806092
:1033B00002F15401FFF7BAFF00F5806002F17001DD
:1033C000FFF7B4FF00F5806002F18C01FFF7AEFF5C
:1033D00000F5806002F1A801FFF7A8FF00F580600A
:1033E00002F1C401FFF7A2FF00F5806002F1E001E5
:1033F000FFF79CFF00F5806002F1FC01FFF796FFEC
:1034000002F58C7100F58060FFF790FF00F000F985
:103410000E4BD3F8902242F00102C3F89022D3F869
:10342000942242F00102C3F894220522C3F89820A6
:103430004FF06052C3F89C20054AC3F8A02008BD95
:103440000044025800000258203C000800ED00E053
:103450001F00080308B500F0C9FAFEF7DDFA0F4BAC
:10346000D3F8DC2042F04002C3F8DC20D3F804217A
:1034700022F04002C3F80421D3F80431084B1A6843
:1034800042F008021A601A6842F004021A60FEF75D
:1034900049FFBDE80840FEF7E7BC00BF0044025802
:1034A0000018024870470000114BD3F8E82042F0A2
:1034B0000802C3F8E820D3F8102142F00802C3F84C
:1034C00010210C4AD3F81031D36B43F00803D363B7
:1034D000C722094B9A624FF0FF32DA6200229A61EA
:1034E0005A63DA605A6001225A611A60704700BF5D
:1034F000004402580010005C000C0040094A08B566
:103500001169D3680B40D9B29B076FEA01011161C1
:1035100007D5202383F31188FEF79EFA002383F357
:10352000118808BD000C0040384B4FF0FF31D3F834
:103530008020C3F88010D3F880200022C3F88020B8
:10354000D3F88000D3F88400C3F88410D3F8840043
:10355000C3F88420D3F88400D86F40F0FF4040F4D3
:10356000FF0040F43F5040F03F00D867D86F20F094
:10357000FF4020F4FF0020F43F5020F03F00D867C8
:10358000D86FD3F888006FEA40506FEA5050C3F804
:103590008800D3F88800C0F30A00C3F88800D3F885
:1035A0008800D3F89000C3F89010D3F89000C3F8C7
:1035B0009020D3F89000D3F89400C3F89410D3F877
:1035C0009400C3F89420D3F89400D3F89800C3F87B
:1035D0009810D3F89800C3F89820D3F89800D3F83F
:1035E0008C00C3F88C10D3F88C00C3F88C20D3F86F
:1035F0008C00D3F89C00C3F89C10D3F89C10C3F83F
:103600009C20D3F89C3000F0C9B900BF0044025898
:10361000614B0122C3F80821604BD3F8F42042F03B
:103620000202C3F8F420D3F81C2142F00202C3F8CE
:103630001C210222D3F81C31594BDA605A689104DC
:10364000FCD5584A1A6001229A60574ADA60002273
:103650001A614FF440429A61514B9A699204FCD529
:103660001A6842F480721A604C4B1A6F12F4407F51
:1036700004D04FF480321A6700221A671A6842F0A9
:1036800001021A60454B1A685007FCD500221A61E6
:103690001A6912F03802FBD1012119604FF0804104
:1036A00059605A67414ADA62414A1A611A6842F41B
:1036B00080321A60394B1A689103FCD51A6842F4BB
:1036C00080521A601A689204FCD53A4A3A499A62C2
:1036D00000225A6319633949DA6399635A64384A94
:1036E0001A64384ADA621A6842F0A8521A602B4B00
:1036F0001A6802F02852B2F1285FF9D148229A6183
:103700004FF48862DA6140221A622F4ADA644FF07D
:1037100080521A652D4A5A652D4A9A6532232D4AE0
:103720001360136803F00F03022BFAD11B4B1A69C5
:1037300042F003021A611A6902F03802182AFAD11B
:10374000D3F8DC2042F00052C3F8DC20D3F8042187
:1037500042F00052C3F80421D3F80421D3F8DC204E
:1037600042F08042C3F8DC20D3F8042142F08042CA
:10377000C3F80421D3F80421D3F8DC2042F000423E
:10378000C3F8DC20D3F8042142F00042C3F804213E
:10379000D3F80431704700BF008000510044025844
:1037A0000048025800C000F0020000010000FF01C4
:1037B0000088900812102000630209012C02040006
:1037C00047040508FD0BFF01200000200010E00069
:1037D00000010100002000524FF0B04208B5D2F8BD
:1037E000883003F00103C2F8883023B1044A13681B
:1037F0000BB150689847BDE80840FEF7E1BD00BF37
:10380000FC4100204FF0B04208B5D2F8883003F0F8
:103810000203C2F8883023B1044A93680BB1D06820
:103820009847BDE80840FEF7CBBD00BFFC41002033
:103830004FF0B04208B5D2F8883003F00403C2F864
:10384000883023B1044A13690BB150699847BDE829
:103850000840FEF7B5BD00BFFC4100204FF0B0426C
:1038600008B5D2F8883003F00803C2F8883023B1D5
:10387000044A93690BB1D0699847BDE80840FEF748
:103880009FBD00BFFC4100204FF0B04208B5D2F808
:10389000883003F01003C2F8883023B1044A136A59
:1038A0000BB1506A9847BDE80840FEF789BD00BFDC
:1038B000FC4100204FF0B04310B5D3F8884004F429
:1038C0007872C3F88820A30604D5124A936A0BB114
:1038D000D06A9847600604D50E4A136B0BB1506B43
:1038E0009847210604D50B4A936B0BB1D06B9847D0
:1038F000E20504D5074A136C0BB1506C9847A30539
:1039000004D5044A936C0BB1D06C9847BDE81040C5
:10391000FEF756BDFC4100204FF0B04310B5D3F880
:10392000884004F47C42C3F88820620504D5164A16
:10393000136D0BB1506D9847230504D5124A936D52
:103940000BB1D06D9847E00404D50F4A136E0BB14C
:10395000506E9847A10404D50B4A936E0BB1D06EFC
:103960009847620404D5084A136F0BB1506F98470B
:10397000230404D5044A936F0BB1D06F9847BDE878
:103980001040FEF71DBD00BFFC41002008B5FFF749
:10399000B5FDBDE80840FEF713BD0000062108B5DF
:1039A0000846FFF7C5FA06210720FFF7C1FA0621EE
:1039B0000820FFF7BDFA06210920FFF7B9FA062112
:1039C0000A20FFF7B5FA06211720FFF7B1FA062102
:1039D0002820FFF7ADFA09217A20FFF7A9FA07217D
:1039E0003220BDE80840FFF7A3BA000008B5FFF792
:1039F0009BFD00F00BF8FDF7BFFCFDF791FBFFF717
:103A000051FDBDE80840FFF773BC00000023054AE4
:103A100019460133102BC2E9001102F10802F8D156
:103A2000704700BFFC41002010B5013902449042AC
:103A300001D1002005E0037811F8014FA34201D025
:103A4000181B10BD0130F2E7034611F8012B03F8F3
:103A5000012B002AF9D1704753544D333248373F78
:103A60003F3F0053544D3332483734332F373533CB
:103A700000000000000000009D10000889100008F0
:103A8000C5100008B1100008BD100008A9100008FA
:103A90009510000881100008D110000800000000F7
:103AA00001000000000000006D61696E0000000070
:103AB00069646C6500000000B03A0008F82300203B
:103AC0007025002001000000151A00080000000009
:103AD0004172647550696C6F740025424F415244C5
:103AE000252D424C002553455249414C25000000EC
:103AF0000200000000000000BD1200082D130008A5
:103B000040004000183E0020283E00200200000037
:103B10000000000003000000000000007513000812
:103B20000000000010000000383E002000000000EF
:103B30000100000000000000AC4000200101020074
:103B4000051E0008151D0008B11D0008951D000880
:103B500043000000583B000809024300020100C076
:103B600032090400000102020100052400100105D1
:103B70002401000104240202052406000107058235
:103B8000030800FF09040100020A00000007050104
:103B90000240000007058102400000001200000002
:103BA000A43B000812011001020000400912415715
:103BB00000020102030100000403090425424F41F1
:103BC00052442500466F7865657248373433763144
:103BD0000030313233343536373839414243444589
:103BE0004600000000000000C9140008811700080A
:103BF0002D18000840004000E4410020E44100206E
:103C000001000000F441002080000000400100009D
:103C1000080000000001000000040000080000008F
:103C20000001816A00000000AAAAAAAA000100649B
:103C3000FFFE00000000000000A00A0000000001DC
:103C400000000000AAAAAAAA00000001FFFF0000CD
:103C50000000000000000000000000000000000064
:103C6000AAAAAAAA00000000FFFF000000000000AE
:103C7000000000000000000000000000AAAAAAAA9C
:103C800000000000FFFF0000000000000000000036
:103C90000000000000000000AAAAAAAA000000007C
:103CA000FFFF000000000000000000000000000016
:103CB00000000000AAAAAAAA00000000FFFF00005E
:103CC00000000000000000000000000000000000F4
:103CD000AAAAAAAA00000000FFFF0000000000003E
:103CE000000000000000000000000000AAAAAAAA2C
:103CF00000000000FFFF00000000000000000000C6
:103D00000000000000000000AAAAAAAA000000000B
:103D1000FFFF0000000000000000000000000000A5
:103D200000000000AAAAAAAA00000000FFFF0000ED
:103D30000000000000000000000000000000000083
:103D4000AAAAAAAA00000000FFFF000000000000CD
:103D5000000000000000000041040000000000001E
:103D600000001A0000000000FF000000000000003A
:103D7000583A00083F00000050040000633A000871
:103D80003F000000009600000000080096000000C0
:103D90000008000004000000B83B0008000000001C
:103DA0000000000000000000000000000000000013
:103DB00000000000FFFFFFFFFFFFFFFFFFFFFFFF0F
:103DC000FFFFFFFFFFFFFFFFFFFFFFFFFFFFFFFF03
:103DD000FFFFFFFFFFFFFFFFFFFFFFFFFFFFFFFFF3
:103DE000FFFFFFFFFFFFFFFFFFFFFFFFFFFFFFFFE3
:103DF000FFFFFFFFFFFFFFFFFFFFFFFFFFFFFFFFD3
:020000040805ED
:020000040806EC
:10000000000600308D0D0608E98512084103060838
:1000100071851208698512086D8512088F0D060812
:100020008F0D06088F0D06088F0D0608C1AD150847
:100030008F0D06088F0D06088F0D06088F0D060818
:100040008F0D06088F0D06088F0D06088F0D060808
:100050008F0D06088F0D0608C1C31508EDC31508DE
:1000600019C4150845C4150871C415087567150825
:100070009D671508C9671508F567150821681508F3
:100080004968150875681508996315088F0D0608E5
:100090008F0D06088F0D06088F0D06089DC41508E4
:1000A0008F0D060801C615088F0D060815C6150820
:1000B0008F0D060819C615082DC615086D6E150892
:1000C000956F15088F0D06088F0D0608BD7215086F
:1000D000D572150875C5150889C515089DC515087B
:1000E00001C515088F0D06088F0D060851C61508A5
:1000F00055C6150869C615086DC61508A168150806
:100100008F0D06088F0D060841C61508ED721508FB
:10011000B1C515088F0D06088F0D06088F0D06084E
:10012000CD681508F5681508216915084D69150889
:10013000796915088F0D06088F0D06088F0D0608C2
:100140008F0D06088F0D06088F0D06088F0D060807
:10015000A1691508CD691508F9691508C5C51508FF
:100160008F0D06088F0D06088F0D06088F0D0608E7
:100170008F0D0608ADB915088F0D06088F0D0608FE
:100180008F0D06088F0D0608D9C51508EDC5150891
:100190008F0D06088F0D06088F0D06088F0D0608B7
:1001A0008F0D06088F0D06088F0D06088F0D0608A7
:1001B0008F0D06088F0D06088F0D06088F0D060897
:1001C0008F0D06088F0D06088F0D06088F0D060887
:1001D0008F0D060899B915088F0D06088F0D0608B2
:1001E0008F0D06088F0D06088F0D06088F0D060867
:1001F0008F0D06088F0D06088F0D06088F0D060857
:100200008F0D06088F0D06088F0D06088F0D060846
:100210008F0D06088F0D06088F0D06088F0D060836
:100220008F0D06088F0D06088F0D06088F0D060826
:100230008F0D06088F0D06088F0D0608B963150887
:100240008F0D06084165150869651508956515083F
:10025000C1651508ED651508196615084566150888
:10026000716615088F0D06088F0D06088F0D06089C
:100270008F0D06088F0D06088F0D06088F0D0608D6
:100280008F0D06088F0D06088F0D06088F0D0608C6
:100290008F0D06088F0D06088F0D06088F0D0608B6
:1002A0008F0D06088F0D06088F0D06088F0D0608A6
:1002B0008F0D06088F0D06088F0D06088F0D060896
:1002C0008F0D06088F0D06088F0D06088F0D060886
:1002D0008F0D06088F0D06088F0D06088F0D060876
:1002E000253F06082978060891BA0608D121070893
:1002F000418A0708C92C0808D5200A0849730C0848
:1003000055790C081DF00C08F54C0D08BD540D086E
:10031000FD570D0845CF0D0895F30D08D1480F087E
:1003200031E40F08217F1208CD1A1408C1B7140850
:1003300055DF140831F61408B1271508D12D15081A
:10034000EFF30383EFF30982EFF30881DFF814D0B2
:100350002DE9FE4F684600F0E3FFBDE8FE4F8D46F5
:100360007047000074320030F1EE101AA0EC200A41
:1003700001607047A0EC108A704700BF81F0004117
:1003800002E000BF83F0004330B54FEA41044FEA7A
:10039000430594EA050F08BF90EA020F1FBF54EA15
:1003A000000C55EA020C7FEA645C7FEA655C00F0B1
:1003B000E2804FEA5454D4EB5555B8BF6D420CDD82
:1003C0002C4480EA020281EA030382EA000083EA05
:1003D000010180EA020281EA0303362D88BF30BDA5
:1003E00011F0004F4FEA01314FF4801C4CEA1131FB
:1003F00002D0404261EB410113F0004F4FEA03335A
:100400004CEA133302D0524263EB430394EA050FE4
:1004100000F0A780A4F10104D5F1200E0DDB02FA53
:100420000EFC22FA05F2801841F1000103FA0EF2E7
:10043000801843FA05F359410EE0A5F120050EF1AD
:10044000200E012A03FA0EFC28BF4CF0020C43FADE
:1004500005F3C01851EBE37101F0004507D54FF0EB
:10046000000EDCF1000C7EEB00006EEB0101B1F53B
:10047000801F1BD3B1F5001F0CD349085FEA300081
:100480004FEA3C0C04F101044FEA445212F5800F8C
:1004900080F09A80BCF1004F08BF5FEA500C50F129
:1004A000000041EB045141EA050130BD5FEA4C0C0C
:1004B000404141EB0101013C28BFB1F5801FE9D269
:1004C00091F0000F04BF01460020B1FA81F308BF8C
:1004D0002033A3F10B03B3F120020CDA0C3208DD58
:1004E00002F1140CC2F10C0201FA0CF021FA02F133
:1004F0000CE002F11402D8BFC2F1200C01FA02F1A3
:1005000020FA0CFCDCBF41EA0C019040E41AA2BFC7
:1005100001EB0451294330BD6FEA04041F3C1CDA8F
:100520000C340EDC04F11404C4F1200220FA04F0AF
:1005300001FA02F340EA030021FA04F345EA030159
:1005400030BDC4F10C04C4F1200220FA02F001FA1B
:1005500004F340EA0300294630BD21FA04F029469D
:1005600030BD94F0000F83F4801306BF81F4801136
:100570000134013D4EE77FEA645C18BF7FEA655CA9
:1005800029D094EA050F08BF90EA020F05D054EA7B
:10059000000C04BF1946104630BD91EA030F1EBF80
:1005A0000021002030BD5FEA545C05D14000494184
:1005B00028BF41F0004130BD14F580043CBF01F577
:1005C000801130BD01F0004545F0FE4141F470015D
:1005D0004FF0000030BD7FEA645C1ABF1946104638
:1005E0007FEA655C1CBF0B46024650EA013406BF39
:1005F00052EA033591EA030F41F4002130BD00BFF8
:1006000090F0000F04BF0021704730B54FF48064B4
:1006100004F132044FF000054FF0000150E700BF35
:1006200090F0000F04BF0021704730B54FF4806494
:1006300004F1320410F0004548BF40424FF0000181
:100640003EE700BF42004FEAE2014FEA31014FEAC4
:1006500002701FBF12F07F4393F07F4F81F0605113
:10066000704732F07F4208BF704793F07F4F04BF5E
:1006700041F40021704730B54FF4607401F000453B
:1006800021F000411CE700BF50EA010208BF70479B
:1006900030B54FF000050AE050EA010208BF70478C
:1006A00030B511F0004502D5404261EB41014FF4F5
:1006B000806404F132045FEA915C3FF4D8AE4FF0FD
:1006C00003025FEADC0C18BF03325FEADC0C18BFE0
:1006D000033202EBDC02C2F1200300FA03FC20FA31
:1006E00002F001FA03FE40EA0E0021FA02F114447E
:1006F000BDE600BF80F0004002E000BF81F0004195
:1007000042001FBF5FEA410392EA030F7FEA226CB7
:100710007FEA236C6AD04FEA1262D2EB1363C1BF47
:10072000D218414048404140B8BF5B42192B88BFB6
:10073000704710F0004F40F4000020F07F4018BFD9
:10074000404211F0004F41F4000121F07F4118BFF9
:10075000494292EA030F3FD0A2F1010241FA03FCA1
:1007600010EB0C00C3F1200301FA03F100F0004389
:1007700002D5494260EB4000B0F5000F13D3B0F151
:10078000807F06D340084FEA310102F10102FE2AC0
:1007900051D2B1F1004F40EBC25008BF20F0010030
:1007A00040EA03007047490040EB0000013A28BFCF
:1007B000B0F5000FEDD2B0FA80FCACF1080CB2EB52
:1007C0000C0200FA0CF0AABF00EBC25052421843D0
:1007D000BCBFD0401843704792F0000F81F4000175
:1007E00006BF80F400000132013BB5E74FEA410348
:1007F0007FEA226C18BF7FEA236C21D092EA030FB4
:1008000004D092F0000F08BF0846704790EA010F2D
:100810001CBF0020704712F07F4F04D1400028BF5A
:1008200040F00040704712F100723CBF00F500003C
:10083000704700F0004343F0FE4040F40000704772
:100840007FEA226216BF08467FEA2363014642021E
:1008500006BF5FEA412390EA010F40F48000704731
:100860004FF0000304E000BF10F0004348BF4042D7
:100870005FEA000C08BF704743F0964301464FF013
:1008800000001CE050EA010208BF70474FF000036F
:100890000AE000BF50EA010208BF704711F00043B0
:1008A00002D5404261EB41015FEA010C02BF844680
:1008B0000146002043F0B64308BFA3F18053A3F5DF
:1008C0000003BCFA8CF2083AA3EBC25310DB01FA26
:1008D00002FC634400FA02FCC2F12002BCF1004FAA
:1008E00020FA02F243EB020008BF20F0010070473B
:1008F00002F1200201FA02FCC2F1200250EA4C008F
:1009000021FA02F243EB020008BF20EADC707047D4
:100910007BB972B90029BEBF00204FF0004106E04C
:1009200008BF00281CBF6FF000414FF0FF3000F0FF
:100930002BBAADF1080C6DE904CE002909DB002BC0
:100940001ADB00F0B9F8DDF804E0DDE9022304B0B9
:100950007047404261EB4101002B1BDB00F0ACF81B
:10096000DDF804E0DDE9022304B0404261EB41011F
:10097000524263EB43037047524263EB430300F080
:100980009BF8DDF804E0DDE9022304B0404261EBAE
:1009900041017047524263EB430300F08DF8DDF8EC
:1009A00004E0DDE9022304B0524263EB43037047E5
:1009B00053B94AB9002908BF00281CBF4FF0FF31C6
:1009C0004FF0FF3000F0E0B9ADF1080C6DE904CE56
:1009D00000F072F8DDF804E0DDE9022304B07047AE
:1009E000430803F05533C01A830803F0333300F093
:1009F0003330184400EB101000F00F3000EB0020F3
:100A000000EB0040000E704708B502460B4643EC71
:100A1000172BB5EEC07BF1EE10FA03D4BDE8084009
:100A200000F02AB8B1EE477B51EC170B00F024F828
:100A3000404261EB410108BD9FED0B6B07EE900A50
:100A40009FED0B5BB7EEE77A27EE066BBCEEC66B4D
:100A5000B8EE464BA4EE457BFCEEC77B16EE101AB3
:100A600017EE900A704700BF000000000000F03D44
:100A7000000000000000F0419FED0B6B41EC170BF4
:100A80009FED0B5B27EE066BBCEEC66BB8EE464BDC
:100A9000A4EE457BFCEEC77B16EE101A17EE900A0B
:100AA000704700BFAFF30080000000000000F03D81
:100AB000000000000000F0412DE9F047089D0446C9
:100AC0008E46002B4DD18A42944669D9B2FA82F201
:100AD00052B101FA02F3C2F1200120FA01F10CFA3D
:100AE00002FC41EA030E94404FEA1C48210CBEFB75
:100AF000F8F61FFA8CF708FB16E341EA034306FBFE
:100B000007F199420AD91CEB030306F1FF3080F08C
:100B10001F81994240F21C81023E63445B1AA4B2D9
:100B2000B3FBF8F008FB103344EA034400FB07F77B
:100B3000A7420AD91CEB040400F1FF3380F00A81BC
:100B4000A74240F207816444023840EA0640E41BB1
:100B500000261DB1D4400023C5E900433146BDE85D
:100B6000F0878B4209D9002D00F0EF800026C5E9FF
:100B7000000130463146BDE8F087B3FA83F6002E17
:100B80004AD18B4202D3824200F2F980841A61EB8F
:100B9000030301209E46002DE0D0C5E9004EDDE7AD
:100BA00002B9FFDEB2FA82F2002A40F09280A1EB95
:100BB0000C014FEA1C471FFA8CFE0126200CB1FBEA
:100BC000F7F307FB131140EA01410EFB03F08842E3
:100BD00008D91CEB010103F1FF3802D2884200F270
:100BE000CB804346091AA4B2B1FBF7F007FB101102
:100BF00044EA01440EFB00FEA64508D91CEB0404A0
:100C000000F1FF3102D2A64500F2BB800846A4EBFA
:100C10000E0440EA03409CE7C6F12007B34022FAE5
:100C200007FC4CEA030C20FA07F401FA06F31C4314
:100C3000F9404FEA1C4900FA06F3B1FBF9F8200C21
:100C40001FFA8CFE09FB181140EA014108FB0EF067
:100C5000884202FA06F20BD91CEB010108F1FF3AB7
:100C600080F08880884240F28580A8F102086144C3
:100C7000091AA4B2B1FBF9F009FB101144EA0141D1
:100C800000FB0EFE8E4508D91CEB010100F1FF347C
:100C90006CD28E456AD90238614440EA0840A0FB14
:100CA0000294A1EB0E01A142C846A64656D353D0EA
:100CB0005DB1B3EB080261EB0E0101FA07F722FA0E
:100CC00006F3F1401F43C5E9007100263146BDE837
:100CD000F087C2F12003D8400CFA02FC21FA03F39A
:100CE000914001434FEA1C471FFA8CFEB3FBF7F01B
:100CF00007FB10360B0C43EA064300FB0EF69E4240
:100D000004FA02F408D91CEB030300F1FF382FD2D8
:100D10009E422DD9023863449B1B89B2B3FBF7F680
:100D200007FB163341EA034106FB0EF38B4208D959
:100D30001CEB010106F1FF3816D28B4214D9023E9A
:100D40006144C91A46EA004638E72E46284605E7B8
:100D50000646E3E61846F8E64B45A9D2B9EB020889
:100D600064EB0C0E0138A3E74646EAE7204694E719
:100D70004046D1E7D0467BE7023B614432E730464C
:100D800009E76444023842E7704700BF02E000F020
:100D900000F8FEE772B6374880F30888364880F3DB
:100DA000098836483649086040F20000CCF200005D
:100DB0004EF63471CEF200010860BFF34F8FBFF3DF
:100DC0006F8F40F20000C0F2F0004EF68851CEF274
:100DD00000010860BFF34F8FBFF36F8F4FF000002B
:100DE000E1EE100A4EF63C71CEF2000108600620DA
:100DF00080F31488BFF36F8FFAF044F8FBF0D4F857
:100E00004FF055301F491B4A91423CBF41F8040B3B
:100E1000FAE71D49184A91423CBF41F8040BFAE732
:100E20001A491B4A1B4B9A423EBF51F8040B42F829
:100E3000040BF8E700201849184A91423CBF41F8DA
:100E4000040BFAE7FAF05CF8FBF032F9144C154D9C
:100E5000AC4203DA54F8041B8847F9E702F0C6FFF6
:100E6000114C124DAC4203DA54F8041B8847F9E7E1
:100E7000FAF044B8000600300022003000000608F6
:100E800008ED00E00000003000060030D8751908B9
:100E9000002200307C30003080300030B8D4013087
:100EA000E00206084003060840030608400306085F
:100EB0002DE9F04F2DED108AC1F80CD0D0F80CD0F0
:100EC000BDEC108ABDE8F08F002383F3118828461B
:100ED000A0470020F8F066FEFEE7F8F0D5FC00DF42
:100EE000FEE7000070B54FF0FF0C4CF4E06C1CEA1C
:100EF00011541DBF1CEA135594EA0C0F95EA0C0F10
:100F000000F0DEF82C4481EA030621EA4C5123EA82
:100F10004C5350EA013518BF52EA033541F48011B1
:100F200043F4801338D0A0FB02CE4FF00005E1FB64
:100F300002E506F00042E0FB03E54FF00006E1FBAE
:100F400003569CF0000F18BF4EF0010EA4F1FF04F1
:100F5000B6F5007F64F5407404D25FEA4E0E6D4131
:100F600046EB060642EAC62141EA55514FEAC52042
:100F700040EA5E504FEACE2EB4F1FD0C88BFBCF5BE
:100F8000E06F1ED8BEF1004F08BF5FEA500E50F16F
:100F9000000041EB045170BD06F0004646EA010135
:100FA00040EA020081EA0301B4EB5C04C2BFD4EB67
:100FB0000C0541EA045170BD41F480114FF0000E60
:100FC000013C00F3AB8014F1360FDEBF002001F0CE
:100FD000004170BDC4F10004203C35DA0C341BDC48
:100FE00004F11404C4F1200500FA05F320FA04F01A
:100FF00001FA05F240EA020001F0004221F000414E
:1010000010EBD37021FA04F642EB06015EEA430EC0
:1010100008BF20EAD37070BDC4F10C04C4F12005F0
:1010200000FA04F320FA05F001FA04F240EA0200A3
:1010300001F0004110EBD37041F100015EEA430E74
:1010400008BF20EAD37070BDC4F1200500FA05F294
:101050004EEA020E20FA04F301FA05F243EA020313
:1010600021FA04F001F0004121FA04F220EA020022
:1010700000EBD3705EEA430E08BF20EAD37070BD68
:1010800094F0000F0FD101F00046400041EB010148
:1010900011F4801F08BF013CF7D041EA060195F02A
:1010A000000F18BF704703F00046520043EB0303E4
:1010B00013F4801F08BF013DF7D043EA06037047D1
:1010C00094EA0C0F0CEA135518BF95EA0C0F0CD0DC
:1010D00050EA410618BF52EA4306D1D181EA030122
:1010E00001F000414FF0000070BD50EA410606BF1C
:1010F0001046194652EA430619D094EA0C0F02D161
:1011000050EA013613D195EA0C0F05D152EA0336A5
:101110001CBF104619460AD181EA030101F00041C3
:1011200041F0FE4141F470014FF0000070BD41F00C
:10113000FE4141F4780170BD4FEA410212F5001200
:1011400015D211D56FF47873B3EB625212D94FEA0E
:10115000C12343F0004343EA505311F0004F23FAF8
:1011600002F018BF404270474FF00000704750EA4D
:10117000013005D111F0004008BF6FF0004070470A
:101180004FF00000704700BF4FEA4102B2F1E04368
:1011900024BFB3F5001CDCF1FE5C0DD901F0004C5E
:1011A0004FEAC0024CEA5070B2F1004F40EB8300AE
:1011B00008BF20F00100704711F0804F21D113F1DA
:1011C0003872BCBF01F00040704741F480114FEA13
:1011D0005252C2F11802C2F1200C10FA0CF320FA9C
:1011E00002F018BF40F001004FEAC1234FEAD323B9
:1011F00003FA0CFC40EA0C0023FA02F34FEA430323
:10120000CCE77FEA625307D150EA01331EBF4FF0AB
:10121000FE4040F44000704701F0004040F0FE40C6
:1012200040F40000704700BF01F0FF01102A2BDBE3
:1012300010F0070F08D010F8013B013A8B422DD077
:1012400010F0070F42B3F6D1F0B441EA012141EAB0
:10125000014122F007047FF000070023F0E8025666
:10126000083C85EA010586EA010685FA47F5A3FAF6
:1012700087F586FA47F6A5FA87F68EB9EED1F0BC67
:1012800001F0FF0102F0070232B110F8013B013A10
:1012900083EA010313B1F8D1002070470138704789
:1012A000002D06BF35460338073815F0010F07D16A
:1012B000013015F4807F02BF013015F4C03F0130CA
:1012C000F0BC0138704700BF10F8012B11F8013B4A
:1012D000012A28BF9A42F7D0D01A7047034613F864
:1012E000012B002AFBD1181A0138704710B50446AB
:1012F00020461CB154F80C3B013300D110BD08222C
:10130000012100F071FB54F80C0C54F8082C14F86F
:10131000041C121AB2FBF1F200F066FBE8E70000D1
:10132000C26AD0E9003112F0040F2DE9F04118BF74
:101330000B46A6B00021594C042601270291CDE9A5
:101340000003D0064CBF03F1200203F168020392B0
:10135000DA690399D2099B6902F004021B880A43E7
:1013600003F47F4303924FF0E022A3F53E41D2F80D
:10137000882D02F4A002B2F5A00F04BF0122029250
:101380004B424B410493464D03A82C6000F02AFACF
:1013900004220121434800F027FB0422012102A876
:1013A00000F022FB10220121019800F01DFB0098A3
:1013B000202201210C3000F017FB019804220121AA
:1013C000103000F011FB0422012103A800F00CFBF7
:1013D00001980C220121143000F006FB0C2201219F
:1013E000009800F001FB029BDA071FD5009BDB6A27
:1013F000DB064ED415A8FEF7BDFFDDF804C00DF1E5
:10140000140E0CF120030CF160081868083353F82F
:10141000041C7246434503C29646F6D1DCF86030A0
:1014200025938422012105A800F0DEFA00F0C0F81F
:10143000FFF75CFF4FF0E023D3F8003D03F4702387
:10144000B3F5402F0ED0184B05A88DF81C600593FE
:1014500014338DF8287006934FF0FF33CDE908332D
:10146000FFF744FF2B68A34206D0104B0422012152
:1014700005A8059300F0B8FA00F02AFA002882D0F7
:10148000049B1BB1019A93690233936126B0BDE8B6
:10149000F08105A8FEF768FFC3E700BFED55CEACAD
:1014A00080300030B44C160828ED00E0ACCE55ED8D
:1014B00037B50E4D2A78202A15D10D4C0D482368DA
:1014C0000D4918440192F8F091FF23680021019A18
:1014D0002033094829702360FFF04AF803B0BDE8C3
:1014E0003040F9F037BC03B030BD00BF743200307B
:1014F0009C320030608419087632003008B526200E
:10150000F6F05AFE144BD3F8902042F40032C3F8A0
:101510009020D3F8902022F40032C3F89020D3F822
:101520009020D3F8E82042F40032C3F8E820D3F842
:10153000102142F40032C3F810216D22D3F810318B
:10154000064BDA604FF0FF321A620D221A60012258
:10155000034B1A7008BD00BF00440258004400400D
:10156000AC320030014B1868704700BFFCFF1F0809
:10157000014B0248C01A7047608419080000200817
:10158000004870476084190807490022074B5B1A1E
:101590009A4201D30120704751F8040B013001D168
:1015A0000432F5E700207047608419080000200825
:1015B0005E4B2DE9F74F1A6802255D4B02F56A581C
:1015C000DFF894911A7808F118085A4F5A4C904451
:1015D000DFF888A1F8F07CF8A9EB070B06460EB1FE
:1015E0004E2D49D9A9EB0702B2EB080700F1928012
:1015F0004E2D00F28F80DFF868C16B1C4F4E0C211E
:10160000DBB2ACEB06006943B84273DD60184FF003
:10161000010C665090463E4480F808C04660B2EB2C
:10162000080213D44F2B11D0454E19464548AB1C28
:10163000351ADBB295424FF00C0505FB01F163DD75
:1016400065180126024460502E726A600C22012146
:101650005343E21811724FF0FF31E15051603A4BA1
:101660001B782BB1394B1B682360394B1B686360B7
:10167000314803B0BDE8F08F336AF06953450ABFC3
:10168000344BF31AA3EB0A0380B10193F9F09CF8F1
:10169000019B58B12A460C2101354A430121EDB284
:1016A000A0180172F169A1500D3141600C20012197
:1016B000984400FB05FCD84504EB0C0244F80C6090
:1016C00006F13C0C1172C2F804C005EB010205F1F1
:1016D0000205D2B2EDB200FB02F204EB020001728D
:1016E000316AA1501944416014D23046F8F000F834
:1016F000064674E767184FF0010E8044665087F87D
:1017000008E0C7F804C08AE7621801256050157226
:1017100056609BE74F2D01D82B4697E7012384F8AD
:10172000BC334FF0FF33C4E9ED3398E79C3200300F
:101730007432003060841908042200308030003098
:1017400000000430B8D4013000220030A032003054
:1017500098320030002200300000200800060030DF
:10176000B8D401300C4B1B7810B50BB9FFF7C6FE8F
:1017700000230A490A48CA699206FCD54A6A1C5CD9
:10178000D2B2944205D10133DBB20E2BF3D100204B
:1017900010BD0023EFE700BFAC3200300044004032
:1017A000B84C160838B5084B04461B780BB9FFF740
:1017B000A5FEE4B2054DAC62EB695B0600D538BD11
:1017C000F9F0C8FAF8E700BFAC320030004400403E
:1017D00010B5441E14F8010F00B910BDFFF7E2FF69
:1017E000F8E7000070B502680446EFF30581D920E0
:1017F0005369C9B2C6F0BEFE294B1B78A3B1294B71
:1018000094E8030083E803002748FFF7E1FF6368DB
:10181000B3B12648FFF7DCFF2548FFF7D9FFFFF7F4
:10182000A1FF2448FFF7D4FF234D2B783BB1246858
:101830001CB12046F8F0C8FF20B900232B7070BD02
:101840001E48E7E720461E4EF8F0D2FF00F2145083
:1018500084421FD22046F8F0CBFF30602046194E5C
:10186000F8F0DAFF04F5E053834217D92046F8F088
:10187000D3FF30600023144A1360144A1370FFF73B
:1018800083FE0028D9D0F9F065FA0120BDE8704048
:10189000F8F034BEA4F214533360DFE73360E9E7B5
:1018A00075320030A4320030C84C1608CD4C1608F2
:1018B000DE4C1608CA4C160800220030D84C160818
:1018C000A0320030983200309C3200307432003048
:1018D000284B1A7870B542B12748FFF779FF274B9C
:1018E0005868003818BF012070BD254A10780028BC
:1018F0003CD0244E244C33682448254D1A1D2178B1
:101900002D1A0A44AA4205D3224A4FF0FF31D16171
:10191000202222702278D2B103F120018D4205D815
:101920001F2A9FBF1B4AD3612022227020221949FF
:101930001844F8F05BFD3268237800211548134401
:10194000202221703360FEF013FEF9F003FA3368B1
:101950009D4207D90F4920220F48CB61F8F046FD80
:10196000F9F0F8F90020F8F0C9FDB8E701221A7083
:10197000BAE700BF75320030244D1608A43200309B
:10198000002200309C32003074320030608419082C
:101990000000200876320030E0FF1F082DE9F843F0
:1019A00007460E460024DFF83890DFF83880B4424E
:1019B00001D1BDE8F88324B1230702D14846FFF7DF
:1019C00007FF3D5D01342B0905F00F0518F80300F2
:1019D000FFF7E8FE18F80500FFF7E4FEE7E700BFB1
:1019E000CA4C1608344D1608474B1B782DE9F74FA3
:1019F00007460E4690465BB1022925D0042938D00F
:101A0000012902D11146FFF7C9FF4048FFF7E0FE68
:101A10003F4B1B78002B4ED03E4A00253E4BA2EB9D
:101A2000030938E037F81430ADF8043024B1620708
:101A300002D12846FFF7CCFE0134022101A8FFF7AE
:101A4000ADFFA045EED1E0E70024304DF9E757F8AF
:101A50002430019324B1A30702D12846FFF7B8FE32
:101A6000042101340DEB0100FFF798FFA045EED1F2
:101A7000CBE70024254DF9E7FFF71AFD022E1DD014
:101A8000042E2CD0012E06D12378795D5A1C2270A9
:101A9000224AD1540135A8450DD0214B214C1B6859
:101AA0002278043313444B45E6D31C4B4FF0FF32EE
:101AB000DA612023237003B0BDE8F08F2378DFF8CC
:101AC0005CA05A1C22703A780AF80320FFF7F0FC59
:101AD00023785A1C227000220AF80320DAE74FF01C
:101AE000000ADFF838B022783B78511C23FA0AF359
:101AF0000AF1080A21700BF80230FFF7D9FCBAF19D
:101B0000200FF0D1C6E700BF75320030CA4C16086E
:101B1000002200300000200860841908763200306E
:101B20009C32003074320030036800221B68184772
:101B30007FB5039140210546B2F048F9039A18B9E0
:101B40000124204604B070BD134E039296F9B236BC
:101B5000002BF5D07BF02EFC437A039A53B97BF02F
:101B600029FC847A039A2CB90C4B40212846B2F008
:101B700035F9E6E70A4BB6F9B416D3F88433B3F96E
:101B800006309942DCDD074B4021284600240093B3
:101B9000054BB2F023F9D4E7B0620030484D160887
:101BA000B0820030674D1608554D1608F0B50D4649
:101BB0009DB020210446B2F009F9002800F0AD8064
:101BC000574E96F9B236BBB106F50052B6F9B436A7
:101BD000D2F88423B2F90A1003F10A02914203DD1C
:101BE00040F28D32934207DC4E4B2A46202120469C
:101BF000B2F0F4F800208EE096F9A136022B05D160
:101C0000494B2A4620212046B2F0E8F8B6F874364F
:101C100041F65832A3F57A739BB293420FD8434FE3
:101C200006F5DC62D7F8243392ED007AD3ED097A19
:101C3000B4EEE77AF1EE10FA03DD3D4BD5E73D4B0C
:101C4000D3E706F2E462D3ED0B7A92ED007AB4EEBC
:101C5000E77AF1EE10FAF0DCB6F9AE36002B01DCD3
:101C6000354BC2E7A7F5405393F89C210D2A06D8BF
:101C70000123934013F4215F01D0304BB5E7304886
:101C800011F03AFE012806D1D7F83003BAF0C6FDAC
:101C900048B1012810D02B4B93F8ED1711F010012B
:101CA0001FD0294BA1E7294B0093294B2A4620211D
:101CB0002046B2F093F89DE7224B93F8983373B126
:101CC0001921244866F0E2F848B1D6F88C6619214B
:101CD000204866F001F98642DDDD1F4BE4E71F4B2B
:101CE000E2E7602204A80391FEF042FC642303AA09
:101CF0001B49D7F82C03B8F019FF18B903AB0093B0
:101D0000184BD3E7642303AA1749D7F82403B5F087
:101D100093FC0028F2D01DB0F0BD0120FBE700BF0E
:101D2000B0620030704D1608834D1608B0A2003026
:101D3000BB4D1608AB4D1608D54D1608EA4D1608D2
:101D400088B20030B0820030644E16082F4E16085C
:101D50000A4E1608484200304E4E16083F4E1608EE
:101D6000794E16087D4E16088F4E160870B59AB03B
:101D70000E4600216022054602A80191FEF0F8FB04
:101D8000642201A9094893F029F8044640B99DF955
:101D9000043043B9064B074A31462846B2F028FAC8
:101DA00020461AB070BD01ABF5E700BF9C83003040
:101DB000944E1608BEB1160807B50448BCF03EFBA9
:101DC00000F0010003B05DF804FB00BFB8A50030CF
:101DD0002DE9F043DFF844910446A5B00D46D9F84B
:101DE000D40703681B699847804619F0E7FE002175
:101DF000074660220CA80B91FEF0BAFB64230BAAE5
:101E00004146384619F06EF9064648B90BAB394AD7
:101E100029462046B2F0ECF9304625B0BDE8F08303
:101E2000354890F0C5FFB8F1000F03D194F91E308A
:101E3000012B0AD1314815F02FFF80B9304A2946CD
:101E400020460026B2F0D4F9E6E710F0060FE3D002
:101E5000A9F5A04015F020FF08B92A4AEFE703A929
:101E6000384618F093FD28B19DF80D305B0601D57A
:101E7000254AE4E7DFF8A8800023D8ED007AF5EEE4
:101E8000C07AF1EE10FAC7DD0DF12009089309932D
:101E900005AA0A9307AB04A93846019306ABCDF80F
:101EA000009019F065FB48463CF0C0FDD8ED007A83
:101EB000B4EEE70AF1EE10FA01DB144ABFE79DED3C
:101EC000057AF4EEC77AF1EE10FA01D8104AB6E7B7
:101ED0009DED047AF4EEC77AF1EE10FA01D80D4ABE
:101EE000ADE79DED067AF4EEC77AF1EE10FA93D8DD
:101EF000094AA4E7A790180824660030B0320030E1
:101F0000AC4E1608C34E1608E94E1608F74E1608D2
:101F10000C4F1608224F1608384F1608B0820030B2
:101F20008069003008B5064B93F8ED379B0704D560
:101F3000044AB2F05DF9002008BD0120FCE700BFB3
:101F4000B08200304C4F160870B50E469AB0202172
:101F50000546B1F03BFF18B9012420461AB070BD08
:101F6000C1F01AFB04460028F6D00021602202A826
:101F70000191FEF0FDFA2046642201A9C1F0D4FAD5
:101F800004460028E8D101AB024A31462846B2F0A7
:101F90002FF9E2E7BEB1160870B50C4C05460E46A7
:101FA000D4F8D40703685B69984710B10124204630
:101FB00070BDA4F5A04015F081FE04460028F5D1BF
:101FC000034A31462846B2F013F9F0E7B0820030F8
:101FD0005C4F16082DE9704E4B4E9BB082468B46E7
:101FE000D6F8F83793F8CB5065B9484B1B68986A18
:101FF00003685B6B9847044640B9454A59465046CA
:10200000B2F0F6F828461BB0BDE8708E7BF0D2F92E
:1020100020217CF087FB58B17BF0CCF91F217CF0AC
:1020200081FB80B300243B4A59465046B2F0E0F8A9
:1020300096F8CA3703F01403142B05D10024364A4E
:1020400059465046B2F0D4F859465046B3F050F8CD
:1020500000216022884202A8019108BF0C46FEF0D0
:1020600087FAD6F8F80701AA642103681B68984725
:10207000054680B92C4601AB284A59465046B2F075
:10208000B7F82546BEE77BF095F9A5217CF04AFB21
:102090000028C7D1CCE7002CF3D0DAF808303BB9E0
:1020A000DAF80030594650469B6B98470446E8E7FB
:1020B00059465046FFF77AFD814659465046FFF78C
:1020C00055FE09EA00005946C4B25046FFF72AFF00
:1020D000594604405046FFF737FF594604405046E2
:1020E000FFF726FD594604405046FFF755FF594675
:1020F00004405046B2F09EF9594604405046B3F0B1
:102100000FF80440BDE700BFB082003018B70030C0
:10211000704F1608874F1608A14F1608B94F1608BA
:1021200008B5FFF757FF054A92F8C81760F3041186
:1021300082F8C817024A907108BD00BFB082003013
:102140000DB90030F7B505460F46B1F07BFE0446E9
:1021500078B102212846B1F039FE064648B114484C
:10216000BCF06CF9C205C0F30723C0F3002403D50B
:102170003446204603B0F0BD9B07F9D50C48BCF0AF
:102180006BF90C4BD3EDB57AF8EEE77A30EE670ACF
:10219000DFED097AB0EEC00AB4EEE70AF1EE10FA0C
:1021A000E6DD064B3A4602212846B1F017FEE0E78D
:1021B000B8A50030B0A200300000C842C44F1608D5
:1021C000F8B504460F46B2F0D5F910210546204671
:1021D000B1F0FCFD58B12046FFF7EEFD064630B9E0
:1021E0003546044B3A4610212046B1F0F7FD28460B
:1021F000F8BD00BFD84F160870B505460E46B1F0C1
:1022000071FD044678B180212846B1F0DFFD50B160
:10221000074B93F8B93D43B10024064B3246802169
:102220002846B1F0DBFD204670BD0446FBE700BF49
:10223000B0820030EC4F160838B50E4C0546D4F885
:102240003003BAF0EBFA012811D0D4F83003BAF019
:10225000E5FA022804D02846BDE83840B1F044BD74
:1022600004F6D87011F048FB0128F4D138BD0020E5
:10227000FCE700BFB0A20030F0B5114C85B00646B7
:102280000F46D4F87C336A460093D4F88033019328
:10229000D4F884330293D4F888330393B2F0B6FEB3
:1022A000054639463046B1F0F3FD94F8C83728406A
:1022B00060F3C303C3F3C00084F8C83705B0F0BDB2
:1022C000B08200302DE9F843DFF8AC90064626488E
:1022D0000F4690F06DFD0446D9F8D407DFF89C80D6
:1022E00003681B699847054630B914F0060F03D1FF
:1022F000D9F80838022B09D139463046B1F09AFE98
:10230000054618B9002488F807400AE039463046E7
:10231000FFF75EFD04460028F4D02DB9012388F8AC
:1023200007302046BDE8F88308213046B1F04EFD65
:102330000028F3D00D4828F0ABFE0028EED00C4B5F
:10234000B02193F8142401FB023203F54053B2F894
:102350001E22B3F9A2369A42E0DD064B3A46082126
:102360003046B1F03BFDCDE724660030D03300307D
:10237000B032003000501608B08200300DB9003085
:1023800070B588B005460E46B1F05AFF044688B3D2
:1023900020212846B1F01AFD60B31B4B93F86C2442
:1023A00042B393F848349B0724D507AA06A91748D7
:1023B0008CF02CFCF0B19DED077ADFED157AB4EED0
:1023C000E77AF1EE10FA15D8B7EEC77A002420218B
:1023D00028468DED027BDDED067AFDEEE77A08A357
:1023E000D3E90023CDED007ACDE90423094B324631
:1023F000B1F0F4FC204608B070BD00BFAFF3008020
:10240000000000403333E33FB0A20030A46A003044
:102410009A99193F105016082DE9F3410F460446CA
:1024200019F0CCFB804618F063FA054640B9564ACD
:1024300001212046B1F0DCFE284602B0BDE8F08163
:10244000524E3946D6F8D40703689B69984705462B
:1024500058B9D6F8D40703681B6C98474C4A034612
:1024600001212046B1F0C4FEE6E7A368002BE3D0CB
:1024700010212046B1F0AAFC20B3D8ED937A98ED54
:10248000920A20EE270AFBF07DF9DFED427AA6F5ED
:10249000005320EE270ADFED407AB3F9743620EEC0
:1024A000270A07EE903AF8EEE77AB4EEE70AF1EE83
:1024B00010FA07DD394B012210212046B1F08EFCC5
:1024C0000025B9E720212046B1F080FC38B196F80C
:1024D000ED37DB0603D5324B01222021EDE7402109
:1024E0002046B1F073FC28B3012F1CD0232F1AD043
:1024F000042F18D0D6F884332A48B3F9083000EEF8
:10250000103AB8EEC00A00F0D1FBB5EEC00AF1EE09
:1025100010FA1DDD244B0122402120460093234B5D
:10252000B1F05CFCCCE7D6F8D4070368DB6B9847C6
:102530000028DFD01E4B1B68D86A0368DB69984708
:102540000128014619D11B4A2046B1F051FEB7E7D8
:10255000D6F8D40703685B69984730B1D6F884335E
:10256000B3F90830002BE5DDD4E7D6F8D4070368CB
:102570001B6898470B28DDD1F0E73946204602B0AA
:10258000BDE8F041B2F0E4BA3C501608B082003029
:102590004D501608E02E65420000C84261501608F2
:1025A000644E1608B0320030674D160869501608A0
:1025B00018B700307550160870B505460E46FFF77F
:1025C00007FC084B04463146D8712846FFF7E4FC67
:1025D00000283146284608BF0024B2F0C5FC204040
:1025E00070BD00BF0DB900302DE9F041524F3B786E
:1025F000002B40F09F80514C0126D4F8F8573E70D4
:1026000095F8CB501DB13B702846BDE8F081B2F083
:102610004FFE054630B94A4A3870137843F001033B
:102620001370F1E76EF0C6FD31466DF0FFFEA4F5C4
:10263000A04007F031FC434B1E710B26013E5EF0BB
:1026400067FF5EF003FF16F0FF06F7D13E4800F08B
:10265000B7FF19F0B3FAD0F80022C4F8202890F898
:102660007C32DA0754D418F0D3FD6EF0A3FD3C2180
:102670006EF0DCFC04F5FC6300221A600021324895
:1026800001F02CF8304815F007FB01462F48C0F048
:1026900083FC2F4B2F4E01211B68D86A03681B68EF
:1026A000984796F8A834D4F8F8076FF3410386F8F2
:1026B000A83403689B6A98470121D4F8F807BCF056
:1026C0006BFE6EF077FD8046D4F8D40703681B6874
:1026D0009847A6F580430146404693F888246EF05B
:1026E0007DF8A6F5E04007F0C9FB6BF023FC6AF02B
:1026F00065FF00233B70C5F0ADFFB4F8CA37C6F8DC
:102700003C0323F4087343F02003A4F8CA377BE7A3
:102710009B07B3D431460C4805F060FC0E48BBF073
:102720009BFEDFED0E7A04F5FC6320EE270A83EDB5
:10273000000AA3E7002567E7AD320030B082003021
:102740002CB900300DB90030B03200302C8200308E
:1027500018B70030B0A20030B8A500300AD7233C2B
:102760002DE9F043374D87B0D5F8F83793F8CB30E3
:10277000002B64D062B1012901D0232908D195F939
:10278000C837002B04DB0024204607B0BDE8F083E7
:10279000B2F03CFE04460028F5D019F00FFA0746C7
:1027A00021F0A2F88046384617F0C8FED8B198F953
:1027B0002830022B17D100264FF00009F1B203AAEE
:1027C0003846CDF80C900191CDF81090CDF81490CA
:1027D00018F012FB019918B103AA404620F010FD31
:1027E0000136032EEAD10121174807F0C1FD01216E
:1027F000154807F0F3FC0021D5F8F807BCF0CCFD34
:1028000012483FF04FF96EF0D5FC00216DF00EFE3E
:102810000F4B00211B68D86A03681B68984795F81E
:10282000CA37D5F8D4176FF345130A4885F8CA3765
:102830000B1A3C3059425941C4F00AF9A4E701246B
:10284000A2E700BFB0820030B03200301CAB0030D5
:1028500018B700300CAE003010B5064CD4F8D407D1
:1028600003685B6A984718B1D4F8F83793F8CB003F
:1028700010BD00BFB082003030B52DED028B89B0A5
:10288000B0EE408A0C46FFF7E7FF0546002836D039
:10289000B4EE488A2268636802A89FED1B0AF1EE35
:1028A00010FA029203937DBFDFED188ADFED167AEE
:1028B00068EE288ADFED168A78BF68EEA78AD4ED25
:1028C000027AF1EE677ACDED047A3BF091FCB4EE3A
:1028D000488A002201238DED050ACDED060A05A9DF
:1028E000F1EE10FA9FED0A0AF0EE680A09488DED44
:1028F000071ACDE9002368BF13460EF031FD2846C4
:1029000009B0BDEC028B30BD0000C842E02E65422C
:102910000000000028B1003007B50191FFF79CFFCF
:1029200030B10199044803B05DF804EB00F010BB2E
:1029300003B05DF804FB00BFB0320030014890F0F6
:10294000C3BB00BF2466003000F5A04008B590F876
:10295000C837C3F340128A420BD061F3451380F8A5
:10296000C83731B16EF026FC0F21BDE808406EF08B
:102970005DBB08BD70B500F5A04605460C46D6F80F
:1029800008388B4212D0012911D0022916D059B92A
:102990006EF010FC1B216EF049FB0D4A05F5AA40B4
:1029A0000621603070F0D4FFC6F8084870BD6EF0A4
:1029B00001FC1A216EF03AFB064AEFE7012100F014
:1029C0008DFE6EF0F7FB1D216EF030FB024AE5E74D
:1029D000E4501608F9501608F450160800F5A04205
:1029E00010B592F8ED370C4603F00101A14209D071
:1029F00064F3000382F8ED37DB0704D406F024FE0D
:102A0000024B9C7210BD07F009F8F9E70DB90030D0
:102A100000F5A04090F8ED3761F3410380F8ED3701
:102A2000014B1973704700BF0DB9003010B5044653
:102A30007AF0C0FC20217BF075FE04F5A04300383D
:102A400093F8CA2718BF012060F3820283F8CA27CF
:102A500010BD000010B504466BF06CFA436F04F52E
:102A6000A04204F5E044D2F8F827D360D4F8242338
:102A70009366D4F82C23C2F80833D4F824030368EF
:102A80005B6D9847D4F824030368BDE810409B6D44
:102A900018470000F8B500F5A04504462DED028B5F
:102AA000D5F8F83793F8CB30002B7DD095F9C8379F
:102AB000002B79DB00F5E04696F89037002B73D1B8
:102AC000D5F8D40703685B69984700286CD1384B68
:102AD000D3F8D40703681B6898470B2864D0D6F84E
:102AE0002C339FED347AD3EDE47AF0EEE77AF4EE0E
:102AF000C77AF1EE10FA57D5D5F8F807443070F0E0
:102B00008FF80346B7EE001A9F20DFED2B0A93EDF6
:102B1000000A35F08BFFB5EEC00AF1EE10FA43DD86
:102B200004F5E6400830BBF0A3FCB0EEC00ADFEDD0
:102B3000237AB4EEE70AF1EE10FA35D504F58057A2
:102B4000D6F82403D7F8903D07EE903A0368B8EE24
:102B5000E78AD3F898309847DFED197A38EE400AC3
:102B6000B0EEC00AB4EEE70AF1EE10FA1CD5D7F8C1
:102B7000943D40F2E63203F2F313934214D8D5F8B1
:102B8000F8079FED100ABDF0DDFFD5F8F83704F522
:102B9000A0509FED0C0AD3ED0C0A1430BDEC028B53
:102BA000BDE8F840A1F0AABCBDEC028BF8BD00BFA7
:102BB000B0820030000000340000000000007042CD
:102BC0000000FA430AD7233C00F5A04008B5D0F82E
:102BD000F80703681B699847F6EE007A20EE270A8B
:102BE000B5EEC00AF1EE10FA48BF9FED010A08BD2C
:102BF0000000000038B500F5E0450446B7EE001AC5
:102C0000712004F5A044DFED110A2DED028BD5F8FB
:102C1000243393ED370A35F009FFD4F8F807B0EE06
:102C2000408AD5F82C53036805F505751B6998474C
:102C300038EE400ADFED067A2846BDEC028B20EE26
:102C4000270ABDE838409EF0F7B900BF0000000039
:102C500000007A4400F5DC50D2ED007A91ED006A74
:102C6000D0ED9A5AD0ED9D6A26EEE77A67EEA57A06
:102C7000A6EE257AE6EE267A81ED007AC2ED007A9C
:102C80007047000000F5A043B3F9483043B900F5A0
:102C90004050B0F9AE060028B8BF404280B270473D
:102CA00083EAE370A0EBE370F8E7000000F5A043CF
:102CB00070B52DED028B93F8ED1782B0044611F03C
:102CC000010605D09FED2E0A02B0BDEC028B70BD4F
:102CD0008DED010A7AF06EFB037F002BF2D0DFED61
:102CE000298A04F54055DFED260A4E20B0EE681A19
:102CF0009DED010A35F09AFE4FF4C8723146B5F9E0
:102D0000B606B0EE408A35F0F9FEA5F8B6062046C4
:102D100014F038FDB5F9B63607EE900AB8EEE77A4A
:102D200007EE903AF8EEE77A77EE676AB4EEE68A55
:102D3000F1EE10FA0DD5204638EE668AFFF7A2FFB5
:102D400007EE900AB8EEE70A20EE088A88EE260A17
:102D5000BAE777EE877AB4EEE78AF1EE10FAB1DDE2
:102D6000B5F9AE3638EE678A78EEE77A00EE103ABB
:102D7000B8EEC00A20EE088A88EE270AA4E700BF52
:102D80000000000000007A440020704700207047D7
:102D90007047000000F55B500430704700487047F2
:102DA0008488160800F5A040D0F8D40703681B6893
:102DB00018470000034808603821117008221A6083
:102DC000704700BF3057160800F5A040D0F8D40770
:102DD0000368DB6C1847000000F5A040D0F8D4076A
:102DE00003689B6C1847000000F5A04300F5F04015
:102DF000D3F8D43730301B1A58425841704700007E
:102E000000F5A04010B5D0F8D4070C460368DB6D80
:102E1000984707EE900A9FED057A0120F8EE677A51
:102E200067EE877AC4ED007A10BD00BF0AD7233C55
:102E300000F5A04010B5D0F8D4070C4603689B6D90
:102E4000984707EE900A9FED057A0120F8EEE77AA1
:102E500067EE877AC4ED007A10BD00BF0AD7233C25
:102E600000F5A04010B5D0F8D4070C4603681B6EDF
:102E70009847DFED047A012020EE270A84ED000A4E
:102E800010BD00BF0AD7233C83F02CBEC0F068BB46
:102E900004F0F8BC88F024BA7CF06EBD6AF094BFF0
:102EA00033F03ABB6DF040BC1CF0DABF7DF040B9A6
:102EB00079F0CEBE77F0A2BC14F0D2B814F06EBD9B
:102EC00007F08EBC15F0C8BD06F014BC06F062B960
:102ED00006F088B814F05CBA85F0DEBB8FF074BDE4
:102EE00011F0BABBFFF7D6BD14F0F6B9AFF05ABF78
:102EF0008BF0AABE14F094BC03F0DEBC14F076B9DB
:102F000014F0F4B87AF0A4B960F064BB29F00ABEFA
:102F100007F02EB802F0C2BF7DF01AB914F0C2BC9F
:102F200007F014BC05F046B807F07EBD06F0ECB81B
:102F300007F0CEB814F020B8FFF78CBD33F0BEBF59
:102F400006F0E8BD0BF01EBC0BF05CBA0BF0F0B95C
:102F50001FB500F5A04304460391D3F8D4070368D6
:102F60005B6A984760B10023DFED060A04F5FC4078
:102F70000399B0EE600A1A46783000930EF0E4FA36
:102F800004B010BD0000000000F5A04310B50446D9
:102F90002DED028BD3F8D407B0EE408A03685B6A4C
:102FA000984720B900242046BDEC028B10BD04F5E3
:102FB000FC409FED070A783028EE000A0DF0EEFC89
:102FC00004460028EED001210248FFF7BDFCEAE7E5
:102FD0000000C842B03200300A4A0B4692F9C827B6
:102FE000002A05DA00228A604A600A6001207047E0
:102FF00000F5E040D0F82423783207CA83E80700C0
:10300000F4E700BFB0820030674B70B5044640F86B
:10301000043B83F087FE002504F1100004F55856A8
:103020001CF060FB04F168006AF05CFC04F5907031
:1030300027F01AFF04F5AA601AF042FF04F2EC60D0
:103040001FF056FE04F6382033F07CF804F6C86012
:1030500083F028FC04F6987064F03EFE04F592506C
:10306000183608306DF042F904F598508FF044F8A6
:1030700004F598501C307CF0F5FE04F59A50183099
:103080001EF0DCFA04F5A0501430A2F0B9F804F5F3
:10309000D5500430AEF0BEFA04F5D6506AF0E2FF27
:1030A00004F5D850143084F0E7FF04F5805304F59C
:1030B000DA503E4A83F8385B04F5D95308301833A8
:1030C00013605DF0B9FF04F5DC502946183016F0A6
:1030D0001DFF04F50950203088F012F904F50A505C
:1030E00010309FF0A1FA04F52C501430A7F0DAF854
:1030F00004F530502C30A5F0D7FE04F531501430D3
:10310000A9F0ECFA04F533502030ADF0DDFB04F506
:1031100035500430AEF012F804F536501C309EF0F5
:10312000C5F904F53950043015F0A8FE04F53E50F9
:103130003030A0F017F804F540500830AFF000FC34
:1031400004F54D501A491C3063F064FB04F54D50F2
:1031500034308FF0D3FC04F550503030AFF0C4FA67
:1031600004F5405383F8885404F552551835284621
:103170000C356FF051FDAE42F9D104F558500D4DAC
:103180002430AFF031FB04F5595008306FF040F8AF
:103190002B6813B10848C5F02BFA2046074963F0A5
:1031A00039FB20462C6070BD6087170850C4003082
:1031B00068581808F0B9003008511608E885170853
:1031C00010B514F057FA7AF0F5F80368BDE810402E
:1031D0005B681847FFF7F4BF10B5044607F016F810
:1031E000204614F083FD204604F02CFD2046BDE867
:1031F000104004F095BE0000FFF7EEBF70B500F57B
:10320000B0450446243528461CF046F920F06CFBF6
:1032100090F9253093B390F844337BB304F5A04381
:1032200004F2EC66D3F8F80744306FF0F9FC03467B
:10323000B7EE001A9F20DFED120A93ED000A35F079
:10324000F5FB94F9243728460021012B04F6481495
:1032500008BF86ED0F0A1BF0EFFEDFED0A7A94ED52
:10326000287A304620EE270ADFED077AA7EE270AF4
:1032700084ED280ABDE8704020F02EBA70BD00BF72
:1032800000000000CDCCCC3D6666663FFFF7B6BFC0
:1032900010B50121044614F065FD60B1114BD3F85F
:1032A000D40703689B6A984728B9204602F0FCFCC3
:1032B000204602F009FD4FF40011204614F052FDA3
:1032C00018B134F0CDFD32F00FFE4FF480212046CE
:1032D00014F048FD28B134F0C3FDBDE8104032F0D1
:1032E00011BD10BDB0820030FFF7D2BF7FB500F531
:1032F000E04604469FED660AD6F824036C303AF0A7
:1033000077FF04F5DC5001A98DED010A1830CDEDF1
:10331000020A8DED031A16F08DFC0221204614F0EE
:1033200021FD70B10121204614F01CFD48B9594B14
:10333000D3F8D40703689B6A984710B9204602F077
:10334000B3FC0121204614F00DFD48B9514BD3F8D0
:10335000D40703689B6A984710B9204602F0B4FC72
:103360000121204614F0FEFC10B9204602F006FDB3
:103370004FF40031204614F0F5FC30B104F5A043C1
:10338000D3F8F80703685B6C98474021204614F097
:10339000E9FC68B104F59255083528466CF058FAF6
:1033A00004F5805393F91C3313B128466CF014FCD8
:1033B0004FF48061204614F0D5FC20B104F5925002
:1033C00008306CF0DFFA2021204614F0CBFC58B115
:1033D00004F5A045D5F8D40703681B699847C8B31E
:1033E000D6F82C03B6F058FA8021204614F0BAFC27
:1033F00000283CD034F034FD32F0A8FC10212046E7
:1034000014F0B0FC68B1D6F82403B2F0B7FE04F5AE
:103410005F5034308BF03EFD04F55C503830AFF037
:1034200033FD4FF6FF71204614F09CFC20B104F5EB
:10343000A0402C30C0F0A2F84FF40041204614F018
:1034400091FC18B304F5E740443004B0BDE8704087
:103450007CF0B0BF20460EF099FF0028C0D1D5F80F
:10346000D40703685B6998470028B9D0BCE74FF4DC
:103470008021204614F076FC0028BBD14FF40021B7
:10348000204614F06FFC0028B4D1B7E704B070BD3B
:10349000E02E6542B0820030FFF728BF10B5012151
:1034A000044614F05FFC10B1204602F067FC802156
:1034B000204614F057FC48B14FF48021204614F008
:1034C00051FC18B934F0CCFC32F01CFC4FF4001164
:1034D000204614F047FC30B104F5A050BDE8104080
:1034E0001430A1F0A3B810BDFFF7D8BF10B5044643
:1034F00006F0DEFB204606F031FA204606F01CFC02
:10350000204615F015FB2046BDE8104004F096B9A2
:10351000FFF7ECBF70B504464FF6FF7114F022FCC4
:1035200004F5A04528B1D5F8C8270721204602F0A8
:1035300057FCD5F8F83793F8CB309BB92046FFF706
:1035400075FAD5F8F80704F5804304F54052016890
:1035500092F8CA260E6A93F89C11B047D5F8F8077E
:10356000BDF0BCFA7BF010FF7BF0D0FB204615F0DD
:10357000DDFA95F8C83704F5E0440F4ADB43D4F888
:103580002453C3F3C013537184F8AD362B681E6FF8
:103590006AF0D0FC6AF038F92846B047D4F82C43DA
:1035A0006AF0C8FC04F505746AF02EF92046BDE8FF
:1035B00070409DF013BB00BF0DB90030FFF7AABFEC
:1035C0002DE9F04100F5805600F5A044054606F6C9
:1035D000983304F60C0804F50167D3F85022C8F8B4
:1035E0000020D3F85C323B60D6F8980D00F58C4093
:1035F000503035F0E9F904F61803C4F8140804F65D
:103600001C04D8F800204FF6FF7128461A603B686A
:10361000236014F0A7FB38B1D6F8982D284609216D
:10362000BDE8F04102F0B2BBBDE8F08100F5A04377
:1036300010B5D3F8081800294FD093F8C927D4073C
:103640004BD56FF30002012900F5DC5083F8C92740
:10365000D3E9DF24B2F9081007EE101AB4F9081004
:1036600006EE901A0CBF03F60C0103F61801B8EE33
:10367000C77A07BFD1ED007A03F50161D1ED007A79
:1036800003F61C010CBFF8EEE66AF8EEE66AD1ED2F
:10369000005A25EEE66AA7EE276A67EEA67AD0ED15
:1036A0009A6AE7EE257A90ED9D7A27EE877AA6EE64
:1036B000267ABDEEC77A17EE101A118190ED9A7A2C
:1036C000D3F8803367EE877A90ED9D7AE6EE477AFD
:1036D000FDEEE77A17EE902A1A8110BD38B505463F
:1036E00000F5A0442DED028B71B1284613F018FEB1
:1036F000D4F8143840F2E6321B1A03F2F313934263
:103700000CD8BDEC028B38BDD4F80838022BF8D1A8
:1037100013F0E6FDB0F57A7FE7D2F2E7C4F81408BB
:1037200000F58C406423503090FBF3F300EE103A28
:103730009FED0C7BB8EEC00B20EE070BB7EEC08BF5
:10374000B0EE480AF9F018F804F6180304F61C0461
:1037500083ED000AB0EE480AF9F080FE84ED000A1D
:10376000CFE700BF000000A046DF913F00F5DC502E
:103770000121183018F088B9FFF7F8BF10B50446DA
:1037800014F006F81021204614F0ECFA98B1204607
:1037900002F0E0F94FF40011204614F0E3FA50B9BA
:1037A00034F05EFB32F0A0FB04F5A050BDE8104001
:1037B0001430A0F03BBF10BDFFF7E0BFF8B50446E2
:1037C00007F04AF8224B4FF6FF76254604F18000B9
:1037D0004FF0FF3745F83C3B1E4BA465C4E9173456
:1037E0001D4BC4E919341D4BE3661EF0DBFD04F1EB
:1037F0009C001EF0D7FD04F1B8001EF0D3FD184B5D
:1038000004F1D400A4F8D060C4F8CC301EF0CAFD96
:10381000144B15492846C4F884721D6062F0FAFF03
:1038200004F52670A4F87870A4F894601EF0BAFD30
:1038300004F52D701EF0B6FD04F534701EF0B2FDD7
:103840000023204684F8E432C4F80833F8BD00BFF2
:103850003CB81608452F0608492F06084D2F0608C4
:103860000000FFFFDCB800301442170810B5044612
:1038700006F0F2FF0A4B04F1400023600123A38706
:103880001EF090FD04F150001EF08CFD04F160006C
:103890001EF088FD04F170001EF084FD204610BD6E
:1038A000A4C316082DE9F043044689B0FFF7ACFB2A
:1038B000B54B04F55B5004F5A045236004F5A7471C
:1038C00030304FF07C5802F059FC04F55A5305A9EA
:1038D00007F120003833CDF8148004F5E64604F5EE
:1038E000AC49C5F890330623083609F1300985F84C
:1038F00094336FF0A7FA07F13800C4F03FF80023C3
:1039000004F5A74004A985F8D0331923C5F8D86376
:10391000683085F8DC3304F5A947CDF810806FF0E6
:1039200091FA04F5A8404FF00108C4F027F81823D5
:1039300004F5A840203785F8243485F818843830F9
:10394000C5F8206406AE7BF021FE3846B0F0D6F90B
:103950008E4B3146381DC5F8A0348DF8188063F0C1
:103960006DFD04F5A9408A4F04F5AA4858305FF070
:10397000E1FD04F5AA4008F160081830AEF0F6FF4A
:10398000844B04F5AA403146C5F818353030069707
:103990006FF058FA04F5AA40314606973C306FF0B4
:1039A00051FA04F5AA4031460697483004F5AB4772
:1039B0006FF048FA784B103708F10C00C5F8603505
:1039C000C3F0DCFF3846143774F070FCB945F9D108
:1039D0001E2340F2CC60C5F860370023A5F8643799
:1039E0001FF07EF9C5F85C0704F5AE406830C3F0FF
:1039F000C5FF04F5AF402C30C3F0C0FF674B1A6819
:103A00000AB9C3F8008004F50048654B04F5AF40DF
:103A10004FF07E5708F16408C5F86035583004F55A
:103A2000E949C5F8D487B1F015FD05F60C0304F596
:103A3000B04005F618051F604FF40071594B243053
:103A40002F6004F5E045079309F15409564B06949D
:103A5000009396E80C001BF0C7F804F5BB40002665
:103A60003C3095F0A3FE04F5E54003A903975830D8
:103A70006FF012FA04F5E54003A903976C306FF07C
:103A8000E1F904F5E54078301EF08CFC04F5DC53D8
:103A900004F5E6404FF400411833C5F8086344309C
:103AA000C5F80C63C5F820330023C5F8106385F80A
:103AB0004133C5F81463C5F81863C5F81C631BF0DF
:103AC000FBFE04F5E74044307CF01CFB04F5E840C5
:103AD000483091F04BFC04F5E940043063F0E4FD1C
:103AE000324B04F5E940C5F8843418308EF00EFFEF
:103AF00004F5E9402E4B34302E49186062F08AFEFE
:103B0000FF232D49484685F8E43485F8EC3462F00B
:103B100081FE2A4B1F6817B12948C4F069FD04F5DE
:103B2000E940C3F8009004F5EB497430B7F018FB96
:103B300004F5EB4009F170096830B7F0CFF9484659
:103B40009CF0FAF904F5EE4049462030BDF0B4FF90
:103B50001C4B1D4904F5EF40C5F8203706234FF0F4
:103B6000140C85F87437194B19603B469FB201332A
:103B70000CFB0712127C002AF8D1154B1F80154B45
:103B80001F685FB31448C8E7A05B16088C5016087E
:103B90000000A040D0501608B8A8170864BE003036
:103BA000205C1608412F0608905B1608E0501608A6
:103BB00058C4003080C817089C56180818C5003033
:103BC0001C51160850AF160834A51608B0B90030BD
:103BD000ACB900306CB900303D511608186004F5DE
:103BE000EF406E4B03A9143004F5F64903936FF0D0
:103BF00029F904F5EF4009F15C09343006F02CFE98
:103C0000674B04F5EF40C5F8B437743006F024FE76
:103C1000644B04F5F040C5F8F4373030FFF7CEFDC3
:103C2000484606F019FE604B09F13C00C5F85C3BC4
:103C3000C1F0B4FB5D4B04F5FA40C5F8983B1C306D
:103C400006F00AFE5A4B04F5FA40C5F81C3D6030F8
:103C500006F002FE574B04F5FB4085F89C7DC5F845
:103C6000603D203006F0F8FD534B04F5FB40C5F8ED
:103C7000A03D5C3006F0F0FD504B04F5FC40C5F86B
:103C8000DC3D05F6186330301E605E609E6006F015
:103C9000E3FD4B4B04F5FC40C5F86C7EC5F8303EA7
:103CA000783006F0D9FD474B04F5FD40C5F8B47EE9
:103CB000C5F8783E3C3006F0CFFD434B04F5FE409E
:103CC000C5F8BC3E05F6BC75043006F0C5FD3F4B9B
:103CD00004F5FE4045F8B83C443006F0BDFD3C4BD1
:103CE00004F5FF4045F8783C58302E606E6004F5CE
:103CF0000045FFF7BBFD404606F0AEFD354B2846BC
:103D00006B66A03010F078FD04F501405C3006F0E1
:103D1000A3FD314B04F50140C5F89871C5F85C313D
:103D2000A03006F099FD2D4B04F50140A5F8DC719B
:103D3000C5F8A031F03006F08FFD294B04F50240A4
:103D4000C5F82C72C5F8F0313430FFF78FFD254BE4
:103D500004F50240C5F8C462C5F834320123C5F841
:103D6000C862D03085F8BD32C5F8CC6205F25C453A
:103D70000BF0D0FE04F50340A43012F0ABF804F5CC
:103D800004401C3006F068FD174B204645F8403CC7
:103D90002E606E6009B0BDE8F08300BFCDCC4C3D15
:103DA0002CB41608D4B41608E4B8160878B9160866
:103DB000DCBA160880BB160824BC1608C0BC16085E
:103DC00004BF1608A8BF1608E8C0160884C1160864
:103DD00028C2160808C5160838BA16082CC91608CD
:103DE00054C0160860C41608F4C9160838B5054B47
:103DF0000A4601461C68236820461D68024BA847F6
:103E0000002038BD18B70030B032003038B5037923
:103E100004463BB905682DB1284631F00FF9284614
:103E20001EF060FF204638BD294B70B50360044684
:103E300000F54B503C301EF03DFA04F5005393F86A
:103E4000382D42B9D3F8345D2DB1284631F0F6F85B
:103E500028461EF047FF04F5D55004F64C7504F6CD
:103E6000EC660430ADF0EAFB04F5B1500830FFF722
:103E7000CDFF04F5B150FFF7C9FF04F5B05018307D
:103E8000FFF7C4FF04F598501C307CF003F8B542EE
:103E900004D0183D284630F02BFDF8E70D4B04F513
:103EA0004A60C4F8383AFFF7B1FF04F69840FFF7CC
:103EB000ADFF04F54960FFF7A9FF04F634306EF05A
:103EC00073FB04F52A606EF06FFB204670BD00BFE7
:103ED000608717084031170838B5104B0446036057
:103EE00000F5E04393F8142742B9D3F810572DB1E9
:103EF000284631F0A3F828461EF0F4FE04F5A0434E
:103F0000074AD3F85C07C3F8602508B11EF0EEFE3F
:103F10002046FFF789FF204638BD00BFA05B16088A
:103F2000B8A8170810B5C3F0F7FF064C064B186089
:103F30002046FFF7B7FC2046044A0549BDE810407B
:103F4000F8F014BCB032003018B7003090210130C6
:103F5000D93E06080120704790F8D0308B4286BFCA
:103F600000EB8100D0F8D4000020704790F8D030EA
:103F70008B4286BF00EB8100D0F8D4000020704750
:103F8000FA207047014B93F87A067047B062003010
:103F9000034BD3F80808431E58425841704700BFEE
:103FA000B0820030034BD3F80808831E58425841B2
:103FB000704700BFB0820030034BD3F8F80708B158
:103FC000BBF0E4BA01487047B08200300C5C1608C0
:103FD000F8B5436A0446444D43F4E0524262826AB3
:103FE00042F4E0528262C26A42F4E052C262D5F800
:103FF0002C23E2B143F4F8434362D5F82C03B4F028
:10400000C3FF38B1A36A43F48043A362E36A43F475
:104010008043E362D5F82C03B5F0E0F838B1A36A29
:1040200043F40053A362E36A43F40053E3622F486E
:104030008AF046FE18B1636A43F0806363622B48DE
:104040008AF0EAFD18B1A36A43F08063A3622748AF
:104050008AF068FE18B9E36A43F08063E362244B98
:104060001E6846B11921304663F010FF18B1636A2B
:1040700043F4807363621F4F97F898336BB1A36A60
:1040800043F48073A36246B11921304663F036FFD2
:1040900018B1E36A43F48073E36295F9F4348BB1A9
:1040A000D4E9092343F0800342F08002A3626262F4
:1040B00095F9F43433B195F8DC351BB1E36A43F07C
:1040C0008003E362636A43F080436362A36A43F060
:1040D0008043A362D7F8F83793F8C1301BB9E36A7D
:1040E00043F08043E362F8BDB0A20030A46A003020
:1040F000BCB90030B082003013B54FF44470CDE944
:1041000000211EF0E7FD044628B1DDE9002177F02B
:104110002DFE024B2360204602B010BD685E1608DB
:104120000020704770470000032070470820704748
:10413000014B93F87C067047B0620030034B93F953
:104140009001003818BF0120704700BFB0720030E6
:10415000014B93F97E067047B06200307047000053
:1041600008B50C4BD3F82C0370B910230A4A43F05E
:104170004000D2F8F82722B192F8CB200AB143F0E0
:10418000C00040F0010008BDB4F0FEFE0028ECD0F5
:104190001823EBE7B0A20030B082003038B5C57804
:1041A0000B4604463522352D4FF00001184628BF36
:1041B0003525FCF0DDF904F10C012A46BDE8384054
:1041C000FCF08CB900B5002389B0029303930493EB
:1041D00005930693079317F0F1FC02A917F0BEFAB6
:1041E000A0B117F0EBFC00F55A7005AB07C883E8E7
:1041F000070018463AF01AFCF1EE047A20EE270A7E
:10420000FCEEC07ACDED017A9DF8040009B05DF8AE
:1042100004FB00001FB5184C94F89A1F04F6446084
:1042200015F04EF878B194F89A1F04F6446015F032
:10423000C7FA40B194F89A1F04F6446004B0BDE890
:10424000104015F001BB002301930293039317F074
:10425000B5FC01A917F082FA20B101A83AF0E6FBFB
:1042600004B010BD28F09CFCB02290F8F43202FBA0
:10427000030090ED3B0AF3E7B052003008B50D4B58
:10428000D3F8F807A8B144306EF0CAFC0346B7EE85
:10429000001A9F2093ED000ADFED070A34F0C6FBF9
:1042A000DFED067A20EE270ABDEEC00A10EE103AC6
:1042B00018B208BDB0820030000000000000C84203
:1042C0002DE9F04FDFF8D8808DB00446334F042538
:1042D00008F5804617F8019BB8F9D43609F1FF3A82
:1042E00043FA0AF3D90742D5207C70F049FB834694
:1042F000207C71F063FA00F121039B4505D2207CFC
:104300000DB0BDE8F04F6FF073BDBAF1030F2ED8BA
:10431000DFE80AF00234393ED6F8240303689B68CC
:10432000984700F1A0035A69D3F800A0D3F804E03D
:10433000D8681969D3F818C008925A6A1B6ACDF870
:1043400025206222CDF82930212306900791C22131
:10435000207CCDF80CA0CDF810E0CDF814C08DF87D
:104360002490CDE90032192303AA70F087FB013DA8
:1043700015F0FF05AED10DB0BDE8F08FD6F82403DF
:104380000368DB68CCE7D6F8240303681B69C7E73A
:10439000D6F82C3303F52D73C5E700BF585F160818
:1043A000B062003007B50190BFF0F6F828B101996E
:1043B00003B05DF804EBBFF0B1B803B05DF804FBE7
:1043C00013B504460748019109F042FF30B901993D
:1043D000204602B0BDE8104071F050BC042002B08D
:1043E00010BD00BFE0AA0030014809F0E5BC00BFE5
:1043F000E0AA00300B4B70B5D3F8943105460E4659
:104400001446DB0703D511460748BDF013FF2146CC
:104410000648BFF079FF224631462846BDE8704085
:1044200076F08CB8B0720030D0A900300083003034
:1044300010B588B0044672F0A1FF0C4BD3F8F80712
:1044400038B90B4A0621204608B0BDE8104072F08A
:104450007DBF69461E22BBF09DF86B46054A0621CA
:10446000204672F073FF08B010BD00BFB08200306C
:10447000585C1608BEB11608034A92F87833013327
:1044800082F8783371F0D0BEB08200300148B7F0C6
:1044900093B800BFA4A7003007B5084601911EF0ED
:1044A00069F838B10448019902F0F2FF002003B026
:1044B0005DF804FB0420FAE724B70030F7B58B8BD6
:1044C00006460C461746CD2B1DD1D1ED067AFCEEE3
:1044D000E77ACDED017A9DF80430022B13D10E4D11
:1044E00095F83D1405F571707BF042FE58B195F8D2
:1044F0003D1405F571707BF043FE20B994ED020A7E
:10450000064802F0A5FF3A462146304603B0BDE812
:10451000F04071F01BBF00BFB0A2003024B70030E4
:10452000162A10B40C4605D0542A03D05DF8044B6B
:1045300071F0C0BB0323012023705DF8044B70476A
:1045400008B571F027FE40F41C6040F00D0008BD76
:104550001FB517F033FB044668461DF023FF69467C
:10456000204617F0A1F80E4B93F8C90710F0200071
:1045700014D003F50053DDED017AD3F82C33F8EEB7
:10458000E77A93ED0F7A77EE877A9FED067A67EEFA
:10459000877AFDEEE77A17EE903A18B204B010BDB4
:1045A000B08200300AD7233C10B504461EF09AFBB7
:1045B000204610BD10B50C4C94F9C837002B0FDB0A
:1045C000D4F8D4070368DB6C984758B9D4F8D407FB
:1045D00003689B6C984700280CBF0220032010BD85
:1045E0000120FCE70420FAE7B082003008B5134B45
:1045F00093F8C90710F020001ED0D3F8D407036841
:10460000DB6D984707EE900AF2EE046AB8EE677A1F
:10461000DFED0B7A27EE277ADFED0A7AB4EEE77A40
:10462000F1EE10FA58BFB0EE677AC7EE267AFCEECC
:10463000E77A17EE903A98B208BD00BFB08200301A
:104640000AD7233C00FF7F4710B44C69012C05D1E9
:1046500001465DF8044B034803F008BD5DF8044BC8
:1046600071F0FCBDB03200302DE9F341B1F90430F6
:1046700006460C461546002B35DB1C4F4FF0000854
:104680009FED1B0A4FF47A73CDE90028B1F902209F
:10469000D7F87C1376F09CFA01239FED150A30467B
:1046A000B4F90020D7F88013CDE900534FF47A73A2
:1046B00076F08EFA9FED0F0A4346B4F90420D7F83E
:1046C00084133046CDE9005876F082FA9FED080A4F
:1046D0004FF47A73B4F90620D7F888133046CDE941
:1046E000005876F075FA02B0BDE8F081B082003073
:1046F0000000FA4400007A4408B5094B93F8C90752
:1047000010F020000AD0D3F8D40703689B6D9847B7
:1047100034F05AF9C82390FBF3F0C0B208BD00BFD3
:10472000B0820030044B187820B9044B93F8CA07C4
:10473000C0F38010704700BFACB80030B0820030CA
:104740007FB5002303930493059317F037FA03A969
:1047500017F004F8D8B117F031FAD0EDDA0A90ED7D
:10476000DB0AF1EE600AB1EE400AF9F073F8DFED12
:10477000097A20EE270A34F09DF8F6EE007A20EE52
:10478000270AFCEEC07ACDED017A9DF8040007B04F
:104790005DF804FBE02E6542124B07B593F8C9079C
:1047A00010F020001AD003F50053D3F82C0300F5C5
:1047B00065703AF03BF9DFED0C7A20EE270ADFED69
:1047C0000B7AB4EEE70AF1EE10FA58BFB0EE670AC2
:1047D000FCEEC07ACDED017A9DF8040003B05DF8DF
:1047E00004FB00BFB0820030CDCC4C3D00007F43C5
:1047F0000B4B93F8B92D7AB993F8ED2792060BD1AC
:1048000093F9C827002A09DB93F8C93713F0200F62
:1048100014BF042001207047052070470320704713
:10482000B082003008B5074B93F9C836032B03D08C
:10483000BDE8084072F002BE034A022172F086FD14
:10484000042008BDB0620030705C1608084BD3F835
:104850009421920701D471F021BA03F54053DFEDA2
:10486000057A93EDBF0AB8EEC00A20EE270A70471A
:10487000B07200300AD7233C10B594B0044603A8A8
:104880001DF090FD1C4B03A9D3F8D40703685B6DA2
:10489000984778B3002103A81DF01CFE50B3247C78
:1048A000C3F0D8FE059B9622DDED047A57210893CC
:1048B000069BF8EEE77A9FED117A0993002367EEE5
:1048C000877A07900B9320460C930D930E930F93CA
:1048D0001093119312934FF6F853CDED0A7AADF879
:1048E0004C3000238DF84E303323CDE9003207AA37
:1048F00070F0C4F814B010BDB08200300AD7233C69
:1049000030B5844C05462DED0A8BD4F8D40799B008
:1049100003685B6A9847002867D004F50054D4F810
:10492000B43E062B00F2E180DFE803F004040463E8
:10493000A0C35F00784840F6F8540DF011F89FEDE1
:10494000778A9FED770AF0EE489AB0EE48AAF0EE2B
:10495000488AF0EE48AAB0EE48BA90ED027B90ED9E
:10496000005BF7EEC76BB7EEC55B90ED047B0BA861
:104970008DED0B5ACDED0C6AB7EEC77B8DED0D7A40
:1049800039F036FCB0EE40CAF0EE60BAB0EE419AB3
:104990002D7CC3F05FFE00238C22B1EE499A0B9070
:1049A0001593F1EE688A16930123B1EE488A5521DA
:1049B0008DF85E30332328468DED0CCACDED0DBA4F
:1049C0008DED0E9A8DED0FBACDED10AACDED118AB9
:1049D0008DED12AACDED139A8DED148AADF85C40E1
:1049E000CDE900320BAA70F049F819B0BDEC0A8B82
:1049F00030BD49484FF440640CF0B2FF9FED480AC7
:104A000090ED027B90ED005BF7EEC76BB7EEC55BF8
:104A100090ED047B0BA88DED0B5ACDED0C6AB7EE33
:104A2000C77B8DED0D7A39F0E3FB3B48F0EE60BAC1
:104A3000B0EE419AB0EE40CA0CF096FF9FED380AF6
:104A400039F0D6FB3448B0EE40BAF0EE60AAF0EE92
:104A5000418A0CF08DFF9FED320A39F0C9FBF0EE70
:104A6000609AB0EE40AAB0EE418A91E72A4840F63B
:104A700007440CF079FF9FED2A0A39F0B9FB26486C
:104A8000B0EE40BA9FED259AF0EE60AAF0EE418AB2
:104A90000CF06EFF9FED220AF0EE49BA39F0A8FB48
:104AA000B0EE49CAB0EE40AAF0EE609AB0EE418A8C
:104AB0006EE7194840F63F44DFED188A0CF058FFC6
:104AC0009FED170A39F094FBF0EE68AAB0EE40AA09
:104AD000F0EE609AB0EE418AB0EE68BAB0EE689A35
:104AE000F0EE68BAB0EE68CA52E79FED0C8A002477
:104AF000F0EE489AB0EE48AAF0EE488AF0EE48AAE6
:104B0000B0EE48BAB0EE489AF0EE48BAB0EE48CAF5
:104B10003EE700BFB082003028B100300000000046
:104B20000AD7233C2DE9F0413C4D04462DED068B80
:104B300095F8C9378CB099066AD505F50057DFEDB1
:104B4000388A9FED380AD7F824036C3039F050FBCF
:104B50008DED041A21EE281AD5F8D4678DED020ADE
:104B600060EE289ACDED030A3046BDEEC11A94F8E6
:104B7000108020EEA89A11EE103A1DB233689B6D9A
:104B8000984707EE900A3046F8EEE77A67EEA87A83
:104B9000FDEEE77A17EE903A1CB23368DB6D98476A
:104BA00007EE900AD7F82C333046B8EE678ADFED6F
:104BB0001E7A93ED0FAA336828EE288A1B6E2AEE20
:104BC00028AAB4EEE78AF1EE10FA58BFB0EE678A71
:104BD00098470023B72220EE280A3E21BCEEC88A5F
:104BE00008934046CDED059A8DED069A18EE103AE1
:104BF0008DED07AA8DED090AADF82C301A23ADF81A
:104C00002850ADF82A40CDE9003205AA6FF036FFF2
:104C10000CB0BDEC068BBDE8F08100BFB082003067
:104C20000AD7233C9F0CB34500FF7F471C4B2DE95F
:104C3000F04F2DED028BD3F824338DB0047CD3F8E4
:104C40008480D3F88870D3F88C60D3F8905093EDBB
:104C5000258AD3F898B0D3F89CA0D3F8DC90C3F0A1
:104C6000F9FC00231622029053218DF82C302523C5
:104C700020468DED078ACDF820B0CDF824A0CDF8E0
:104C80002890CDF80C80049705960695CDE9003262
:104C900002AA6FF0F3FE0DB0BDEC028BBDE8F08F01
:104CA000B0A2003070B58A7A06464B7A0C4643EAC9
:104CB0000223CA7A43EA02439D2B21D1134D95F872
:104CC0003D1405F571707BF053FAC8B195F83D14A9
:104CD00005F571707BF060FA022811D195F83D144A
:104CE00005F571707BF04CFA50B9D4ED057A9FED63
:104CF000080AF8EEE77A074827EE800A02F0A8FBD8
:104D000021463046BDE8704071F08EB9B0A2003047
:104D10000AD7233C24B70030054BD3F8F8372BB122
:104D200093F8CA00002808BF02207047022070478D
:104D3000B082003008B5034BD3F8D40703681B6872
:104D4000984708BDB0820030024B93F8C907C0F302
:104D500040107047B082003070B52C4E05460C46AE
:104D6000D6F8D4072DED028B036886B091ED018A49
:104D70005B6A984750B9BDEEC88A18EE103ADB0757
:104D800004D4022006B0BDEC028B70BDD4E904014E
:104D900035F064F90028F4D002A81DF003FB02AA44
:104DA0002146284675F022FE0028EAD0184902A8BC
:104DB0001DF0ECFB03460028E3D1DFED160A0246A6
:104DC000009002A9B0EE600A13480CF0BDFBD8B108
:104DD000D6F8D40703685B6A9847044608B10020F8
:104DE000D0E7022204210D4806F078F960B1DFED2A
:104DF000090A2346224602A9B0EE600A064800943A
:104E00000CF0A2FB0028EAD10420BBE7B0820030FE
:104E1000A8A500300000000028B10030B0320030FA
:104E200008B591F82030032B1CD1D1ED027A9FED0B
:104E30000E7AF0EEE77A91ED060A0C4BF4EEC77AA3
:104E4000DFED0B7AD3F8D40720EE270AF1EE10FA43
:104E50004CBF0121002113F0B5FA002814BF002037
:104E6000042008BD0220FCE700000034B0820030BE
:104E70000000C84210B52DED028BD1ED007A82B052
:104E80000C46F5EEC07AF1EE10FA04DA042002B016
:104E9000BDEC028B10BD9FED197AF4EEC77AF1EEEE
:104EA00010FAF3D891ED030A9FED158AF0EEC07A5F
:104EB000F4EEC87AF1EE10FA19D5D4ED037A114860
:104EC000F4EEC87AD4ED027AD4ED010AFDEEE77A69
:104ED00094ED000AF1EE10FACDED017AACBF01229B
:104EE00000229DF9041002F015FA0020CFE7F7EE3A
:104EF000000A33F039FC0028C8D0DEE70000B443D4
:104F00000000003424B7003091ED010AB5EEC00A6C
:104F100008B5F1EE10FA01DC042008BD9FED107A0F
:104F2000D1ED007A20EE070A9FED0E7A0E4BF4EEDB
:104F3000C77AD3F8D407F1EE10FA036805DDDB6E0B
:104F400098470028E8D00020E7E79FED087AF4EEC4
:104F5000C77AF1EE10FACCBF9B6E5B6EF0E700BF34
:104F60000000C8429A993940B08200303333F33F91
:104F700008B5D1ED007A9FED157AF0EEE77AF4EE00
:104F8000C77AF1EE10FA1DD5D1ED017AF0EEE77A8D
:104F9000F4EEC77AF1EE10FA14D5022203210C4880
:104FA00006F09CF880B10A480121FDF7CDFC0948C4
:104FB00090F87038012B03D000F66C003CF0D8FF5D
:104FC000002000E0022008BD0420FCE700000034BF
:104FD000B0320030B0A2003010B5D1ED007AFCEE56
:104FE000E77A17EE903A9CB2012C02D0022C06D040
:104FF0004CB92146054883F0CDFF002010BD044880
:1050000003F0E6FDF9E70420F8E700BF64A70030ED
:10501000B03200301FB5D1ED017A0B7CFCEEE77A9F
:10502000CDED027AD1ED007A0093FCEEE77AD1ED76
:10503000030A91ED020A01469DF80830CDED037A8E
:105040009DF80C20024811F0FDFE05B05DF804FB50
:10505000B032003013B513480C46BEF0B7F9F0B1CA
:10506000D4ED017AFCEEE77ACDED017A9DF80400EB
:10507000012807D002280CD088B90B4B83F83A00DE
:1050800002B010BD94ED020A0648BEF0B1F900204E
:10509000F6E794ED030A0348BEF0EAF9F7E70420C7
:1050A000EEE700BFDC820030B082003010B50A4C61
:1050B00094F8ED37DB070CD402220521A4F5A040BB
:1050C00006F00CF828B90222A4F5A040114606F01B
:1050D00005F8002010BD00BFB082003010B5D1ED42
:1050E000007A0446FCEEE77A17EE903A13F0FF03DD
:1050F0000FD10F4BD3F8D40703689B6F984708B1C3
:10510000002010BD0B4A2046062172F01FF9042032
:10511000F7E7012B09D1064BD3F8D4070368DB6FFF
:1051200098470028ECD1044AEDE70220E9E700BFE8
:10513000B0820030945C1608A45C160801F10C03E0
:105140009FED0A7AF1EC017AF4EE677AF1EE10FA4B
:105150000AD6F0EEE77AF4EEC77AF1EE10FA03DC45
:105160009942EFD1012070470020704700007A4437
:1051700030B5002305462DED028B8DB003930493CB
:10518000059316F01BFD03A916F0E8FA58B316F0C4
:1051900015FD00F55A7306AC2D7C93E8070084E8F2
:1051A0000700DDED060A9DED070AF1EE600AB1EE9B
:1051B000400AF8F04FFB2046B0EE408A39F036FC4A
:1051C000089B0122DFED0A7AA8210B930C2328EE1D
:1051D000278A28468DED0A0ACDE9003209AA8DED0D
:1051E000098A6FF04BFC0DB0BDEC028B30BD00BFE7
:1051F000E02E65424029F7B505460E461ED00AD876
:105200001B290CD024290CD03146284603B0BDE818
:10521000F04075F081BFA1F14203012BF4D80124C5
:1052200005E00C216EF0F6FD044618B90024204676
:1052300003B0F0BD2846FFF79BFFF8E726216EF08C
:10524000E9FD04460028F1D0297C10489AF0CAFFF5
:105250000F4B1F68002FEAD0262128466EF0DAFD9A
:1052600004460028E3D000230DF10602314628460B
:10527000ADF8063076F0A4FE0028D8D0BDF80620A0
:105280003846297C93F0F4FAD1E700BFA0A800309B
:1052900014C5003038B5184C0D4694F8ED37DB07CF
:1052A0000AD4D4F8F83793F8CB303BB9012204F58F
:1052B00094601146FDF798F9002038BD94F9C8377D
:1052C0000222002B12DA0521A4F5A04005F006FF0A
:1052D0000028F1D095ED000A0121DFED087AD4F81D
:1052E000D40720EE270A13F06DF8E5E70921A4F5AD
:1052F000A04005F0F3FEDFE7B08200300000C842B6
:1053000010B5214C94F8ED37DB070ED4D4F8F837FC
:1053100093F8CB304BB194F9C837002B07DA012250
:10532000082104F59460FDF71BFA002010BDD1EDB3
:10533000007A9FED167AF0EEE77AF4EEC77AF1EE96
:1053400010FA0BD502221121114805F0C7FEA0B9B1
:1053500002220F48114605F0C1FEE6E7D4F8D40753
:1053600003681B6898470428DFD0D4F8D407036883
:105370001B6898471428E5D1D7E740F6C4110548C3
:1053800009F07AFDD1E700BFB082003000000034A0
:10539000B0320030CCAF003073B58B8B05460C4675
:1053A000C12B44D8BB2B0DD8202B67D02ED8113B56
:1053B00099B2052918D92146284602B0BDE87040A7
:1053C00077F0DEB8BC3B052BF5D801A151F823F0EE
:1053D000215506082B550608B7530608B75306088B
:1053E000AF540608BB540608052BE4D801A151F8B8
:1053F00023F000BF07550608B7530608B753060841
:105400001B5506081B540608D1540608732B30D0D0
:1054100006D8542B5CD0552BCDD10222092174E043
:10542000B22BC8D102B0BDE87040FFF76DBD4AF2A3
:105430001146B34258D00BD8D12B44D0B3F5967F48
:1054400057D0D02BB7D102B0BDE87040FFF7C4BD34
:105450004AF21346B34242D04AF26866B3424DD094
:105460004AF21246B342A6D102B0BDE87040FFF73F
:1054700011BF02B0BDE87040FFF7FCBCD1ED007A6F
:10548000F5EEC07AF1EE10FA54DD9FED2B7AF4EED2
:10549000C77AF1EE10FA4DD8FCEEE77A274ACDED47
:1054A000017A9DF80430A2F85230002033E0214602
:1054B00002B0BDE87040FFF74FBC214602B0BDE826
:1054C0007040FFF70BBE02B0BDE87040FFF7A2BD11
:1054D0002146284602B0BDE87040FFF7A1BC02B0EB
:1054E000BDE87040FFF70CBF02B0BDE87040FFF7A9
:1054F000DDBD02B0BDE87040FFF73ABD02B0BDE8C7
:105500007040FFF7A7BD022205210D4805F0E6FD1A
:105510000028CAD1042002B070BD02220621F4E79F
:105520000221084807F0FCF8F2E70221054807F0DD
:10553000C1F8EDE70220EEE700007F43B0820030C3
:10554000B0320030E0AA0030F6EE007A08B591EDF6
:10555000007AB4EEE77AF1EE10FA06DD01220521B9
:105560000348FDF7FDF8002008BD0420FCE700BF5C
:105570005087003030B52DED028BCD7893B00C46BE
:105580002722272D4FF0000108A828BF2725FAF071
:10559000EFFF04F10C0108A82A46FAF09FFF424BE6
:1055A000D3F8D40703685B6A9847002841D09DF878
:1055B000465068063DD400244FF07E5329060493DC
:1055C00007940694059427D504A837F067FAEA07EC
:1055D00005F006030194029403942ED4002B2ED1DF
:1055E0000D9B01930E9B02930F9B03932F480BF08F
:1055F000D9FC9DED100A044630B3B7EE001A40F214
:10560000ED40FFEE000A33F011FA234601AA04A987
:1056100026480BF0CFFC0CE0099B04A804930A9BDE
:1056200005930B9B06930C9B079337F03DFA0028DC
:10563000CDD113B0BDEC028B30BD062BD6D00121ED
:105640001A480BF04BFCF4E7DFED190AB7EE001A2D
:105650004FF49E6033F0EAF9F6EE000AB0EE408AAD
:1056600033F082F8E8B9B6EE000A124BD3F83033C3
:10567000B4EEC08AF1EE10FA08DD38EE400A30EEE2
:10568000008A93ED070A28EE000ABEE730EE480ACA
:10569000D3ED087AF0EEE77A30EE000A27EEC00A82
:1056A000B3E79FED030AB0E7B082003028B10030C5
:1056B00000000000B0A200302DE9F0439DB081460B
:1056C00008460EA9FEF76AFD844BD3F8D407036899
:1056D0005B6A984750B19DF86C30012B09D0DA1FF6
:1056E000022A06D901217E480BF0F8FB1DB0BDE867
:1056F000F083BDF86840A20504F0070604F03807FF
:1057000004F4E07501D5002DF0D04FF00008CDF87D
:105710001480CDF81880CDF81C803EBB9FED716AD7
:10572000083B9DED107ADDED117A012BDDED0F6A5E
:1057300027EE067A67EEC67A66EE866A8DED067A01
:10574000CDED077ACDED056A04D806AA05A966480D
:10575000FDF780FA9DF86C30073B022B06D86348B2
:10576000B8F076FE014605A838F062FDCDF820803D
:10577000CDF82480CDF82880F7B9DDED147A08A99A
:10578000129B4846F1EE677A0893139BCDED0A7A97
:105790000993FFF7D3FC0028A4D09FED520A08A874
:1057A00038F07AFD9DF86C30083B012B04D809AA2B
:1057B00008A94D48FDF74EFACDF82C80CDF8308081
:1057C000CDF83480EDB99DF86C309FED466A9DEDC3
:1057D000167A083BDDED177ADDED156A27EE067ABD
:1057E00067EEC67A012B66EE866A8DED0C7ACDEDFA
:1057F0000D7ACDED0B6A04D80CAA0BA93A48FDF737
:1058000029FA14F4806233D1DFED397A9DED180A5C
:105810009DF86C1020EE270ADFED327A0839012955
:1058200020EE270A8CBF0021012114F4006305BF7C
:10583000DFED2F7ADDED190ADFED2E0A60EEA70A03
:1058400004BFDFED287A60EEA70AAEB9002F35D18C
:10585000B3FA83F3B2FA82F2029105A95B092048F8
:10586000520901930BAB009208AA0BF071FF3DE7C0
:1058700000219FED200AD8E77FB9B3FA83F3012016
:105880005B090093B2FA82F30BAA5B09CDE9011020
:1058900008A913480BF0FAFC28E7002D7FF422AF8B
:1058A0000120B3FA83F3B2FA82F25B095209CDE91F
:1058B00000100BA90A480BF07FFC17E7002D3FF4FE
:1058C00011AFB3FA83F3B2FA82F205485B095209C9
:1058D000CDE9001605A90BF057FD07E7B0820030AF
:1058E00028B100300000C842B0320030B8A5003006
:1058F000E02E6542000000002DE9F047A2B080468E
:10590000084614A9FEF74AFC7E4BD3F8D407036877
:105910005B6A9847C0B1BDF88040A30504F0070951
:1059200004F4E07700D57FB10CAE30461CF03AFDB0
:10593000B9F1000F29D1DDE9150134F08FFB30B941
:10594000012171480BF0CAFA22B0BDE8F08709AA1C
:105950009DF88410404675F033F80028F0D0DDED56
:10596000177A10AD9FED697A099B284667EE877A12
:105970000093FDEEE77ADDE9151217EE903A1CF080
:1059800031FD95E80F0086E80F00002514F0380A75
:1059900006950795089514D1DDED1A7A06A9189B8E
:1059A0004046F1EE677A0693199BCDED087A07938E
:1059B000FFF7C4FB0028C3D09FED540A06A838F0B7
:1059C0006BFC09950A950B959FB99FED506A9DED6B
:1059D0001C7ADDED1D7ADDED1B6A27EE067A67EE97
:1059E000C67A66EE866A8DED0A7ACDED0B7ACDED3C
:1059F000096A14F4806805BFDFED457A9DED1E0A43
:105A00009FED440A20EE270A04BFDFED407A20EE26
:105A1000270A14F4006405BFDFED3D7ADDED1F0AAF
:105A2000DFED3C0A60EEA70A04BFDFED387A60EED6
:105A3000A70AB9F1000F31D1BAF1000F52D13046A7
:105A4000CDED050A8DED040A1CF0DCFC03289DED6C
:105A5000040ADDED050A3FF473AF10A93046CDED21
:105A6000050A8DED040A1095119512951CF040FE63
:105A700000283FF465AFB4FA84F4B8FA88F3DDED9A
:105A8000050A06AA64099DED040A5B0910A9CDF870
:105A900004A000941C480BF0D1FE55E7BAF1000FAA
:105AA0000FD10123B4FA84F409AA06A9640916489F
:105AB000CDE901A3B8FA88F300945B090BF0E6FB8B
:105AC00042E7002F7FF43CAF0123B8FA88F209A91E
:105AD0000D485209CDE90073B4FA84F35B090BF069
:105AE0006BFB31E7002F3FF42BAFB4FA84F3B8FA25
:105AF00088F23146CDF800905B09034852090BF05B
:105B000023FD21E7B082003028B100300000C842F8
:105B1000E02E6542000000004B7ACA7A10B48C7AFD
:105B200043EA042343EA0243542B07D0562B09D0FF
:105B3000522B0BD15DF8044BFFF71CBD5DF8044BF5
:105B4000FFF7BABD5DF8044BFFF7D6BE5DF8044B16
:105B500075F03EBE2DE9F04300F5A046044600274F
:105B600004F5E0492DED028BD6F8D40791B0DFEDB6
:105B70004B8A03685B699847002840F08A80D9F80F
:105B80002C3393EDE07BB7EEC77BD3EDE77AFDEEE8
:105B9000E77A27EE288A17EE903A1DB204F5A84856
:105BA00001A908F12808404611F088FF18B96BF0E8
:105BB00001FB3B4B01933722002102A8FAF0D8FCED
:105BC000A3238DF8083095238DF80930C2F04AFDE3
:105BD000D9F82433CDF80B00D6F8F807D3F8DC2039
:105BE000D3F8E0304430CDF80F10CDF81320CDF8C5
:105BF00017306DF015F80346B7EE001ADFED290AED
:105C00009F2093ED000A32F011FFD6F8F80710EE4E
:105C1000103A04F5E646CDF81B30083603681B69D8
:105C2000984710EE103A3046CDF81F3018EE103A73
:105C3000CDF82330B8F010FC20EE280A404610EED4
:105C4000103ACDF82730D9F8D432CDF82B30019B5B
:105C5000CDF82F3011F054FF10EE103A3046CDF849
:105C60003770CDF83330ADF83B50B8F001FCBDEEE5
:105C7000C00A04F59250372202A9083010EE103AFB
:105C8000ADF83D306AF0EAFB11B0BDEC028BBDE827
:105C9000F083002508EE107A80E700BF0AD7233C86
:105CA0002292CA7F0000000010B500F5E044D4F84D
:105CB0002403AFF0E9FBD4F82C13D4F82403BDE897
:105CC0001040AFF047BC000070B54FF4805105465E
:105CD00012F048F800284FD005F5E04605F592543B
:105CE000D6F82403083403689B689847692100F1BB
:105CF000A00220466AF0FCF9D6F824030368DB68AA
:105D000098476A2100F1A00220466AF0F1F9D6F81E
:105D1000240303681B6998476B2100F1A002204609
:105D20006AF0E6F9D6F82C236C21204602F52D7294
:105D30006AF0DEF92021284612F014F8E0B105F5EA
:105D4000A043D3F8D40703681B69984778B1D6F805
:105D50002C2320466E2190326AF0CAF9D6F82C2303
:105D600020466F21BC32BDE870406AF0C1B92846B8
:105D70000CF00CFB0028EAD170BD000008B515F04E
:105D80001DFFBDE8084015F06FBC00007FB50E4652
:105D90004FF6FF710446154611F0E4FFE8B11022FA
:105DA00000216846FAF0E4FBA3238DF80030952328
:105DB0008DF8013003238DF80230C2F053FCCDF88A
:105DC000030004F59250CDF8071010226946083000
:105DD0008DF80B6003956AF0C1FB04B070BD000044
:105DE0007FB50E464FF6FF710446154611F0BAFF17
:105DF000E8B1102200216846FAF0BAFBA3238DF81F
:105E0000003095238DF8013004238DF80230C2F064
:105E100029FCCDF8030004F59250CDF807101022AC
:105E2000694608308DF80B6003956AF097FB04B063
:105E300070BD000030B52DED048B87B004460D46D3
:105E4000182200216846B0EE409AF0EE608AB0EE6B
:105E5000418AFAF08DFBA3238DF8003095238DF84D
:105E6000013006238DF80230C2F0FCFBCDF80300B0
:105E700004F59250CDF807101822694608308DF8C5
:105E80000B508DED039ACDED048A8DED058A6AF0F5
:105E9000E5FA07B0BDEC048B30BD000010B54FF43F
:105EA0008011044611F05EFF30B104F5DC50BDE80E
:105EB0001040183013F098BF10BD00002DE9F04FCE
:105EC0002DED028B8DB080462F2200216846F0EE2A
:105ED000408AB0EE608A11EE10BA11EE90AA12EE6E
:105EE000109A12EE907A13EE106A13EE905A14EE96
:105EF000104AFAF03DFBA3238DF8003095238DF86E
:105F0000013009238DF80230C2F0ACFB18EE903A54
:105F1000CDF8030008F59250CDF80710CDF80B30FE
:105F20002F2218EE103A69460830CDF813B0CDF89C
:105F30000F30CDF817A0CDF81B90CDF81F70CDF81D
:105F40002360CDF82750CDF82B406AF087FA0DB0CA
:105F5000BDEC028BBDE8F08F30B52DED088B8BB01A
:105F600004460D46282200216846B0EE40BAF0EE05
:105F700060AAB0EE41AAF0EE619AB0EE429AF0EE5D
:105F8000628AB0EE438AFAF0F3FAA3238DF8003068
:105F900095238DF801300A238DF80230C2F062FBA0
:105FA000CDF8030004F59250CDF807102822694679
:105FB00008308DF80B508DED03BACDED04AA8DEDB0
:105FC00005AACDED069A8DED079ACDED088A8DEDE7
:105FD000098A6AF043FA0BB0BDEC088B30BD0000B3
:105FE0002DE9F0438FB01446054689463122002141
:105FF00001A89846DDE91676FAF0BAFAA3238DF8DF
:10600000043095238DF8053008238DF80630C2F052
:1060100029FB23683122CDF8070005F5925004933F
:1060200063680830CDF80B1001A90593A3688DF8BB
:106030000F9006933B688DF81C80CDF81D307B686F
:10604000CDF82130BB68CDF825303368CDF8293044
:106050007368CDF82D30B368CDF831306AF0FEF9B1
:106060000FB0BDE8F083000070B52DED068B8CB04D
:10607000144605460E462C22002101A8B0EE409A97
:10608000F0EE608AB0EE418AB0EE61AAF0EE429A7C
:10609000FAF06EFAA3238DF8043095238DF80530BD
:1060A0000B238DF80630C2F0DDFADFED1A7A2C22D0
:1060B00094ED007ACDF8070005F5925027EE277A87
:1060C000CDF80B1029EE279A01A968EEA78A0830AF
:1060D0008DED077A28EE278A94ED017A8DF80F600E
:1060E00027EE277A8DED049ACDED058A8DED068A8F
:1060F0008DED087A94ED027A8DED0AAA67EE277A83
:10610000CDED0B9ACDED097A6AF0A8F90CB0BDEC93
:10611000068B70BDE02E6542AE20704730B5044658
:1061200089B0144B1E2204F592556946D3F8F8073E
:106130000835B9F02FFA6A460F4928466AF02AFB5B
:1061400004F5A043D3F8D40703681B68984704F507
:1061500040530146284693F888246AF03FFB04F533
:10616000DC50183015F092FF04F5907025F04CFCCF
:1061700009B030BDB0820030BEB11608434B444A6E
:1061800070B54360002342634FF080424361044690
:106190008361483040F82C3C4FF4306540F80C3CAB
:1061A0003C4B40F8102C40F8083C3B4B3B4E40F831
:1061B000043CACF0E5FB04F5827088F077FB04F555
:1061C0002B6076F075FF364BC4F8B03A601977F063
:1061D00027F966513035B5F5606FF7D104F5606089
:1061E00004F5805678F080FF04F5C45000212D4D51
:1061F0000C30BCF005FC04F5C9501C30BDF0D6F8DD
:10620000C6F85C5904F5CB50BDF04EFEA5F5E7632A
:1062100004F5CF50C6F8F0391C308EF0ABFDA5F573
:106220000C7304F5DE50D435C6F8B43B9FED1E1A4E
:106230000430DFED1E0A9FED1E0AC6F8C05BAFF00A
:1062400039FF9FED191A04F5DE509FED1A0AF0EEA2
:10625000410A1C30AFF02EFF9FED131A04F5DF50FA
:106260009FED140AF0EE410A1430AFF023FF04F55D
:10627000E2500430B4F0AAFC20460F4960F0CAFA9C
:1062800020460E4960F0C6FA204670BD78410030C5
:106290000000C8410AD7233C0000E04018AF1608B0
:1062A0002CAF160880B50030000000009A99993E86
:1062B0000000B44300804A43B4A11608A4A4160801
:1062C00070B5ADF50E7D4B4DD0224B4906465AA810
:1062D000FAF004F90EAC0FCD0FC40FCD0FC40FCDE3
:1062E0000FC495E80F0084E80F0000245AABB7EE06
:1062F000000A0021181910345FF04CFFD02CF5D1A2
:106300003E4B02AC0FCB84E80F0001A920465FF0A2
:10631000F5FE90B19DF90430F0EE007ADFED386AB9
:10632000B7EE000A07EE103AE068B8EEC77AE7EE7B
:10633000267A80EE270A60F00BFE00240EAB0021C7
:1063400018191034B7EE000A5FF024FF402CF5D185
:1063500090222C4936A8FAF0C1F80022092136A86B
:106360005FF0C2FF96F9146BD6B9274D1EAC0FCD66
:106370000FC40FCD0FC40FCD0FC495E80F0084E8F4
:106380000F00324604211EA85FF0AEFF9FED1F0AEA
:106390001F4860F0DDFDB7EE000A1E4860F0D8FD32
:1063A0001D4C06AD9FED1D0A0FCC0FC594E80F00E4
:1063B00085E80F00002106A85FF0ECFE00219FEDAC
:1063C000170A28465FF0E6FE04F11001002460225F
:1063D0001EA8FAF083F81EABB7EE000A00211819C8
:1063E00010345FF0D7FE602CF5D178F0F7FB0DF597
:1063F0000E7D70BD1C4616084C4516085C461608F6
:10640000CDCCCC3D6C461608FC46160800000000BA
:106410009CA01608ABA016083C47160800003442A2
:1064200010B5B4B00024D02207496846FAF056F8F7
:106430000DEB04001034B7EE000A00215FF0AAFE55
:10644000D02CF5D134B010BDBC4716082DE9F0476B
:1064500090B01D200DF1060178F0B2FC002800F08C
:106460009E809DF806301121604A0BA80133DBB2F3
:106470008DF80630C1F0A8FA00220DF107010BA833
:106480005FF070FB9DF80630594A112105460BA8B4
:10649000C1F09AFA00220DF107010BA85FF062FB30
:1064A0009DF80630534A112106460BA8C1F08CFA1C
:1064B00000220DF107010BA85FF054FB9DF8063098
:1064C0004D4A112103F03F0307460BA8C1F07CFAA7
:1064D00000220DF107010BA85FF044FB8046002D60
:1064E0005DD0002E5BD0002F59D0002857D0284611
:1064F0005FF04EFD002852D130465FF049FD002884
:106500004DD138465FF044FD002848D140465FF049
:106510003FFD002843D1394C0DF10C0C0DF11C0945
:1065200094E80F0010348CE80F0094E80F0089E81D
:106530000F0002A960465FF0E1FD98B3BDF8084086
:1065400002A948465FF0DAFD00284AD0BDF80830BD
:1065500054BB23B340F2E2449C420FFA84FA0FFA90
:1065600083F927D80DF10A013046ADF80A9060F0A2
:10657000E5FF0DF10A012846ADF80AA060F0DEFF44
:106580000DF10A013846ADF80AA060F0D7FF0023EC
:106590000DF10A014046ADF80A3060F0E9FF10B095
:1065A000BDE8F0870024CBE740F2D662002B08BF9D
:1065B0001346D1E70DF10A013046ADF80AA060F0AC
:1065C000BDFF0DF10A012846ADF80A9060F0B6FF54
:1065D0000DF10A013846ADF80A9060F0AFFF0123D3
:1065E000D6E7002CDBD040F2D663B5E7BCA0160896
:1065F000C8A01608D4A01608E1A016088C481608F2
:1066000037B500F55951044678220125383167F035
:10661000B3FF00220C2126485FF066FE2046FFF7FC
:1066200015FF04F55A50B7EE000A002202210C3083
:106630005FF0E2FE04F54D5100231E4A343145203F
:1066400000955FF055FE1C4A1368D90708D404F57D
:106650003E531A49156030330B6004F59853CB60F4
:1066600004F55B5002221549012530305FF092FE9F
:1066700004F592510023124A0831FD2000955FF085
:1066800037FE104B012110481A68D2075FBF0E4A2F
:1066900004F5D6541D6014605FF098FE60F0BEFAF9
:1066A0000A4A138843F00103138003B030BD00BFD2
:1066B000F4A01608D84E18081CB70030C4250030C6
:1066C000288E170820B70030DC250030A0B9003034
:1066D0000F299DBF302303FB01005030002070477D
:1066E000014B93F9BF067047B0620030024B93F83C
:1066F000ED0700F001007047B0820030044BB3F8A2
:106700008436DB075ABF0069C0F340100020704791
:10671000B0620030014BD3F888037047B08200307C
:1067200008B503689B68984730B9044B93F9EC07A8
:10673000B0FA80F0400908BD0020FCE7B0820030CC
:1067400038B50C1E2EDB184DE3B295F894239A420F
:1067500028D3D5F890330122A5F5A040195D04F0A7
:10676000BDFCF8B176F026FE032177F0DBFFC8B957
:1067700076F020FE0D2177F0D5FF98B9A5F50052EF
:10678000A5F5A04092F9A436E340DB0756BF92F985
:10679000BE160221E140BDE8384058BF01F00101BA
:1067A000FCF7E8B838BD00BFB0820030022910B550
:1067B000044606D1014635220948BDE8104004F0E0
:1067C0008DBC084BD3F8D40703681B6898478442F4
:1067D00005D176F0EFFDBDE8104076F075BD10BD37
:1067E000B0320030B082003029B1022907D1044B09
:1067F000C3F8CC177047024B0122C3F8CC2770476F
:10680000B082003031B1022907D1044B012283F854
:10681000D0277047014B83F8D0177047B082003003
:1068200000F5A043DFED186A9FED187A012110B53D
:10683000D3F880230446D3F87C3300F5DC50B2F95A
:106840000820B3F90830183007EE902AF8EEE77AFE
:10685000C7EEA60A07EE903AF8EEE77A87EEA60AA8
:1068600060EE870A20EE070A15F04AFA6AF0A2FCE9
:1068700026216AF0DBFB04F5AA40054A06216030B8
:10688000BDE810406DF064B80000C84235FA8E3C97
:10689000F0AC160800F5E042002300F5AA400621FE
:1068A00082F84033024A60301372024A6DF050B8E9
:1068B0000DB90030FCAC1608F8B500F5E04504460B
:1068C00095F84013002955D02B4B2C4AD3F8D40708
:1068D000904204D1D3F8F83793F8CB3023B920464F
:1068E000BDE8F840FFF7D6BF254E012004F5A043D0
:1068F00095F84173307293F9C827C7BB002A39DB7A
:1069000085F841030139DFED1F6A9FED1F7A04F519
:10691000DC50C9B2183085F84013B1FA81F1D3F8D0
:106920008023D3F87C334909B2F90820B3F9083041
:1069300007EE902AF8EEE77AC7EEA60A07EE903A3D
:10694000F8EEE77A87EEA60A60EE870A20EE070ADD
:1069500015F0D6F995F8403363B904F5AA403372BF
:106960000A4A06216030BDE8F8406CF0F1BF002A09
:10697000C8DAB4E7F8BD00BFB082003014B300300D
:106980000DB9003000007A4535FA8E3C10AD16087E
:106990006D2900F3E380012901DC77F0A9BC8B1E8F
:1069A0006B2BFAD80FF2040C5CF823F0BB6B0608D3
:1069B000B56B0608BB6B0608BB6B06089B6906082F
:1069C000BB6B06089B6906089B690608B56B060841
:1069D0009B690608BB6B0608B56B0608B56B060815
:1069E0009B690608BB6B0608BB6B0608BB6B0608F9
:1069F0009B6906089B690608B56B0608BB6B060811
:106A0000B56B06089B690608B56B0608B56B0608EA
:106A10009B6906089B6906089B6906089B6906082E
:106A20009B690608B56B0608BB6B06089B690608E0
:106A30009B6906089B690608BB6B06089B690608EC
:106A4000B56B06089B6906089B690608BB6B0608C0
:106A5000B56B0608B56B0608BB6B06089B69060894
:106A6000BB6B0608BB6B0608BB6B06089B69060878
:106A70009B690608BB6B06089B6906089B690608AC
:106A8000BB6B0608BB6B0608BB6B06089B69060858
:106A90009B690608BB6B0608BB6B06089B6906086A
:106AA0009B6906089B6906089B6906089B6906089E
:106AB0009B690608BB6B0608BB6B0608BB6B060828
:106AC000BB6B0608BB6B0608BB6B06089B69060818
:106AD000B56B0608B56B06089B6906089B69060836
:106AE0009B6906089B6906089B6906089B6906085E
:106AF000BB6B0608B56B06089B6906089B69060810
:106B00009B6906089B6906089B6906089B6906083D
:106B10009B6906089B6906089B6906089B6906082D
:106B20009B6906089B6906089B6906089B6906081D
:106B3000BB6B06089B6906089B6906089B690608EB
:106B40009B6906089B6906089B6906089B690608FD
:106B50009B6906089B690608B56B0608A12921DC1C
:106B600096297FF71AAFA1F197030A2B3FF615AFCD
:106B70000FF2040C5CF823F0BB6B0608BB6B060835
:106B80009B690608BB6B06089B6906089B6906089B
:106B90009B6906089B690608B56B0608B56B060875
:106BA000BB6B0608B42908D0DB2903D0B2297FF4D7
:106BB000F4AE7047002377F06DBB7047632970B562
:106BC00014468AB000F3D280012905DC22460AB0BF
:106BD000BDE8704077F06CB88B1E612BF6D801A22F
:106BE00052F823F0E76D0608FB6D06081B6E0608D9
:106BF000256E0608CD6B0608556E0608CD6B060897
:106C0000CD6B0608056F0608CD6B0608CD6B060830
:106C1000096E06082B6F0608CD6B0608FF6E060886
:106C2000676F0608776F0608CD6B0608CD6B060800
:106C30008F6F06089D6F0608AB6F0608CD6B0608C0
:106C4000D16F0608E36F0608CD6B0608CD6B06080A
:106C5000CD6B0608CD6B0608CD6B0608F56F0608F0
:106C60000F700608CD6B0608CD6B0608CD6B0608C5
:106C700015700608CD6B06081B700608CD6B06085C
:106C8000CD6B060835700608CD6B06083B7006080C
:106C9000EB6D0608CD6B0608CD6B0608CD6B0608BC
:106CA000CD6B0608CD6B0608CD6B0608DB700608B9
:106CB000CD6B0608CD6B06087D6F0608836F06084E
:106CC000896F0608CD6B0608CD6B06085B70060859
:106CD00091700608CD6B0608CD6B0608CD6B0608D3
:106CE000CD6B0608CD6B0608CD6B0608C97006088B
:106CF000CF700608D5700608E1700608E770060830
:106D0000ED700608CD6B060831710608F3700608B1
:106D1000CD6B0608CD6B0608CD6B0608CD6B06085B
:106D2000CD6B0608CD6B06086571060883710608F1
:106D3000CD6B0608CD6B0608CD6B0608CD6B06083B
:106D4000CD6B0608CD6B0608CD6B0608CD6B06082B
:106D5000CD6B0608CD6B0608CD6B0608CD6B06081B
:106D6000CD6B0608CD6B060899710608A0291FDCBB
:106D700096297FF72BAFA1F19703092B3FF626AF9A
:106D800001A252F823F000BF9F710608A571060802
:106D9000CD6B0608B9710608CD6B0608CD6B0608E9
:106DA000CD6B0608CD6B060891710608DD710608EB
:106DB000B42900F0DB80DB2917D0B2297FF406AFBD
:106DC000002A00F0C881022A0FD1A54BD3F8D407BE
:106DD00003689B6F984740B974F056F8A14A0421A4
:106DE0006CF0B6FD01E0022C01D001242FE0352229
:106DF0000E219D4804F072F9F7E7211E18BF01210A
:106E00009948FBF7B7FDF0E7012C04D0022C14BF22
:106E100000210221F4E72146F2E721460620FFF790
:106E2000C5FCE2E7022CE0D18D4DD5F8D40703680C
:106E3000DB6A984704460028D7D0D5F88433B3F9E5
:106E40000830002BD1D1A5F5A040FFF7E9FC204682
:106E50000AB070BD022CC8D1814D844BD5F8D4271F
:106E60009A42C2D0D5F8F83793F8CB30002BBCD07B
:106E700005F50054B4F9A0382BB9D5F88433B3F92B
:106E80000830002BB1D005AE1C22002103A8F9F078
:106E90006FFB30461BF086FAB4F9A03893B916237D
:106EA00003A97348ADF80E30D4F8FC32642BB8BF98
:106EB0006423069338F0AEFC20B16AF07BF92721F9
:106EC0006AF0B4F804F53E7494E80F0086E80F0009
:106ED000D5F8843303A96648B3F90830002BCCBF3A
:106EE00010231523ADF80E3038F094FC00283FF441
:106EF0007CAF6AF05FF927216AF098F875E72146C0
:106F000003208CE7022C04D0554B002283F89823F1
:106F10006BE71921574860F0B9FF04460028F3D009
:106F20004F4B012283F8982391E7012C0BD0022CC0
:106F300012D0002C7FF459AF4F4B83F8E8466AF02B
:106F400039F92B21D8E74C4B83F8E8466AF032F93F
:106F50002C216AF06BF87AE7474B83F8E8466AF031
:106F600029F92D21C8E721460F2058E7114643484B
:106F7000BFF036FF39E72146092050E721460420BB
:106F80004DE7214605204AE72146172047E7A01E86
:106F9000414241413A4881F0FDFF26E7022C7FF44F
:106FA00024AF314801F014FE1FE7012C06D0022C5B
:106FB00009D0002C7FF419AF2146EBE72146304879
:106FC00081F0E8FF43E701212D4881F0E3FFE8E786
:106FD000A21E2C4B5442D3F82433544183F8204052
:106FE00003E7A31E59425941264BD3F82403B0F0BE
:106FF0008DF9FAE6013C1A4B012C93F8CA278CBF95
:107000000024012464F3041283F8CA27EDE6214624
:10701000112004E72146122001E7012234B1022C9D
:107020007FF4E3AE174B83F8402FDEE6154B83F871
:10703000404FDAE621461520F1E6012C08D9022C52
:107040007FF4D3AE9FED100A1048BCF011FACCE6E5
:10705000034B002283F83A20C7E621461820DEE6DB
:10706000B08200304BAD1608B0320030E0AA0030DC
:107070001CAB003048420030B062003048AE0030F7
:1070800064A70030B0A2003000000000DC820030B5
:10709000594BD3F8D407594B98427FF4A6AE0190D0
:1070A0000FF09CFA012C019808D0022C0AD0002C79
:1070B0007FF49BAE21460FF041FB96E600210FF0D6
:1070C000A5FAC4E60121F6E721460020A7E62146FD
:1070D0001020A4E621460220A1E6214601209EE6DA
:1070E000214616209BE62146072098E621460B20E4
:1070F00095E6022C424B0ED1012483F890476AF0AA
:1071000059F84A2169F092FF73F0BEFE3D4A06210C
:107110006CF01EFC9BE6002283F890276AF04AF888
:107120004B2169F083FF73F0AFFE374A062157E623
:10713000012C09D0022C0CD0002C7FF456AE01217A
:10714000324810F0F3FC50E60021304810F0EEFC1D
:107150007DE62146F4E7284BD3F8D4070368DB6FBC
:10716000984742E6244BD3F8D407244B98427FF447
:107170003CAE022C02D10FF0EBFB36E60FF0D2FA58
:1071800033E62146FFF730FB214804F0EDFC2CE606
:107190002146FFF737FB28E621461B203FE6214624
:1071A0001C203CE6022C7FF420AE1A48FCF708FABB
:1071B00073F06AFE184AB9E7214676F0D9FB174802
:1071C000ACF0F8FD044600283FF40FAE0A4A92F8EE
:1071D000CB3743F0020382F8CB3738E6012234B1D3
:1071E000022C7FF402AE044B83F86023FDE5024BD2
:1071F00083F86043F9E500BFB082003054B6003038
:10720000B0A2003028AD160839AD1608D886003077
:1072100064AA0030B032003064AD160850870030E8
:1072200010B504460448B7F015F904F10801BDE8AB
:10723000104032F091BE00BFB8A5003038B504460A
:1072400012482DED028BB7F00BF9054636F0C0FB66
:107250000F48B0EE408A10F01FFD90B1DFED0D7ABF
:10726000B4EEE78AF1EE10FA0BDDD5ED000A95EDEC
:10727000010AF6F0EFFADFED087A20EE270A84ED36
:10728000080A94ED080ABDEC028B38BDB8A50030A1
:10729000B032003000401C46E02E6542074B93F9A7
:1072A000A506022805D0032806D0003818BF012003
:1072B000704781F00100704704207047B0620030D1
:1072C00003688B4216D00429C0E9001302D00729B5
:1072D0000ED07047084B9FED097A03F69853D3ED13
:1072E000007AF8EEE77A67EE877AC0ED087A7047A1
:1072F00000238362704700BFB04200300AD7233CAE
:10730000024608B5FFF7CAFF01461046BDE808402F
:10731000FFF7D6BF70B5044616460D462DED048B1B
:10732000F0EE408A9FED349AB0EE608ADFED339A3A
:10733000C1F090F9E0616EB3236843B9304B03F6B6
:107340009853D3ED007AF8EEE77AC4ED097A68EE47
:10735000898A002DB7EE000AFFEE007A20FE270A88
:1073600068EE808AC4ED058AB4EEE98A254BD3F82D
:107370002403F1EE10FA30DAAEF082FF20EE090AB3
:1073800084ED060A20460321BDEC048BBDE8704065
:10739000FFF796BF94ED090A98EE890A31F0DEFAFC
:1073A000002D84ED050A0BDAB4EEE90AF1EE10FACD
:1073B000DADBDFED157A30EE670A84ED050AD3E7F4
:1073C000D2D0DFED127AB4EEE70AF1EE10FACBD8A4
:1073D000DFED0D7A30EE270AEFE7AEF051FFB4EEA5
:1073E000480AF1EE10FA48BFB0EE408A28EE098A4A
:1073F00084ED068AC6E700BF0000C84200000034E2
:10740000B0420030B0A2003000A00C47000000B431
:1074100010B52DED028BF0EE408A0446B0EE608A86
:10742000C1F018F9DFED090A0621E061204668EE97
:10743000A08A68EE200AC4ED098AC4ED0A0ABDECF0
:10744000028BBDE81040FFF73BBF00BF0000C84201
:1074500010B504462DED028BB0EE408AC1F0FAF86B
:1074600094ED090ADFED097AE061A8EE270A31F010
:107470005FFA0023204684ED090AA3620621BDECD1
:10748000028BBDE81040FFF71BBF00BF0000C842E1
:1074900070B54B6806460C46144D73B98B6863B9DA
:1074A000C96851B91248FFF72BFF95F83D1405F54F
:1074B0007170BDE8704078F0C3BF95F83D140D4879
:1074C00078F05EFE48B906F1080120461BF010F97D
:1074D00018B102210648FFF7F3FE224695F83D1445
:1074E0000448BDE8704078F09FBF00BFB0A20030F4
:1074F00024B7003074A60030072108B5FFF7E0FE7E
:1075000080ED0A0A08BD000008B50368032B23D1EB
:10751000D0ED057A9FED127AF0EEE77AF4EEC77AB5
:10752000F1EE10FA1AD50F4B90ED090A03F69853B5
:10753000D3ED007AF8EEE77A37EEC00A31F00EFAB2
:10754000B0EEC00ADFED087AB4EEE70AF1EE10FA09
:1075500094BF0120002008BD0120FCE70020FAE7CD
:1075600000000034B04200300000484330B50368EA
:1075700085B00446023B082B6FD8DFE803F0050D09
:1075800030374D6341636300FFF74AFE84ED090A1B
:1075900094ED090A05B030BDC1F05CF8E369DFED98
:1075A000320AC31AE06194ED050AF12007EE903A21
:1075B000F8EE677A67EEA07AD4ED060A20EEA71AF5
:1075C00067EEE00A31F032FAD4ED057A77EEC07A50
:1075D000C4ED057AD4ED097A37EE800AD6E7FFF7D5
:1075E0002DFEDFED227A20EE270ACFE7204B03F5B0
:1075F0000263D3ED007AF8EEE77AC0ED097AC7E7C7
:107600001C4DD5F83803B4F091FD0028C0D0D5F852
:1076100038331B6C6362BBE7C1F01CF8E3699FED74
:10762000127AC31AD4ED0A6AE06107EE903AF8EED6
:10763000677A67EE877A94ED097AA6EEA77A84EDE9
:10764000097AA5E70B4B9FED0C0AD3F824036C30A5
:1076500036F0CEFD84ED091A9AE7064BD3F82C33A9
:10766000D3F85033D6E700BF6F12833A0000C84208
:10767000B0820030B0A200309F0CB3450368092BE4
:1076800008D8DFE803F0050A05050505070705101A
:107690000023836290ED0A0A7047044BD3F82C3321
:1076A000D3F85433F5E7C36AF3E700BFB0A2003064
:1076B000F0B5304D04460E46D5F8D4072DED028BBB
:1076C000036889B0D3F88030984700283FD005F58B
:1076D0000057D5F8D40703F061FB08EE100AD7F87D
:1076E0002C33D7F82403D3EDD28A0368D3F898302B
:1076F0009847D7F82C33D5F8D40778EEC00A93ED25
:10770000D31A0368CDED050A9B6C8DED041A9847DA
:107710000390D5F8D4070268D26C9047B8EEC88AB7
:107720009FED150A3246009007A928EE000A039B38
:107730009DED041A05F54D70DDED050AB3F05EFA16
:1077400048B10A212046FFF7BBFD079BA36209B0A1
:10775000BDEC028BF0BD23680A2BF8D100236168D1
:107760002046A36211B9FFF7CBFDF0E7FFF7A8FDB4
:10777000EDE700BFB08200300AD7233CF8B5002304
:10778000264F04460D46CB6297F8ED37244E13F092
:10779000010F37D1D7F8D40703685B6F984788B3D8
:1077A000D7F8D40703F056FE85ED0B0AB0EEC00AF9
:1077B000DFED1C7AB4EEE70AF1EE10FA03D40921EA
:1077C0003046FFF77DFDD5ED0B7A2846FDEEE77AD2
:1077D00017EE903A19B2FFF76BFF1148FFF7C6FE9C
:1077E0000F4884ED000AFFF749FF336884ED010A72
:1077F0000A2B0FD8DFE803F00C1010101010100C3B
:10780000100C0C003368092BDDD100210448D8E7A7
:107810000223A3602046F8BD0123FAE7B0820030BE
:1078200024B7003000000034034B01221A6000220C
:107830009A60DA601A61704724B7003013B50446C5
:1078400001A910F0A5F804F5E04320B9012283F85E
:107850006D2402B010BD03F58C62DDED017ADFED21
:10786000086AB8EEE77AD2ED007A67EEA67AB4EE4F
:10787000E77AF1EE10FA54BF01220022E7E700BFD9
:107880000000C84210B5044600F5EB40703098F097
:10789000ABFE04F5EE40BDE810402030BAF0A0BCCD
:1078A00008B50F22084803F019FC60B90F22062121
:1078B000054803F013FC30B90F2209210248BDE846
:1078C000084003F00BBC08BDB032003070B5154E57
:1078D00004460D4696F8ED37DA0622D56FF3041309
:1078E00086F8ED37A6F5005669F064FC00221421F5
:1078F00069F0BCFB96F888340E2B12D1022D0AD009
:10790000032D0AD0012D0CD194F854102046BDE867
:107910007040FFF7C5BF0621F8E794F8541003291B
:10792000F4D070BDB082003010B50E4C49B9D4F817
:10793000D40703681B689847A0F1130358425841C5
:1079400010BDD4F8D40703681B6898471328EED0FD
:107950000E221321A4F5A04003F0C0FB0028E6D1BD
:10796000EEE700BFB082003030B50D4689B0114659
:10797000FFF7DAFF0446F0B104A81AF013FD14F083
:107980001DF904A913F090FE28B12869059B8342D4
:10799000D4BF002001209FED127A124B8DED017AA9
:1079A000D3F830238DED027A40B1D369039301A956
:1079B0000D4807F06DF9204609B030BDD2ED087AC8
:1079C000A3F58041D3F8FC22F0EEE77AD1F88C36AB
:1079D0009A42F1EE677A67FE877ACDED037AE6E7A1
:1079E00000000000B0A200300CB40030F0B50F462B
:1079F00085B011460646FFF797FF044658B10025AB
:107A000001AA39463046019502950395BAF0F4FC77
:107A1000044618B90024204605B0F0BDDDED017A1A
:107A20009FED177AF0EEE77A0395F4EEC77AF1EE60
:107A300010FA08D5DDED027AF0EEE77AF4EEC77AB7
:107A4000F1EE10FAE6D401A836F0F0FF01A836F006
:107A500037FC0C4B9DED017A01A9D3F83033DDEDF5
:107A6000027AD3ED066A084827EE267A67EEA67AF0
:107A70008DED017ACDED027A07F00AF9CBE700BF70
:107A800000000034B0A200300CB4003070B50E46D7
:107A9000114605462DED028B84B0FFF745FF0446E5
:107AA00080B39FED238A01AA314628468DED018AD5
:107AB0008DED028A8DED038ABAF09EFC044608B370
:107AC0001C4B9DED017AD3F83023DDED027AD2ED27
:107AD000066A27EE267A67EEA67A8DED017A9DED8D
:107AE000037ACDED027AB4EEC87AF1EE10FA0EDD2B
:107AF000D2ED077A67EE877A01A90F48CDED037AB8
:107B000007F0C6F8204604B0BDEC028B70BDD2ED84
:107B1000087AA3F58041D3F8FC22F0EEE77AD1F899
:107B20008C369A4267EE877A67FE887AE4E700BF70
:107B300000000000B0A200300CB400302DE9F0418C
:107B40003D4F14460646884697F8ED37DA0616D4B8
:107B5000D7F8D40743F01003012587F8ED37036801
:107B60001B68984786F85400D7F8D40703681B6849
:107B70009847092805D100242046BDE8F08100255A
:107B8000F2E7D7F8D40703681B6898471228F2D0A9
:107B9000D7F8D40703681B6898470E28EBD0012C50
:107BA00012D8062C38D801A353F824F0797B0608A4
:107BB000197C06080B7C06081F7C06082B7C06082F
:107BC000E17B0608017C06081C4801F05FFE0028E6
:107BD000E7D001220A211A48FAF7C2FD00241BE06F
:107BE000002DC9D00E220621144803F077FA00B9FF
:107BF000002469F0DFFA2246142169F037FABBE766
:107C0000002DB9D00E220521EEE72A464146304626
:107C1000FFF7AAFE0028E1D0002DADD0E9E72A4603
:107C200041463046FFF7E2FEF4E72A464146304639
:107C3000FFF72CFFEEE700BFB0820030B03200301B
:107C40005087003000F540532DE9F04F00F5DC5926
:107C5000054600F5E04409F118092DED068B93F96E
:107C6000FA368BB043B100F5A047D7F8F83793F850
:107C7000CB80B8F1000F0FD10021A4F8841748463B
:107C800014F02CFA94F8851748460BB0BDEC068B1F
:107C9000BDE8F04F14F02CBAC0F0DCFC8346D4F8F9
:107CA0002C0307AE9FED968A90EDE4AAB1F06CF933
:107CB000002800F0CD80D4F82C3303F5657393E8E9
:107CC000070086E8070030468DED098A36F0AEFEE3
:107CD000B0EE409A05F5E64A28460FF0DDFF0AF1BE
:107CE000080A002800F0B7805046B6F0B9FB07C874
:107CF00086E8070030468DED098A36F097FEF0EEF3
:107D0000409AD7F8D40703681B689847122840F0B8
:107D1000AB80002384F88437D7F8D40703685B6905
:107D2000984728B1D7F88433B3F90830002B0CDC1E
:107D300097F9C837002B08DA5046C4F888B7B6F070
:107D40008BFB04F28C7383ED000A94F884375BB1EB
:107D5000D4F8880741F28833ABEB000B9B4540F227
:107D60009180002384F88437D4F824039FED650ABA
:107D70006C3036F03DFA04AB8DED070ACDED080A04
:107D80008DED091A9FED600A96E8070001AE83E8C1
:107D9000070086E80700304636F02AFA2846B0EE9B
:107DA000408A8DED040AF0EE608ACDED050A8DED76
:107DB000061A0FF071FF002876D0DFED547AF4EE4A
:107DC000E79AF1EE10FA94BF01250025D4F82C03B0
:107DD000B1F0DAF830B1DFED4D7AB4EEE79AF1EEBA
:107DE00010FA0AD9002D66D1D7F8D40703681B68AA
:107DF0009847022866D04FF00008D4F82C03B1F061
:107E0000EDF90546002876D0B5EEC0AAF1EE10FADD
:107E100070D5DFED3F7AB4EEE7AAF1EE10FAACBF11
:107E2000012600265046B6F023FB66B9B0EEC00A24
:107E3000DFED387AB4EEE70AF1EE10FA5DD8002DE6
:107E400008BF4FF0000894F8841784F8858716E778
:107E5000B0EE489A3EE728460FF0E6FE00287FF491
:107E600043AFDFED279A4CE7D7F8F83793F8CB30DC
:107E7000002B3FF451AF97F9C837002BBFF64CAF3A
:107E8000012347E75046B6F0E7FA04F28C73D3EDCE
:107E9000007A30EE670ADFED207AB4EEE70AF1EE01
:107EA00010FA3FF75EAF5FE728460FF0BDFE0546CC
:107EB000002882D18AE7D4F82C03B1F065F80028B5
:107EC00092D19AE7B0EE680AF4F056FCF0EE408AE0
:107ED000B0EE480AF4F050FCDFED107A20EE280AEC
:107EE000B4EEE70AF1EE10FACCBF4FF001084FF004
:107EF000000882E700252E4694E7B046A3E700BFBE
:107F0000000000009F0CB345D30237390000FA424D
:107F10000000C8C2000070420000484255CF7D3FBB
:107F200038B504460FF0B8FE04F5DC55183548B9ED
:107F300020460FF079FE014620B92846BDE83840BA
:107F400013F0E6BA04F5A044D4F8D40703689B6C98
:107F5000984720B9D4F8D4070368DB6C98470146EA
:107F6000EBE7000030B5044689B004F5DC556846FF
:107F70001AF018FA04A818351AF014FA69462846B7
:107F800013F092FB98B104A9284613F0FFFB70B1DF
:107F9000059B00226946204601932368DB6C9847C5
:107FA00028B104F59E4001217C30BAF0F5FF09B0FC
:107FB00030BD000000F5805292F8142ED2070BD489
:107FC00000F5A042D2F8F82792F8CB1009B1FFF7DC
:107FD000C9BF03689B6C18477047000030B587B075
:107FE000044602A801911AF0DDF904F5DC5002A95B
:107FF000183013F059FB019A18B90025284607B02C
:1080000030BD236802A92046DB6C9847054600284E
:10801000F3D004F59E4001217C30BAF0BDFFEDE7BE
:10802000F0B5044685B00F46154604F5DC566846A3
:108030001AF0B8F969461836304613F0A7FB10B9A4
:10804000002005B0F0BD3946304613F0D3F90028C2
:10805000F6D0002DF5D004F58054284694F8143E4F
:1080600043F0020384F8143EEBE700002DE9F04FE3
:108070002DED0A8BBDB0044624220E4618A800211F
:10808000F8F076FA2422002121A8F8F071FA2422CF
:1080900000212AA8F8F06CFA2422002133A8F8F075
:1080A00067FA04F5A0450023CDE90D330F9395F849
:1080B000C93713F0080837D143F0080395F878233F
:1080C000079285F8C9371BF00FFC90F9253003B3F0
:1080D00090F84433EBB104F2EC67C24638461BF02B
:1080E000FBFA5FFA8AF194F812378B421FD93846AF
:1080F0000AF1010A1BF0CEFA81460028F1D1C94AE3
:10810000022130466FF022F995F8C93769F3C303AD
:1081100008E0C54A022130466FF018F995F8C937D2
:108120006FF3C30385F8C9374FF001083CE304F54A
:10813000A9430121203318460BEE903AFAF79CF838
:10814000814608B9B94ADBE720460FF093FAD5F823
:108150008433B3F90890B9F1000F01D0B44AD9E7DC
:1081600095F9C837002B01DBB24AC9E720469FEDDD
:10817000B28A01F091FE04F5B0434A460CA92433BB
:1081800018460CEE103A16F0A7FF00284FF08F01AA
:1081900013AA14BF02230123307C0393F123ADF80B
:1081A0005490CDE913390A234FF00009CDE900318D
:1081B00003234D216CF062FCA04B012206213046C6
:1081C0005A729F4A6FF0C2F8039B06213046022B79
:1081D0000CBF9C4A9C4A6FF0B9F804F540534946DD
:1081E000384683F8B2961BF0B9F95FFA89F194F832
:1081F00012378B420CD913AA38468DED138A09F138
:1082000001098DED148A8DED158A1BF025F8ECE738
:108210004FF0000A4FF07C0B38461BF05DFA5FFA16
:108220008AF994F812274A4519D9494638461AF06E
:1082300005FF3CAAC0B20C230AF1010A0BFB004067
:1082400003FB092C00F5F060ACF1900C07C88CE83A
:1082500007003CAA02EB890909ED2F8ADFE741F20A
:1082600088310AA82CF090FCD5F8F8079FED729A97
:108270000368F0EE499A9FED75AA9B6A9847D5F876
:10828000F80701210025B7F087F8714BDFED71AADF
:1082900001211B68D86A029303681B689847C0F0E5
:1082A000D9F90590C0F0D6F9069004F5A049079ACF
:1082B00099F87833934240F0D58094F8321A3846D2
:1082C0001BF0E8F9002800F0CD80D9F8F83793F8D2
:1082D000CB300493002B00F0C58041F288310BA80D
:1082E0002CF052FCC0F0B6F9059BC01A132840F2DE
:1082F000D680C0F0AFF9059020460FF0BBF977F0BB
:1083000043F8824676F0CAFFD9F88433D9F8F807E3
:10831000B3F9083000EE103AB8EEC00A20EE0A0AAF
:10832000B8F0FEFD504676F0C1FF38461BF0D4F998
:108330001CEE100A17F0B0F8D9F88433A220B7EE7B
:10834000001AB3F90830DFED3C0A00EE103AB8EE3F
:10835000C00A20EE0A0A30F069FBB4EEE90A0022F6
:108360000CA91CEE100AF0EE408AF1EE10FA58BF8C
:10837000F0EE409A16F0B0FE08B900230C939DED84
:108380000C8ADFED357AB4EE498AF1EE10FAF4EE9C
:10839000E78A48BFB0EE498AF1EE10FA80F28D808C
:1083A0004FF0000A9FED2D9ADFED2D8A5FFA8AFBD0
:1083B00094F812375B4540F294814FF00C0918ABEA
:1083C000B0EE490A0AF1010A09FB0BF903EB0900B7
:1083D00035F00EFF59463846CDED110A8DED121AD3
:1083E0008DED100A1AF02AFE7C23C0B2B0EE680AA6
:1083F00003FB004000F5F06035F0FAFE3CAB13A93A
:1084000010A899448DED130ACDED140A8DED151ABF
:1084100035F0C2FE09ED240A49ED230A09ED221ABE
:10842000C4E700BF69AF160858AF160887CC160816
:1084300077AF160889AF1608000000000DB90030AC
:1084400094AF1608A9AF1608674D16086F12833A45
:1084500018B700300000C84200000034A4707D3F0F
:108460000AD7233CD9F8F80703689B6A984700218C
:10847000D9F8F807B6F090FF029B0021D86A03688C
:108480001B689847002D40F05F813046C94A05219E
:108490006EF05CFF294638461BF060F870E1029BE5
:1084A000B0EE498A0521986A03685B6898470BA873
:1084B0002CF076FBB0EE489AF7E64FF000094FF04B
:1084C0000C0B04F22C7A5FFA89F394F812279A4283
:1084D00022D91946384608931AF0B0FD089B4FF090
:1084E0007C0CC0B209F101090BFB03F13CAB0CFBA6
:1084F00000A05A185430A2F16C03CDE9083218AB31
:10850000194435F05FFE089B099A02ED1B0AC3ED82
:10851000010A83ED021AD6E7039B4FF0000A012BF4
:1085200046D14FF00C0B9FEDA4BA9FEDA49A94F89E
:1085300012375FFA8AF5AB4240F286800BFB05F5F5
:108540003CABB0EE680A0AF1010A03EB0509A9F198
:108550004803089321AB581935F05AFE089B09EDE2
:10856000120AB0EE4B0AC3ED010A83ED021A33ABD7
:10857000581935F03DFE2AAB8DED100AB0EE490AD0
:108580005819CDED110A8DED121A35F031FE13A9EF
:1085900010A88DED130ACDED140A8DED151A35F0E6
:1085A00011FE09ED090A49ED080A09ED071ABEE7AF
:1085B000F0EE088A9FED809A9FED80BA94F812370A
:1085C0005FFA8AF94B4564D99DED0C0AB4EEE80ACE
:1085D000F1EE10FA35DB0C2303FB09F93CAB03EB9E
:1085E000090521AB03EB090035F012FE33AB05EDB5
:1085F000120AB0EE490A45ED110A03EB090005ED38
:10860000101A35F0F5FD2AAB8DED100AB0EE4B0ACD
:1086100003EB0900CDED110A8DED121A35F0E8FDDE
:1086200013A910A88DED130ACDED140A8DED151ABE
:1086300035F0C8FD05ED090A45ED080A05ED071AF4
:10864000049D0AF1010AB9E74FF000094FF00C0A46
:1086500094F812375FFA89F5AB4241D933AB09F18F
:1086600001090AFB053036F0E1F91BEE900AF0EE45
:10867000408AABF09BFB07EE900A3CABB8EE677A02
:1086800003EB8505C8EE877A67EEAA7A45ED2F7A67
:10869000DEE74FF0000A4FF00C0B94F812375FFA48
:1086A0008AF94B451DD933AB0AF1010A0BFB09309E
:1086B00036F0BCF9C8EE297A1BEE900A67EE808A84
:1086C000ABF074FB07EE900A3CABB8EE677A03EBB5
:1086D0008909C8EE877A67EEAA7A49ED2F7ADCE736
:1086E000049DBFF0B7FF069BC01AB0F5FA7F27D9EB
:1086F000BFF0B0FF04F5A0430C9AB121D3F8843346
:10870000DDED0D7A1B891392FCEEE77A339AADF812
:108710005C30149217EE903A349AADF85E30142320
:108720001592359A06901692F022307CCDE90032EF
:1087300013AA6CF0A3F99AF0D9FC317C9AF0A4FB4F
:108740000BA82CF02DFAB5E600254FF00C0A039982
:1087500038461AF003FFE9B294F812378B4207D972
:1087600033AB384601350AFB01321AF075FDF2E7EA
:1087700038461AF083FD124A062130466EF0E6FDB7
:10878000104B002520465D7201F078FB04F55A502D
:1087900032305EF013F999F8C9370AA865F3C303BC
:1087A00089F8C9372CF0FCF940463DB0BDEC0A8B86
:1087B000BDE8F08F31D61808A4707D3F0AD7233C5E
:1087C000B1AF16080DB90030F0B5534F85B004466F
:1087D000D7F81033DA0700F19C8000F5A045D5F8F2
:1087E000F83793F8C120002A40F0938093F8CB30FB
:1087F000002B00F08B8095F9C837002BC0F28680E3
:1088000000F5E04696F89037002B40F08280D6F8CD
:1088100024039FED420A6C3035F0EAFCCDED020AEC
:1088200060EEA00ADFED3E7A8DED010A8DED031AB0
:10883000E0EE000AF4EEE70AF1EE10FA66DCD6F894
:1088400024339FED387AD3ED377AF4EEC77AF1EE20
:1088500010FA04D5D5F8F8371B7A002B56D0B5EEB0
:10886000007AF4EEC77AF1EE10FA4FD404F5E64040
:108870000830B5F0FDFDDFED2C7AB4EEE70AF1EE3D
:1088800010FA43D8D6F824339FED287AD3ED367A00
:1088900067EE877AB3EE0E7AF4EEC77AF1EE10FA4D
:1088A00034DA234AB4F9A410138801339BB213803D
:1088B00019B9B4F8A210A4F8A410B4F8A4109942FD
:1088C00027D80026168068F075FC0122192168F06F
:1088D000CDFBD5F8F80703685B699847431C04F59E
:1088E000AA40144A314660306BF032F8D5F8F837B8
:1088F000012283F8C120D7F810335B0709D504F5AE
:10890000985005B0BDE8F04089F03ABC084B002211
:108910001A8005B0F0BD00BFB08200309F0CB34597
:108920004054094A6666663F000000B4E02E654286
:108930005EB70030C8AF1608494B70B52DED028BFD
:10894000D3F8103384B004469B071FD400F5E045EC
:10895000DFED448AD5F8240303681B699847D0EDFE
:10896000017AF4EEE87AF1EE10FA0FDB04F5A04399
:1089700004F5EF46D3F8F827143692F8C11049B140
:10898000002303A9304603936AF04CF904B0BDEC10
:10899000028B70BD92F8CB20002AF1D093F9C83732
:1089A000002BEDDB95F89037002BE9D1D5F82403A7
:1089B00003681B699847D0F8B030D5F824030393B7
:1089C00003681B69984704F58C7200F1B0013046CA
:1089D0006AF04AFADDED037AB0EEC08AF0EEE77A8B
:1089E000F4EEC87AF1EE10FA03D503A930466AF026
:1089F00019F9D5F8240303681B699847D0ED040AD8
:108A0000F4EEE80AF1EE10FAC0DBF6EE087A60EE5A
:108A1000A77AF4EEC87AF1EE10FA1AD5BFF01AFE72
:108A2000D5F8A03742F21072C31A9342AED99FED27
:108A30000E0A0021C5F8A00704F5AA4028EE000A96
:108A40000A4A6030B7EEC00A8DED000B6AF080FF75
:108A50009CE79DED030A2FF087FE0028DED195E705
:108A6000B0820030000000340000C842E4AF1608B5
:108A700010B5044600F5E940343080F09DFA04F565
:108A8000E94001215430BDE8104090F0C7B8000023
:108A9000F8B500F5E045044695F9B4344BB300F55C
:108AA000A04695F8C82400F5E94700F5E64096F899
:108AB000C83708303437DB43C3F3C01363F3C30252
:108AC00085F8C824B5F0D4FCDFED3D7A384620EEB9
:108AD000670A80F0F1FA95F8903753B9384680F07C
:108AE00097FAD6F8F83793F8CB301BB9354B0022FC
:108AF0001A80F8BD95F8C834DB07FAD4D6F8D40745
:108B000003689B6B98470028F0D096F9C837002B74
:108B1000ECDB2C4E33884BB9B5F9BA3433B164224F
:108B200013FB02F3D5F8FC229A42E2DB384680F0D0
:108B3000DFFAD5F824339FED247AD3ED367A67EE49
:108B4000877AB3EE0E7AF4EEC77AF1EE10FA05D812
:108B50003388002BCDD0013B3380CAE7B4F9A43071
:108B60001BB9B4F8A230A4F8A4303388B4F8A42018
:108B7000B4F9A40093421549D5F8D4223CBF01337F
:108B800033803388012B01D10A60B2E70968914232
:108B9000ACDD18B9B4F8A220A4F8A420B4F8A4203D
:108BA0009A42A6D80023338068F004FB02220C21ED
:108BB00068F05CFA2046BDE8F840FFF759BF00BFF7
:108BC0000AD7233C5CB70030E02E654258B700302E
:108BD00000F5E04208B592F9B4346BB300F5A04358
:108BE00093F9C837002B0EDA00F5AA40134A062184
:108BF00060306AF0ADFE68F0DDFA03220F21BDE8B7
:108C0000084068F033BAB2F9BA348BB16421D2F8B3
:108C1000FC2213FB01F39A420ADA00F5AA40084A43
:108C2000012160306AF094FE68F0C4FA0222E5E7A0
:108C3000BDE80840FFF71CBF08BD00BFFCAF160829
:108C40000EB01608F0B500F5A0450446574E2DEDC0
:108C5000028BD5F8F8378DB093F8CB3043B195F946
:108C6000C837002B04DB00F5405393F9CE362BB9FF
:108C7000002333800DB0BDEC028BF0BD00F5E04762
:108C800097F89037002BF3D101F06CFB002874D1DA
:108C9000D5F8D40703689B6B98470028E8D004F503
:108CA000E54058306AF014F835F0C0FEF0EE087A6E
:108CB000F0EE408AB4EEE70AF1EE10FAD8DA04F5E5
:108CC000DC539FED3B8AD3ED997A93ED980A20EE21
:108CD000270AF4F057FDF2EE0E7A20EE080AB4EE01
:108CE000E70AF1EE10FAC3D9D7F82433F3EE0E7A7F
:108CF00093ED367A27EE088AB4EEE78AF1EE10FAA1
:108D0000B6D904F5DC50002309A9183009930A9359
:108D10000B9312F047FD002837D13388B4F9A42013
:108D200001339BB23380002A3AD0B4F8A420B3EBCD
:108D3000420F9FDB68F03EFA01220C2168F096F9A1
:108D400000221C4BB7EEE80AB7EEC88A04F5AA4029
:108D500000216030CDE90623174B00228DED040B76
:108D6000CDE902238DED008B144A6AF0F1FD01225A
:108D70000C211348F9F7F4FC7CE7D5F8D407036815
:108D8000DB6C9847002883D172E709A835F04EFEC6
:108D9000F2EE047AB4EEE70AF1EE10FABDDB67E713
:108DA000B4F8A220A4F8A420BFE700BF54B7003055
:108DB000E02E65420000084000003E4024B0160846
:108DC00050870030F0B500238BB0044600F5DC502E
:108DD000079302AA089304F5A046099305AB03A9DB
:108DE0001830019307AB009304AB12F0C1FB0546AA
:108DF00086F8540518B9002528460BB0F0BDBFF021
:108E00001DFCD6F858359FED337A0746C31A04F592
:108E1000AA4006AA02A907EE903A3030F8EE677A27
:108E200067EE877ACDED067A6AF01EF804F5AA405F
:108E300006AA03A98DED020A3C306AF015F804F584
:108E4000AA4004F55B5406AA04A948308DED030A34
:108E50006AF00AF8C6F85875D4ED047AF5EEC07ACF
:108E6000F1EE10FAC7D9DDED086A9DED077AD6F864
:108E7000D82487FE267ADDED096A87FE267AF4EE8D
:108E8000C77A9DED037AF1EE10FA94BF0123002317
:108E90001AB196F8DC24D20712D477EEA76AF4EE62
:108EA000C76AF1EE10FA0BD80233DBB29DED027AFD
:108EB000F4EEC77AF1EE10FA09D8002B9BD09BE7AD
:108EC000F4EEC77AF1EE10FAF0D80133EDE7012B9A
:108ED00092D890E7BD37863570B500F5A0450446B9
:108EE00095F8ED3743F0040385F8ED3768F062F943
:108EF0000122112168F0BAF8D5F8F83793F8CB3091
:108F0000002B43D0D5F8D40703681B68984709287D
:108F10000AD1204609F03AFA30B104F5FD40BDE827
:108F200070403C3009F01ABA194BD3F8D4070368E3
:108F30001B69984704F5405340B993F9CD36032B8C
:108F400024D10621204609F00DFA0DE093F9CD1643
:108F50000229F6D195F8ED37DB07F2D40622204638
:108F600002F0BCF80028ECD00122D5F8D407094B58
:108F70005A7303681B6C9847034604F5AA40064AD7
:108F800002216030BDE870406AF0E2BC70BD00BFF5
:108F9000B08200300DB9003058B0160800F5A0427C
:108FA00008B592F8ED37590717D56FF3820382F8A9
:108FB000ED370A4B5A7B42B1002200F5AA4002214C
:108FC0005A736030064A6AF0C3FC68F0F3F8002276
:108FD0001121BDE8084068F049B808BD0DB900305E
:108FE0007CB01608F0B5054685B005F5DC57684637
:108FF00019F0D8F969461837384612F0C7FB80B126
:1090000005F55B53384CD3ED047AF5EEC07AF1EEFA
:1090100010FA08D80023354A28462380D373FFF777
:10902000BDFF05B0F0BD2846FFF7CCFE064628463A
:109030000EF0FAFD10B928460EF0D0FD002EA378F0
:1090400018BF00200343DBB2A370002BE9D0637884
:10905000A8BB83BB23780133DBB2082B237003D179
:109060004EB3384612F0F6FA2378092B02D138466F
:1090700012F0E8FA2378092B1DD94FF48573238069
:1090800068F098F80222102167F0F0FFBFF0E2FAD2
:109090006368C01A47F23053984209D905F5AA40CF
:1090A000134A022160306AF053FCBFF0D3FA6060CB
:1090B0002846FFF711FF62780C4BDA73B1E7267888
:1090C000002EF8D0013EF6B22670002BF3D0002E11
:1090D000F1D1667068F06EF83246102167F0C6FF75
:1090E0002846FFF75BFFE6E760B700300DB90030B8
:1090F00094B0160800F5A04393F8ED375B0701D54F
:10910000FFF7EABE7047000073B5044600F5DC5077
:1091100001A904F5A045183012F062F80646D5F80A
:109120001C3583420CD004F5E043D3F82403AEF0A1
:1091300095FCC5F81C6568F03DF83E2167F076FFA8
:1091400004F5805695F9201596F9A82E96F8A83EB4
:1091500091421BD0FF2B19D004F5E043D3F8240330
:10916000AEF07CFC96F8A83E85F8203568F022F831
:1091700095F82025182167F079FF04F5AA4095F9A4
:1091800020350421024A60306AF0E2FB02B070BD73
:10919000A4B016082DE9F0438FB00546BFF05AFA87
:1091A000002305F5DC580646059308AA069308F146
:1091B0001808079305A90893404609930A930B934F
:1091C0000C930D9304AB019303AB00930BAB12F024
:1091D000ADF9DFED477A9DED077A0746B4EEE77A01
:1091E000F1EE10FA30DB9DED0A7AB4EEE77AF1EE9B
:1091F00010FAACBF0124002405F5A049404699F8B7
:109200005435002B08BF002712F0A4F98046EFB9AF
:10921000444699F9A832012B29D164B1D9F8F8371D
:1092200093F8CB403CB1D9F8D40703685B69984701
:1092300080F00100C4B299F82435CBBBCCB9C9F891
:1092400028650FB0BDE8F0830024D5E7002CDFD0FF
:1092500005F5AA403C3069F0E3FCF7EE007A90EDAA
:10926000007AB4EEE77AF1EE10FAD2DCD0E700240F
:10927000E1E7D9F82805301AB0F57A7FE1D9C9F8C5
:109280002C35012405F5E04389F82445D3F82C3327
:1092900083F8484467F08EFF22461D2167F0E6FE02
:1092A000144A05F5AA40022160306AF051FBC8E774
:1092B00014B1C9F82C65C4E7D9F82C0543F69823F6
:1092C000361A9E42BDD905F5E043C9F8284589F80C
:1092D0002445D3F82C3383F84844C9F82C4567F06B
:1092E00069FF22461D2167F0C1FE034AD9E700BF8E
:1092F00000000034BCB01608D6B016080B4B012293
:1093000010B504465A72BFF0A5F904F5E042D2F850
:109310007C37C31A142B08D9C2F87C0704F5DA503D
:10932000BDE81040083058F091B810BD0DB90030BC
:109330002DE9F743044600F55B5000230DF10701CA
:1093400004F5A04608308DF807305EF0A5F8D6F891
:10935000F80790F9C030026883B3083B9569DBB227
:10936000012B2BD93221A84704F1100004F5AA489B
:1093700016F00CFA1F4B4FF0000908F160081F6847
:10938000F86A0368DB69984701281ED1BFF062F9CB
:1093900041F28733A0EB090205469A4205D9A94656
:1093A000154A062140466AF0D3FA2046FFF7A6FF89
:1093B000B86A032103685B689847E1E704F5405306
:1093C0009269B3F8DC169047CEE70121D6F8F8078A
:1093D000B5F0E2FFD6F8F8070368DB6A984775F046
:1093E00097FBF86A012103681B6803B0BDE8F043EE
:1093F000184700BF18B70030F4B0160870B504461F
:1094000000F5AA40184A06216030184E2DED028B57
:109410009FED178A6AF09CFA2046FFF789FF2046E5
:10942000FFF76CFF20460EF025F933680321986A98
:1094300003685B68984775F0A7FF054675F02EFF37
:1094400004F5A043D3F88423D3F8F807B2F9082031
:1094500000EE102AB8EEC00A20EE080AB7F060FD50
:10946000284675F023FFDAE718B1160818B7003060
:109470006F12833A2DE9F047044600F5AA402B4AC3
:109480000621603004F5A046DFF8A89041F2873A43
:109490002DED028B6AF05CFA2046FFF749FF75F06C
:1094A00073FF054675F0FAFEB7EE000AD6F8F80726
:1094B000B7F036FD284675F0F9FEBFF0CBF8074649
:1094C000BFF0C8F8C01BD9F80080504517D99FEDF0
:1094D000188A284675F0E2FEB0EE480AD6F8F8077A
:1094E000B7F01EFD284675F0E1FE2046FFF706FFA7
:1094F000D8F82800032103685B689847E9E7284605
:1095000075F0CCFEB7EE000AD6F8F807B7F008FD04
:10951000284675F0CBFE2046FFF7F0FED8F828006D
:10952000032103685B689847CAE700BF48B1160883
:109530000000000018B700302DE9F34100F5A04607
:109540000446D6F8F83793F9C030032B2BD06525A5
:1095500000F5E048344F013D15F0FF050CD0D8F878
:1095600078374BB93B681421986A03685B68984761
:1095700020460EF07FF8EEE704F5A94001212030E7
:10958000F8F77AFE04F5405393F9C83670B953B131
:10959000092B08D08DF8070004F55B500DF1070189
:1095A00008305DF079FF02B0BDE8F081032B34D8BC
:1095B000DFE803F002252D30D6F88433B3F9082014
:1095C00040F2B5339A422ADD04F55B5001250DF1D6
:1095D000070108308DF807505DF05EFF04F5AA40E2
:1095E000124A022160306AF0B3F9114B5D720E4BE2
:1095F0001C68A06A052103685B689847F9E7D6F8FC
:109600008433B3F9082040F2B5339A4207DD20468F
:10961000FFF7F4FE2046FFF72DFF092BC3D00023F0
:109620008DF80730B8E700BF18B700306CB11608E6
:109630000DB9003000F5AA400B46024A0421603003
:109640006AF086B98CB1160810B5044667F0B2FD11
:109650000022052167F00AFD04F5AA40034A04210F
:109660006030BDE810406AF073B900BF98B11608C9
:109670000B4613B54AB100F5AA4000920421054AF1
:1096800060306AF065F902B010BD02B0BDE810406C
:10969000FFF7D0BFB0B1160800F5AA40064A042172
:1096A000603008B56AF054F967F084FD00220821A3
:1096B000BDE8084067F0DABCC4B1160838B5044606
:1096C0000D46BEF0C7FF04F5A0433DB9D3F8E4272B
:1096D000C3F8E8070AB9C3F8E40738BDD3F8E827A8
:1096E000801A642882BF0022C3F8E827C3F8E42761
:1096F000F3E7000037B5044600F5E6400830B4F063
:109700009DFE04F5A042C0F3803592F8CA37C3F33A
:109710004001A9421DD065F3410304F5AA4482F833
:10972000CA3760346DB167F045FD02220B2167F046
:109730009DFC094A0221204603B0BDE830406AF092
:1097400007B967F037FD2A460B2167F08FFC034A03
:10975000F0E703B030BD00BFDCB11608F8B1160861
:1097600038B50A460C460621054601F0B7FC28B17B
:10977000054A137843F00803137038BD2146284684
:10978000BDE8384008F0EEBD2CB9003038B50A46C7
:109790000D461521044601F0A1FC28B1094A1378B1
:1097A00043F00803137038BD04F5AA400421064AAB
:1097B00060306AF0CDF829462046BDE8384008F010
:1097C000D1BD00BF2CB9003008B2160838B50A4622
:1097D0000D461521044601F081FC28B1094A137891
:1097E00043F00803137038BD04F5AA400421064A6B
:1097F00060306AF0ADF829462046BDE83840FFF7F2
:10980000AFBF00BF2CB9003030B2160838B50A46D9
:109810000D461B21044601F061FC28B1094A13786A
:1098200043F00803137038BD04F5AA400421064A2A
:1098300060306AF08DF829462046BDE83840FFF7D1
:109840008FBF00BF2CB9003046B2160838B50A46A3
:109850000D461121044601F041FC28B1094A137854
:1098600043F00803137038BD04F5AA400421064AEA
:1098700060306AF06DF829462046BDE8384008F0AF
:1098800071BD00BF2CB9003058B2160810B500F5F4
:10989000A04494F8CA379A0623D4D4F8D4070368AE
:1098A0001B689847032808D005D802280ED194F8E1
:1098B000C807C00914E01B28F9D194F8C80700F0C4
:1098C000A000A0F180035842584109E0B4F8C8074D
:1098D00020F4FE4020F07F0080B2003818BF012045
:1098E00010BD0120FCE7000038B500F5A045044696
:1098F00000F5AA40184A95F8ED370221603043F090
:10990000080385F8ED376AF023F867F053FC01226D
:10991000172167F0ABFB2046FFF7B8FF40B104F515
:10992000A940012215212030BDE83840F8F718BFC2
:10993000D5F8D40703681B689847062806D104F5B4
:10994000FF40BDE83840583009F0BCBF20460B212D
:10995000BDE83840FFF704BF6CB2160870B500F5DB
:10996000A0450646D5F8E427D5F8E8379B1A41F21A
:109970008832934211D9D5F8D40703681B6D9847F4
:10998000044695F8ED37C3F3C003A34213D034B1B6
:109990003046BDE87040FFF7A7BF0024F1E767F04D
:1099A00009FC2246172167F061FB95F8ED3764F357
:1099B000C30385F8ED3770BD0B46114610B504465C
:1099C000072B07D8DFE803F029041215181B2326FC
:1099D00008F0C8FC04F5A043D3F8AC329B061CD5B4
:1099E00004F59850BDE8104088F0CABBFFF7B8FEF8
:1099F000F0E7FFF7EBFEEDE7FFF7C8FEEAE700F55B
:109A0000A940012214212030F8F7AAFEE2E7FFF76F
:109A1000FDFEDFE7FFF71AFFDCE710BD70B5044677
:109A200067F0C8FB0122052167F020FB04F54053D5
:109A3000204693F8B236072B96BF2F4A0126D65CF4
:109A4000FFF724FF68B12D4A20462D49FFF710FE8D
:109A500004F5A940012210212030F8F781FE0026EC
:109A600014E004F5A045D5F8D4070368DB6C9847EB
:109A700098B195F8B93D83B195F9B83D012B0CDC4F
:109A8000204A214901262046FFF7F2FD31462046B3
:109A90000322BDE87040FFF78FBFD5F8D4070368F5
:109AA000DB6C984718B1D5F8AC32190715D4D5F846
:109AB000D40703681B689847032803D1D5F8AC3254
:109AC000DA070DD4D5F8D40703685B6A984768B9FC
:109AD0000B492046FFF7AEFDD8E70A4A0849D1E70F
:109AE0000A4A07492046FFF7C3FDB8E7D5F8AC326C
:109AF0005B07EDD5064AF4E738B316088CB21608B2
:109B000055C9170896B21608A9B21608B9B21608B0
:109B1000C9B2160870B50446154667F04BFB012222
:109B2000062167F0A3FA2046FFF7B0FE98B104F5CE
:109B3000A9400122072100252030F8F711FE134A21
:109B400013492046FFF794FD294620460422BDE82C
:109B50007040FFF731BF04F5A046EDB2D6F8D40748
:109B60000368DB6C984758B1D6F8AC321B0707D5B1
:109B700035B1084A204606490125FFF779FDE3E79C
:109B800003492046FFF756FDDEE700BF8CB21608FA
:109B9000E6B2160896B21608F8B5044667F00AFB56
:109BA0000122082167F062FA04F5A04573F002FB78
:109BB00004F5405393F8A136072B96BF354A022689
:109BC000D65CD5F8F83793F8CB705FB932492046A8
:109BD000FFF730FD0026314620460522BDE8F8405B
:109BE000FFF7EABE2046FFF751FE60B104F5A94039
:109BF000012212212030F8F7B3FD284A26492046D9
:109C0000FFF736FDE6E7D5F8D4070368DB6C984725
:109C100068B195F8B93D53B195F9B83D012B06DC13
:109C20001F4A204920460126FFF722FDD3E7D5F839
:109C3000D4070368DB6C984718B1D5F8AC32190724
:109C400013D4D5F8D40703681B689847032803D1B9
:109C5000D5F8AC329A070BD4D5F8AC32DB0609D470
:109C60000D492046FFF7E6FCB5E70D4A0A49D9E75A
:109C70000D4AC3E7D5F8D4070368DB699847054662
:109C80000028EDD1094A204603492E46FFF7F0FC93
:109C9000A1E700BF40B316087E9D16088CB21608D7
:109CA00096B21608E0B21608EEB2160803B316080C
:109CB00000F5405370B593F9A1360446ABB300F5F7
:109CC000A045D5F8586786B3BEF0C4FC95EDC20A2E
:109CD000DFED167A861B9FED161A8D2020EE270ADF
:109CE000DFED140A2EF0A2FEBCEEC00A10EE103A10
:109CF0009E420CD295F8ED379A0716D520460021E2
:109D0000F8F786FE2046BDE87040FFF7C5BC0CD9C9
:109D100095F8ED379B0708D420460121F8F778FE27
:109D20002046BDE87040FFF737BF70BD00007A44A1
:109D30000000804F000000002DE9F341074600F5C8
:109D4000E64007F5A0440830B4F078FBC0F3804843
:109D50000190BEF07FFC94F8F03745460646434537
:109D60000DD007F5AA4084F8F0876030002D3FD071
:109D70003A4B3B4AC4F8F467022169F0E9FD94F8D4
:109D8000F03743B394F8F1372BBBB4F91E3340F2EC
:109D900057109FED340A07EE903A9FED331ADFED2E
:109DA000330AF8EEE77A27EE800A2EF03FFEBCEE8B
:109DB000C00AD4F8F40710EE103A361A9E420AD9B7
:109DC000012307F5AA402A4A022184F8F1376030BE
:109DD000224B69F0BDFD94F91D33002B94F8ED374B
:109DE0000DDC6FF3451384F8ED3702B0BDE8F08168
:109DF0001A4B204AC4F8F48784F8F187BCE7C3F310
:109E00004012AA42F1D065F3451384F8ED379B0662
:109E1000EBD5194BD3F8D40703681B699847002882
:109E2000E3D067F0C7F901221F2167F01FF9384618
:109E3000FFF72CFD48B107F5A94001222121203070
:109E400002B0BDE8F041F8F78BBC322294F81D1344
:109E5000384602B0BDE8F041FFF7AEBD1CB31608AE
:109E60005CC1170800007A440000804F0000000029
:109E70002BB3160837C11708B082003008B501228D
:109E8000034B1A70BEF0DAFB024B186008BD00BF2E
:109E900069B700306CB70030014B00221A70704770
:109EA00069B700302DE9F0410446BEF0C7FB2A4BEC
:109EB0000546B4F8BE201988284E91420ED01A806B
:109EC000274B18603378A3B10024347067F072F91F
:109ED00022461321BDE8F04167F0C8B83378214F1E
:109EE000DBB93B782BB11E4B1F4A1B68C31A934248
:109EF00001D8BDE8F0810123337004F5A043D3F805
:109F0000F80790F8CB3013B103689B6A984767F065
:109F100051F90122132167F0A9F83B78002BE8D012
:109F20003378002BE5D00E4A10491368EB1A8B42A8
:109F3000DFD904F5A0441560D4F8F80790F8CB30C9
:109F4000002BD6D00021B5F027FAD4F8F807036823
:109F5000BDE8F0415B6A18476AB7003068B7003067
:109F60006CB7003069B7003080841E0040420F009B
:109F70002DE9F84300F5A04500F540580446D5F812
:109F8000D40798F8B0730368DB6C9847014650B962
:109F900095F9C837002BA9BFD5F8F837012193F8F8
:109FA000CB0080F0010104F54D5909F13409484610
:109FB00089F02EFAD5F8F837064693F8CB30002B07
:109FC0007BD0002865D03E4B93F9C837002B04DBCB
:109FD00002463C49484688F0F3FD98F97A7357B138
:109FE00095F9C837002B0EDA04F5A94001220F219C
:109FF0002030F8F7B5FB67F0DDF832460921BDE8FF
:10A00000F84367F033B8D5F8D40703685B6998471D
:10A0100058B195F9C937002B07DA95F8ED37DA070B
:10A0200003D498F8B033DB07DED53146484689F0D3
:10A0300055FADFED257AB4EEE70AF1EE10FA05DD08
:10A040000A220921204601F049F8D4E7023F032FF4
:10A0500011D801A353F827F041A0060869A006080B
:10A0600087A006088DA006080A221521204601F0C7
:10A0700035F80028BFD10A220621204601F02EF82B
:10A080000028B8D1DCE70A221121F6E70A221521BF
:10A09000F3E797B198F8B0337BB9094B93F9C83718
:10A0A000002B06DB04F5AA40084A0521603069F060
:10A0B0004FFC67F07FF80022A0E7BDE8F88300BFFF
:10A0C000B082003048B316080000C84251B31608E9
:10A0D00070B500F5E64500F5A04386B004460835A6
:10A0E00093F824152846B4F057F902A818F05AF945
:10A0F00004F5DC5002A9183011F0D6FA04F5E0435B
:10A10000049A2846C3F80023059AC3F80423B4F040
:10A1100095F982061AD5284604F5E545B4F09CF970
:10A12000FDEEC07A783504F58054022217EE901ABD
:10A13000284617EE906A18F03BF994F8143EDB07B6
:10A1400006D401223146284618F032F906B070BD17
:10A150000121284618F0BEF90028F2D0F6E70000E9
:10A1600070B500F5E04486B00D461646B4F8AC373D
:10A170008B4203D1D4F8A837934221D0BEF06AFABB
:10A18000D4F8A437C31A132B1AD9C4F8A867A4F8B3
:10A19000AC57C4F8A40767F00DF80446BEF062FAA5
:10A1A000084B094A1B68CDE90453084B0193084B3F
:10A1B000CDE9020100932046064B074966F086FD73
:10A1C00006B070BD70B7003068B3160880B31608CB
:10A1D0000A861608C16516087BB3160838B500F55F
:10A1E000A0440D4694F8C937C3F380138B420BD0BB
:10A1F00021B166F0DFFF112166F018FF94F8C9372E
:10A2000065F3861384F8C93738BD0000F0B500F552
:10A21000A045064600F5E0442DED048BD5F8F8374F
:10A220008BB093F8CB30002B67D095F9C837002B53
:10A2300063DBD5F8D40703685B699847002861D1D0
:10A24000D4F8240301AF9FED430A6C3033F0D0FF04
:10A250000AAACDED080A04AB8DED091A8DED070AA7
:10A2600012E9070083E8070087E80700384633F063
:10A27000B9FB06F5E540D4F82433B0EE409A5830E7
:10A28000D3ED368A68F024FD34F0D0FBD4F82C33BB
:10A29000D5F8D407B0EE408AD3EDE49A0368DB6CBE
:10A2A0009847DFED2D7AB4EEE79AF1EE10FA02DC72
:10A2B00095F8D0370BB1002838D0DFED287A68EE5A
:10A2C000A78AF3EE0E7AF4EEE78AF1EE10FA2DDCAF
:10A2D000F0EE087AB4EEE78AF1EE10FA26DCF5EE3D
:10A2E000C09AF1EE10FA21DAD4F8240303689B6FC8
:10A2F00098470BB0BDEC048BF0BDD4F82403036881
:10A300009B6F0DE0D5F88423D4F82403B2F908201C
:10A310000368002A03DCD5F8CC27022AF0D1DB6FD2
:10A320000BB0BDEC048BBDE8F0401847D4F82453C3
:10A33000B7EE001A40F2AB10DFED090A2B68D3F834
:10A340008060D4F82C3393EDCC0A2EF06FFB2846B6
:10A35000B047CEE79F0CB3450080BB44E02E65427A
:10A360000000000000F5A04090F8D0077047000002
:10A370002DE9F04100F5A04506460C4695F8C83792
:10A38000B1EBD31F48D0254B00221A6000293FD0E3
:10A3900066F010FF122166F049FE95F8C83784F088
:10A3A000010806F5405764F3C71385F8C83798F0DD
:10A3B000DDFF414698F0B6FFB8F1000F06D097F8E0
:10A3C0008A341BB9BEF046F9C7F88C0487F88A8432
:10A3D00014B3B7F884365B071ED5D5F8F83793F871
:10A3E000CB30CBB1D5F8D40703685B69984798B9EF
:10A3F000D5F8D407202103689B69984760B106F51A
:10A40000A94001220D212030BDE8F041F8F7A8B99C
:10A4100066F0D0FE1C21BEE7BDE8F08170B70030C9
:10A420002DE9F04F00F5A045044600F5E0472DED7D
:10A430000A8BD5F8F8378DB093F8CB601EB901219F
:10A44000FFF796FF0BE095F9C827002A65DAD5F8E3
:10A45000D40703689B6C98470646002841D04FF00C
:10A46000000B95F9C827B24E002AC0F25481D6EDF0
:10A47000007AB4F9A420B8EE677A1AB9B4F8A22029
:10A48000A4F8A420B4F8A430DFEDAA6A07EE903A4D
:10A49000F8EEE77A67EEA67AB4EEE77AF1EE10FA14
:10A4A000ACBF012100212046FFF798FE95F9C8278F
:10A4B000002A95F8C927B8BF4BF0010B530697F84F
:10A4C000902748BF4BF0020B0AB14BF0080B3268E3
:10A4D000594620460DB0BDEC0A8BBDE8F04FFFF7A2
:10A4E0003FBED5F8F837204693ED0C8AF8F76CFBA1
:10A4F000B4EEC80AF1EE10FAB1D5D5F8F83793F8F2
:10A50000A130032BABD165F037F84FF48011422214
:10A5100064F0EAFF3146204692E797F890A7BAF137
:10A52000000F03D00023824A136098E7D7F8240372
:10A5300093F8079003685B6F984780460090D5F8C2
:10A54000D40703685B69984720B1D5F8CC37022B54
:10A5500000F0E380B9F1000FB7EE00BA0CBF4FF086
:10A56000000B4FF4007BB8F1000F02D04BF4806B6E
:10A57000009604F5E9489FED70CAF3EE0EBADFEDE0
:10A580006F8A08F1540840468EF068FB0130D7F816
:10A5900024030CBF012302239FED690A6C3008EEEF
:10A5A000103A33F025FE0CAB0DF10C0E0DF1180C2A
:10A5B000CDED0A0A8DED0B1A8DED090A13E907009E
:10A5C0008CE807008EE80700704633F00BFAD7F8E6
:10A5D0002423DFED5C7AB4EECC0A92ED36AA04F5C2
:10A5E000E540F0EE40AA2AEE27AA5830F1EE10FA24
:10A5F000B4EEEBAAC8BF4BF4807BF1EE10FAC8BFF3
:10A600004BF4807B68F064FB34F010FAB8EEC88A33
:10A6100004F5E640F0EE409AB4EEC80A0830F1EED8
:10A6200010FA98BF4BF0800BB3F022FF68EE288A37
:10A630002046B0EEC09AB4EEE89AF1EE10FA48BFA8
:10A640004BF0400B0DF022F9002846D14BF0200BC7
:10A65000019640468EF002FB01284FD14BF0100BC3
:10A66000B2463349B9F1000F53D0009B002B50D0B4
:10A67000F4EECCAAF1EE10FA4BDCB4EEEBAAF1EE5C
:10A6800010FA46DCF4EEC89AF1EE10FA41D8B4EEB6
:10A69000E89AF1EE10FA3CD5019BD3B3BAF1000F62
:10A6A00037D00A68B4F9A40007EE902AB8EE677AAA
:10A6B00018B9B4F8A200A4F8A400B4F8A43007EEC6
:10A6C000903AF8EEE77A67EE8B7AB4EEE77AF1EE3D
:10A6D00010FA19D501320A60C3E604F5A74020300C
:10A6E00068F09EFADFED187A90ED007AB4EEE77A22
:10A6F000F1EE10FAAAD400230193AAE740468EF0A7
:10A70000ADFA0130ADD1A9E701212046FFF730FEB7
:10A71000A7E60022DFE70121C5E6B9F1000FB0EEA0
:10A7200008BA0CBF4FF0000B4FF4007B1EE700BFD0
:10A7300070B70030CDCC4C3E0080BB440000C84216
:10A740009F0CB345E02E65420000484300F5F753E7
:10A750009FED217A30B5083389B0044602AD93E805
:10A76000070085E80700DDED047A04F5E54077EEA3
:10A77000877A9FED1A7A5830CDED047AD4ED2B7A92
:10A78000F0EEE77AF4EEC77AF1EE10FA0BD5B4F9F1
:10A79000A230F7EE006A07EE903AF8EEE77A86EE1E
:10A7A000A77A84ED2B7AD4F8AC3001AA294601931C
:10A7B00068F080FB2046FFF733FE2046FEF768F97D
:10A7C0002046FEF73FFA2046FDF7FEFF2046FEF743
:10A7D000B3F809B030BD00BF0AE81C4100000034E6
:10A7E00010B504461D202DED028B74F063FB60B3A1
:10A7F00004F5A043D3F8D40700F0D0FA192108EEED
:10A80000100A04F698705DF037FB02281AD003385E
:10A81000012808D804F5A740203068F001FA90ED2F
:10A82000008ABDEEC88AB8EEC88A9FED090A04F511
:10A83000E94028EE000A5430BDEC028BBDE8104020
:10A840008EF092BA9FED038AEDE7BDEC028B10BD4E
:10A850000AD7233C00000000114A0260114A02F1AD
:10A8600078014260816001F57151C160043101617C
:10A870000839416124398161A2F5D75102F50652A8
:10A88000C1614262A2F27C420749826204320162E3
:10A89000C2620432026304324263044A8263704734
:10A8A000F0CD160828690030D4A50030C833003038
:10A8B0001C2968D8DFE801F0130F171B27232F1F6F
:10A8C000672B67336767373B3E42464A4D515458C2
:10A8D0005B5F6767640000F5EF403430704700F558
:10A8E00000406430704700F5EF407430704700F569
:10A8F000F0403030704700F5FA406030704700F5A6
:10A90000FE400430704700F5FC407830704700F599
:10A91000FD403C30704700F5FF405830704700F56F
:10A92000FB402030704700F5FB405C30704700F57D
:10A93000F640FAE700F5FE404430704700F5FA4073
:10A940001C30704700F50140A030704700F5014011
:10A95000EBE700F50140F030704700F50240BCE73E
:10A9600000F5A040C06C704700F5FC40C1E700F561
:10A970000340A430704700F5A040D0F8A40270470F
:10A9800000F50440DCE700207047000073B50B6859
:10A99000054608460C461B6C16469847034605F5C7
:10A9A000AA400F4A04210096603068F0D1FF66F09B
:10A9B00001FC2368054620461B6898470A21024689
:10A9C000284666F053FB074B93F8C9379B0641BFF7
:10A9D000054A137843F00403137002B070BD00BF42
:10A9E00084B31608B08200302CB9003038B50C4A58
:10A9F000182305460C4664F0EFFA78B12146284644
:10AA0000FFF756FF30B10146064A2846FFF7BEFF62
:10AA1000002038BD284664F097F9F9E70120F8E7EF
:10AA200004B41608A4B3160810B5002300F5A0441A
:10AA300000F5E04084F83434074BD0F8240393F851
:10AA4000C817C909ABF08AFCD4F8D4070368BDE87D
:10AA50001040DB68184700BFB082003070B5054673
:10AA600008680C46164603685B69984790B13068E1
:10AA700003685B69984768B905F5A043D3F8F827E0
:10AA800092F8CB2032B193F9C837002B02DB28466D
:10AA9000F8F7B0F804480DF0F1FC20680368BDE851
:10AAA00070409B68184700BF68B8003070B500F56B
:10AAB000A04504460C4ED5F8D4070368DB699847D7
:10AAC0003074D5F8D40703681B689847F070D5F840
:10AAD000D40703685B6C9847014604F5DA50BDE87B
:10AAE0007040083056F0FCBC0DB90030254B70B5F5
:10AAF0002DED028B93F8ED37B0EE408AF0EE608AD0
:10AB000082B0DB0706460D46144606D500232B60AF
:10AB1000236002B0BDEC028B70BD72F04BFC037F72
:10AB2000002BF3D0F36A01A99FED171A68461B6842
:10AB30009FED160A68EE811AB3F9083028EE011A63
:10AB400007EE103AB36A1B68B8EEC77AB3F908305B
:10AB500067EE000A07EE903AF8EEE77A27EE800AF1
:10AB60002FF01CF8DFED0A6A9DED007ADDED017A29
:10AB700027EE267A67EEA67A85ED007AC4ED007A94
:10AB8000C7E700BFB08200300AD7233C53046939BD
:10AB90000000C84270B5002306462DED028B88B038
:10ABA000B0EE408A029306AD039302AC324B93F8A9
:10ABB000ED3713F0010F03D172F0FCFB037F5BB99B
:10ABC00094E8030085E803009DED060ADDED070A21
:10ABD00008B0BDEC028B70BDB36ADFED286A1B685C
:10ABE000B3F9083007EE903AF36A1B68F8EEE77A9B
:10ABF000B3F9083067EEA67A07EE103AB8EEC77AD6
:10AC0000CDED037A27EE267AF1EE476AB0EEC77AE9
:10AC1000CDED026ADFED1A6AB4EEE67AF1EE10FAD3
:10AC200006D5F0EEE77AF4EEE67AF1EE10FAC7D444
:10AC300003AA21461348F8F70DF8DDED027A9DEDE1
:10AC4000037A2046F0EEE77AB0EEC77AF4EE477A60
:10AC5000F1EE10FA37FE870A32F012FE04A88DEDED
:10AC6000040ACDED050A32F0BDFE204688EE000A4A
:10AC700032F036FEA4E700BFB082003053046939D9
:10AC800000000034B0320030094B93F9C827002A85
:10AC90000CDAB5EEC00AF1EE10FA07D9D3F8F8379E
:10ACA00093F8A100C31E58425841704700207047D6
:10ACB000B0820030436A1B6893F8CB3043B1054B38
:10ACC00093F8C80700F0A000203818BF0120704793
:10ACD00001207047B082003010B5436A04461868FE
:10ACE000D1B10221B4F068FB236A9FED0C1A1868F9
:10ACF000F0EE410A0368B0EE410ADB6A9847236A26
:10AD0000074A00211868D2ED000A03689FED030A84
:10AD10005B6EBDE8104018470121E3E7000000002A
:10AD20003069003010B5436A04461868002930D0F5
:10AD30000221B4F041FB236A1868ABF0DFFA636AC2
:10AD40001B6893F8A130012B04D8236A01211868ED
:10AD5000ACF08AF863691868AFF06CFA6369186838
:10AD6000AFF012FB63699FED0C0A1868AFF044FD69
:10AD700063691868AFF0BCFD236A9FED071A186875
:10AD8000F0EE410A0368B0EE410ADB6ABDE810400C
:10AD900018470121CDE700BF0000000013B50446AD
:10ADA00001A90C480CF0F4FD10B1019802B010BDDF
:10ADB00063691868AEF0E8F818B9074BD3F8FC02DD
:10ADC000F4E701AA0321054817F028FB0028F4D076
:10ADD000EBE700BFB0320030B0A20030A8A50030D1
:10ADE000F0B504462DED048B89B0002940F0FC80BD
:10ADF00083687F4E03F58053B3F95A59642DB8BF69
:10AE00006425FFF7CBFF6268A8422046B2F93430D0
:10AE1000AABF96F8C9570125C5F38015002BD5BFE9
:10AE200063695B421B6807EE903AD4BF93EDC78A13
:10AE3000B8EEE78AB2F93230002BB8BF5B429BB262
:10AE40005B4207EE903AA368F8EEE77A03F5805389
:10AE5000B3F95A79F4EEC87AF1EE10FA38FE278A7F
:10AE6000642FB8BF6427FFF799FF6369391AA26B93
:10AE70001B6800EE101AD2ED001A93EDC91AD3ED3B
:10AE80000E0AB8EEC00A2EF073FA6368F0EE480AB4
:10AE900040F29720B3F93230002BB8BF5B429BB22F
:10AEA0005B4201EE103AB8EEC11A2DF0BFFD6369A6
:10AEB000B0EE408A1868AEF067F896F8CA370746D1
:10AEC0001A077ED44B48B0F069FA002879D0002FD9
:10AED00077D09FED499A01A946488DED019A8DEDF5
:10AEE000029AB0F0E3FA00287BD0A069B3F0B2FA7E
:10AEF00003AB03C883E80300194601A832F0A4FCA1
:10AF000005A88DED050ACDED060A32F06BFDF0EED9
:10AF1000409A3A4E05A9DFED3A7AD6ED008AA6F1BD
:10AF200024008DED059AA6F5A36668EEA78A8DED3F
:10AF3000069A8DED079AB0F0E3FAF4EEE89AF1EE96
:10AF400010FA08DDF0EEE88ADFED2E7AF4EEE78AFB
:10AF5000F1EE10FA49D5DDED077A9FED2B7AF4EE8C
:10AF6000C77AF1EE10FA2CDD9FED287AF4EEC77A5D
:10AF7000F1EE10FA25D5B6F830355B0721D46368B9
:10AF8000F2EE0E7AB3F93230002BB8BF5B429BB2BF
:10AF900008EE103ABAEEEF8A88EE277A67EE297A41
:10AFA000F5EEC07AF1EE10FA48BFDFED137A37EE16
:10AFB000C88AFAEE047AB4EE678AF1EE10FA37FE28
:10AFC000888A6369B0EE480A29461868AEF07CF8B2
:10AFD0006369186809B0BDEC048BBDE8F040AFF0C0
:10AFE00087BCF0EE499A94E700259FED038AE8E7D5
:10AFF000B0820030A4A7003000000000C8A70030D5
:10B000000000C8420000003400000C420000484329
:10B01000436A186803681B691847000038B52DEDAE
:10B02000028B03680446D3F884309847236B2A4880
:10B03000F0EE408A1B68B3F908500CF0A3FB041E25
:10B040004FF47A724FF000012846D8BF4FF4FA74DB
:10B050002DF054FDB6EE000A84422ADD07EE900A78
:10B06000B8EEE77A07EE904AF8EEE77A27EE007A34
:10B0700087EE278A4FF46D7038EEC00AF5EE087A35
:10B08000B7EE001AB1EE400AFEEE000A80EE270A83
:10B090002DF0CCFCF7EE007A77EEC07A28EE000AAD
:10B0A00020EE080A20EE080AA7EE880ABDEC028B03
:10B0B00038BD031BC4F57A7407EE103A07EE904AC8
:10B0C000B8EEC77AF8EEE77A27EE007A87EE278A9D
:10B0D00038EE008ACEE700BFB03200302DE9F04FE5
:10B0E00000F5E04900F5A04605460F4690462DEDD7
:10B0F000028B99F8B04783B089F8B027D6F8D40707
:10B1000003681B689847B84221D105F54055B8F14E
:10B110001A0F85F8888406D128B9D9F82433D6F8CF
:10B12000E422C3F8FC208F4B93F8C9379D0606D460
:10B130000124204603B0BDEC028BBDE8F08F4445EE
:10B14000F6D0894A137843F002031370F0E7B8F1A0
:10B15000020F0CD01B2F12D105F5F04041463030C4
:10B1600003B0BDEC028BBDE8F04F01F00FBB3946D8
:10B170002846FFF73BFC04460028EBD1D9E73946C7
:10B180002846FFF795FB0446019018B9284663F05E
:10B19000DBFDCEE7D6F8F83793F8CBB003688BF039
:10B1A000010A5B69984705F5FB43019A20339A42EF
:10B1B00008BF0120BBF1000F08D101985146036878
:10B1C0005B689847044648BB684A22E096F9C8374E
:10B1D000002B80F2B980002800F0B680DFF884B13F
:10B1E000DBF8D40703685B6998470446002840F001
:10B1F000AB800198FFF712FFB0EE408AABF5A0409C
:10B20000F7F7E2FCB4EEC08AF1EE10FA40F39C804E
:10B21000574A01992846FFF7B9FB8AE705F5AF4180
:10B2200001AA284605F5405A5431FFF717FC01984A
:10B23000C6F8D4078AF8888403681B6898470146D3
:10B2400005F592504246083065F0C8FA05F5AA4067
:10B250000021603071F06CF9FB1E012B02D9B91F7F
:10B260004C424C4189F8AE469AF97A3323B105F540
:10B270004D50343088F056F9D6F8D40703681B686F
:10B280009847C21ED9F8243350425041012F89F803
:10B29000B403D6F8B422C3F8F820D9F82433D6F88A
:10B2A000E422C3F8FC2001D00B2F05D1D9F82433B8
:10B2B000D6F8CC22C3F8FC202846FFF7F7FB294B31
:10B2C00093F8C9379B063FF53CAF31E705F540538E
:10B2D00093F87423002A3FF470AFB3F89023D0079B
:10B2E0007FF56BAF93F8B023002A3FF466AFD6F832
:10B2F000F82792F8CB20002A3FF45FAF93F8883408
:10B300000A2B7FF45AAF96F9C837002BFFF655AFDA
:10B31000184A284601990024FFF738FB09E7164828
:10B320000CF0CCFC0028D1D1D6F8D40703685B69B7
:10B3300098470028CAD0019803685B69984704467B
:10B340000028C3D10D4A64E7019803681B69984738
:10B350000028E4D008480CF09FFC04460028DED109
:10B36000074A56E7B08200302CB9003026CF1808C3
:10B37000CCB31608F0B31608B0320030DEB31608AE
:10B38000EA4D18080148FFF7A9BE00BFB0320030EF
:10B3900013B504468DED010A8BF07CFC01A96369AD
:10B3A000A26B1B6892ED001A93ED0E0AD3EDC90A49
:10B3B0008AF07CFA9DED010A02B010BD436A18685C
:10B3C00003685B6A1847000038B5436A05461C6885
:10B3D00094F8CB1061B92046B3F0EEFF6B6A1B689E
:10B3E00093F8A10018B1012814BF0320022038BD32
:10B3F000164803783BBBFFF747FC20BB144A92F882
:10B40000C83703F0A003202B17D0B5EEC00AF1EE29
:10B4100010FA10D592F8CA375B070CD401212046E8
:10B42000B3F0CAFF6B6A1B6893F8A130012B0CBF05
:10B4300002200320DBE70221F1E720460221B3F0DE
:10B44000BBFF0420D3E70120D1E700BF68B800307C
:10B45000B0820030154B10B52DED028B93F8ED370F
:10B460000446DB0704D59FED120ABDEC028B10BD2C
:10B4700071F0A0FF037F002BF5D0636B186872F0AA
:10B48000C1F8A368DFED0B7A03F5805303F6F832B9
:10B4900003F6FC3392ED008AD3ED000A28EE278AEA
:10B4A0002EF036FB28EE000ADFE700BFB082003046
:10B4B000000000000000C8420148F7F7F7BB00BFDA
:10B4C000B03200300148F8F7B1B800BFB0320030F8
:10B4D0000148FFF703BE00BFB0320030F0B55F4E49
:10B4E00004460D4696F8ED372DED028B13F0010F53
:10B4F0008FB005AF5FD143689B899A071CD5584828
:10B5000067F08EFBDFED577A90ED007AB4EEE77AC4
:10B51000F1EE10FA10DD65F04DFE3D2165F086FD7F
:10B5200009220521A6F5A040FFF7D8FD20B9092280
:10B5300002212046FFF7CCFF636893F95430002BBB
:10B5400039D000230593089323691868B2F0E6FC0C
:10B55000236AB0EE408A186803689B6E984708AA71
:10B56000F0EE400A3946B0EE480A2046FFF7BEFA30
:10B57000DDED057A9FED3C7AF0EEE77AF4EEC77ADE
:10B58000F1EE10FA08D5DDED087AF0EEE77AF4EE88
:10B59000C77AF1EE10FA0ED496F8CA371B0704D416
:10B5A00065F008FE492165F041FD96F8CA3743F081
:10B5B000080386F8CA3795ED027A08A895ED005A77
:10B5C000B1EE477A95ED016AB7EEC55AB7EEC66A95
:10B5D000B7EEC77A9FED1F0B8DED085B8DED0A6B03
:10B5E0008DED0C7B33F064FD636908A98DED0A1BBA
:10B5F0008DED0C2B8DED080BDFED1C0A9FED1C0A69
:10B600001868AEF087FC63691868AEF0BDFE636928
:10B610001868AFF06DF9236A1D6863691868ADF0AA
:10B62000FDFE384613498DED020ACDED030A8DED7E
:10B63000041AFCF7A3F8079B02A92846009397E891
:10B640000C00AAF00BFF0FB0BDEC028BF0BD00BFE9
:10B65000AFF300800000000000005940B0820030CD
:10B660009CA5003000002F440000003400007A4404
:10B670000000000024B700302DE9F041AA4D00265B
:10B68000044695F8C9372DED028B5A0692B00596FF
:10B69000069603D543691868ADF0D6FA95F8ED37EC
:10B6A000DB0755D463689B899F071BD59F4867F0CC
:10B6B000B7FADFED9F7A90ED007AB4EEE77AF1EE1B
:10B6C00010FA0FDD65F076FD3D2165F0AFFC092233
:10B6D00005219848FFF702FD20B9092202212046E2
:10B6E000FFF7F6FE636893F954308BB39148F7F790
:10B6F0009DFFE3689FED908AB6EE000A1B68204626
:10B700009FED8E7AD3ED0A7AF4EEC87AF1EE10FA54
:10B7100067FE877A27EE800AFFF73CFACDED060A2E
:10B720008DED050AB0EEC00AB4EEC80AF1EE10FACB
:10B7300040F1AC80F0EEE00AF4EEC80AF1EE10FA47
:10B7400040F1A4807E4BB3F83035980700F1AE800D
:10B7500095F8CB376FF3820385F8CB3795F8CA3766
:10B760001A0700F1A8807748AFF018FE95F8CB379C
:10B770000EAF60F3820313F0040F85F8CB3740F06F
:10B780009C80606901230E963A460F9605A90068D1
:10B79000ADF0CEFA63691868AEF0F6FD636918681B
:10B7A000ADF03CFEA3688DED0B0ACDED0C0A8DEDDE
:10B7B0000D1AD3ED007AF5EEC07AF1EE10FA52DDF3
:10B7C000614B20469FED618AB3F9743600EE903AE2
:10B7D000F8EEE00ACDED030AFFF7E0FAA368B7EE52
:10B7E000002A07EE900ADDED030AD3ED001AB8EE49
:10B7F000E71A9FED4F0A31EE822A61EE881A22EE97
:10B80000082A2DF02DF8DFED527A20EE270ADFED21
:10B81000517A20EE270AF1F021FEDFED4F7A0BA8D6
:10B8200020EE270A20EE088A32F0DCF8B4EEC08A57
:10B83000F1EE10FA17D5C8EE006A9DED0B7ADDED3A
:10B840000C7A636927EE267A67EEA67A8DED0B7A7D
:10B85000CDED0C7A1B68D3F8AC23C3F8B823D3F82A
:10B86000B023C3F8BC23236A38463C491C68FBF765
:10B8700085FF109B0BA92046009397E80C00AAF0C7
:10B88000EDFD12B0BDEC028BBDE8F08195F8CA3732
:10B89000190704D465F08EFC492165F0C7FB95F8C3
:10B8A000CA3743F0080385F8CA3751E795F8CA3715
:10B8B0006FF3C303F7E7002058E70DF11C08214898
:10B8C00007964146089609960A96AFF0EFFD28B90B
:10B8D000A069B2F0BFFD03C888E80300A069B2F018
:10B8E000C1FD09AA01461748AFF046FE9DED087A52
:10B8F0009DED076A0123B7EEC77A6069B7EEC66AA5
:10B9000000930B960BAB0C9609AA39468DED0E6B86
:10B910008DED107B0068ADF043FA95F8CB375B07EF
:10B920007FF52FAF36E700BFB08200309CA5003016
:10B9300000002F44B03200300000003400007A4391
:10B94000B0A20030A4A70030B06200300000C842AE
:10B950000AD7233C35FA8E3C0AE81C4124B7003054
:10B9600013B504460191FFF787FE0199204602B006
:10B97000BDE81040FFF734BA1FB5194B044693F8E1
:10B98000CA371B0729D4002301A916480193029343
:10B990000393AFF099FB032807D8DFE800F0150EFA
:10B9A000020801A92046FFF799FD04B010BD0D481B
:10B9B000AFF0ACFB30B10128F7D100212046FFF7F2
:10B9C000CFFFF2E70121F9E763F0D6FD40F28632BE
:10B9D0004FF4801163F088FDEFE70021EFE700BF2F
:10B9E000B082003098A8003008B5034619B9064A5D
:10B9F00092F9F4241AB91846FFF7B2FF08BDBDE862
:10BA00000840FFF7B9BF00BFB0A200300148FEF701
:10BA1000AFBC00BFB0320030004870471088003023
:10BA20000148F7F72FB900BFB032003030B5174DDD
:10BA30008BB000230022044604A9D5F82C03CDE9DD
:10BA40000423CDE90623CDE90823ADF0FFFC08A9C6
:10BA5000D5F82C03ADF05AFD022201A920469DED38
:10BA6000067B9DED045BF7EEC76BB7EEC55B9DED06
:10BA7000087B8DED015ACDED026AB7EEC77B8DEDE7
:10BA8000037A17F02FF820460BB030BDB0A200307B
:10BA9000014B01221A70704774B7003000207047C4
:10BAA000002070470020704700207047002070473A
:10BAB000002070470020704700207047002070472A
:10BAC000002070479FED010A704700BF0000000092
:10BAD0000020704700207047002070470120704709
:10BAE00000207047002070470020704701207047F9
:10BAF00000207047012070470120704700207047E8
:10BB000001207047012070470020704700487047AF
:10BB10001CB41608004870471CB41608836803F567
:10BB2000805393F80C3CDB0706D50023022280F8F3
:10BB30003C30024BC3F8CC2701207047B082003064
:10BB400090F83C3053B9836803F5805393F80C3C6C
:10BB5000DB0742BF034B0122C3F8CC27002380F848
:10BB60003C307047B0820030012380F83C30704791
:10BB70002DE9F0432DED0C8BF0EE409A97B020EEBE
:10BB8000000A0025F0EE60AA0446B0EE41CA8946DC
:10BB9000A0EEA00A9046F7EE00CA1F460195029556
:10BBA00003950495B7EEC00A05950695F1F0C0FD22
:10BBB000B7EEC00BA3689FEDCDDA03F58053B4EE6A
:10BBC000EC0A03F6C83203F6CC33F1EE10FAD3EDEB
:10BBD000000A92ED009AC8BFCCEE807A29EE0D9A49
:10BBE000C4BF69EEA79A6AEEA7AAB0EE690A2DF063
:10BBF0008FFFA36829EE009A03F58053B0EE6A0A1E
:10BC000003F6C83203F6CC33D2ED008AD3ED000A36
:10BC10002DF07EFFA36868EE8D8A03F5DF5268EE93
:10BC2000808A92ED008AB0EE4C0AD2ED010A2DF026
:10BC30006FFF636828EE0D8A93F9703028EE008A52
:10BC4000002B00F0D980236A9FEDA90A18686C3098
:10BC500032F0CEFAB0EE60AACDED080A8DED091AE9
:10BC60008DED070A2CF07AFEBDEEC0BA40F6B83270
:10BC7000A0491BEE100A2CF031FF4342B0EE4A0AF5
:10BC800007EE903A6368F8EEE77A93ED1A7A67EE7A
:10BC9000877ACDED017A2CF061FEFDEEC0BA40F658
:10BCA000B83294491BEE900A2CF018FF42426368A8
:10BCB00007EE902A039593ED1B7AF8EEE77A93F955
:10BCC0007030022B67EE877ACDED027A6ED18A4B07
:10BCD000B8EECBBAB3F974360AEE103A236AB8EE6E
:10BCE000CAAA1A68B4EECABAF1EE10FA3DDDA3682A
:10BCF0003AEE4B0ADFED810A03F5DE53A16B92EDBC
:10BD0000051A93ED027AD1ED001A27EE0D7AC7EEEF
:10BD1000200A2DF02DFBDDED017A37EE800A8DED46
:10BD2000010AB8EEEB0A236A1A68B4EECA0AF1EE09
:10BD300010FA34DDA3683AEE400AA16B03F5DE5336
:10BD400092ED061AD1ED001AD3ED020A20EE8DDA3B
:10BD5000DFED6A0ACDEE200A2DF00AFBDDED027A56
:10BD600037EE800A8DED020A20E0B1EE4A0AB4EE09
:10BD7000C0BAF1EE10FAD4D5A36830EE4B0AA16B2D
:10BD800003F5DE53DFED5D0AD1ED001A93ED027A83
:10BD900092ED051A27EE0D7AC7EE200AB9E7B1EE4B
:10BDA0004AAAB4EECA0AF1EE10FAC3D4236A12AD5D
:10BDB0000EAED3F800C00CF184030FCB85E80F0062
:10BDC0000AAD86E80F0085E80F0004AB01AA2946FA
:10BDD0006046AAF0FDFF636893F97030022B16D11C
:10BDE000DDED047A39EE279ADDED057A78EEA78A43
:10BDF000DDED067A38EE278A89ED009AC8ED008AD3
:10BE000087ED008A17B0BDEC0C8BBDE8F083F0EE37
:10BE1000E99ADFED3B0AF0EEEAAAAD20B0EECCCA1B
:10BE2000CDED009AB7EE001AF4EEE9AACDED0AAA1C
:10BE30008DED0ECAF1EE10FA48BF6D46D5ED007AD1
:10BE4000F4EECC7ADFED2F7AF1EE10FAD8BF35465A
:10BE500095ED007A87EE270A3CEEC00A2CF0E6FD4D
:10BE6000E36904A8D3ED937A20EE270A32F0C0F9F3
:10BE70008DED061AB0EEC91AB520F0EEC07A8DED40
:10BE8000040ACDED050A39EE000A31EE671AB0EE6C
:10BE9000C11AF1EE410A2CF0C9FDB0EE409A9DEDB9
:10BEA000050AB0EEE81ABA20F0EEC07A38EE800A41
:10BEB00031EE671AB0EEC11AF1EE410A2CF0B6FD70
:10BEC000F0EE408A9DED060AB0EEC81ABF20F0EEF3
:10BED000C07A38EE000A31EE671AB0EEC11AF1EE00
:10BEE000410A2CF0A3FDB0EE408A85E70000C8426D
:10BEF0009F0CB34548F4FFFFB062003000007A4465
:10BF00000000000000A08C4510B52DED028B836A67
:10BF1000044686B0186871F075FBE36AB0EE408A9B
:10BF2000186871F06FFB636B8DED010A186871F092
:10BF300069FB05ABB0EE401A03A92046B0EE480AF3
:10BF400004AADDED010AFFF713FE636A186890F892
:10BF5000CB1000293CD1B3F02FFA2046FFF75EF852
:10BF6000636AB0EE408A1B6893F8A11001293FD0A4
:10BF7000032946D051B9236A01211868ABF03CFE71
:10BF8000236A1868AAF0A4F99FED218A236A9DED1F
:10BF9000030A1868A368026803F58053DDED040AFC
:10BFA0009DED051A93F80C3C9B074CBFD36B936B2C
:10BFB0009847236A174AB0EE480A18680021D2ED64
:10BFC000000A03685B6E984706B0BDEC028B10BD9B
:10BFD000114B93F9C927002A06DBD3F8CC37022B83
:10BFE00004D190F8A1300BB90121B4E70221B2E7E6
:10BFF000236A1868ABF000FE236A1868AAF07EF97D
:10C00000C2E7D9790029C1D12046FFF7FFFCBDE77F
:10C010000000000030690030B0820030836803F611
:10C02000A82393ED000AB5EEC00AF1EE10FA01DC88
:10C03000FEF7EEBF70470000704700000020704719
:10C040000120704702207047002070470020704791
:10C05000012070470020704781F001007047000008
:10C06000012070470120704700487047B8B4160897
:10C0700000487047C4B4160838B5436904461868C8
:10C08000ADF0ACF818B963691868AEF0CDFA636921
:10C0900020461D68FFF7C4FC6368B3F93820B3F984
:10C0A000363001EE102A00EE903A4342B8EEC11A43
:10C0B000284600EE103AF8EEE00AB8EEC00AACF0FE
:10C0C00071FF636920461D68FFF7AAFC6368B3F936
:10C0D0003820B3F9363001EE102A00EE903A434290
:10C0E000B8EEC11A284600EE103AF8EEE00AB8EEB3
:10C0F000C00AACF0CDFF012038BD000030B50446C9
:10C100002DED028B436985B01D68FFF789FC6368DC
:10C11000B3F93820B3F9363001EE102A00EE903A28
:10C120004342B8EEC11A284600EE103AF8EEE00A93
:10C130005C4DB8EEC00AACF035FF2046FFF7C2F9FF
:10C14000B5F9743608EE103A236A1868B8EEC88A52
:10C1500003689B6E984702AAF0EE400A01A9B0EE70
:10C16000480A2046FEF7C2FC2046FFF773F9236B0E
:10C17000F0EE408A20461B68B3F9083000EE103A12
:10C18000B8EEC00AFFF798F92046B0EE408A8DED70
:10C19000030AFFF745FC6368B3F93630B0EE480A8E
:10C1A00001EE103A43422B2000EE903AB8EEC11A4D
:10C1B000F8EEE00A2CF03AFC20468DED030AFFF77A
:10C1C00003F9042813D8DFE800F0032F252A4B00D9
:10C1D000236A1868AAF07CF8236A00211868AAF07C
:10C1E00043FE63699FED300A1868AEF005FB236AD1
:10C1F000B0EE681ADDED020A18689DED010A0368C9
:10C20000DB6A984763691868AEF072FB05B0BDEC55
:10C21000028B30BD236A01211868AAF025FE236A2B
:10C220001868AAF06BF8DCE7204D2B7863B96368D7
:10C2300045209FED1F1ADFED1C0A93ED040A2CF038
:10C24000F5FB28460CF000F920469DED030AFFF7A8
:10C250009FF803A915488DED030A0CF031F9C6E7E4
:10C26000636A02211868B3F0A7F8B5F9743602AA18
:10C2700001A900EE103A0F48B8EEC00A8AF084FC1B
:10C2800020469DED030AFFF783F80B488DED030A66
:10C290000BF09AFB63699DED030A1868ACF004FF8C
:10C2A000A5E700BFB06200300000000068B80030B1
:10C2B00000007A44F8A60030D8860030002070478D
:10C2C00090F80D33002B14BF1B2003207047000093
:10C2D000002070470120704790F8E402062804D03F
:10C2E000A0F10A03584258417047012070470000EE
:10C2F000012070470120704790F80D03034A044B5A
:10C30000002814BF10461846704700BF60B51608D5
:10C310005164180890F80D03034A044B002814BF19
:10C3200010461846704700BF6CB5160851641808CF
:10C3300090F8E4020B3818BF0120704790F80D33D5
:10C340002BB9044BD3F8000300F001007047002024
:10C35000704700BFB0820030024BD3F80003C0F337
:10C36000C0107047B082003090F8E43223B9034B1C
:10C37000187880F0010070470020704740B8003006
:10C3800038B590F8E4420546012C01D0002038BDB4
:10C39000C368186803681B6998470028F6D1EB68E2
:10C3A00020461B6883F8B848F1E70000C368002204
:10C3B00001201B6883F8B82870470000002370B57F
:10C3C0002DED028B80F80D3384B0B0F87030044648
:10C3D0000D46012B01D8002949D0636A264E1B68FF
:10C3E00093F8CB308BBB0723244884F8E4320368EE
:10C3F000022B02D10021FAF763FF9FED218A01256C
:10C40000E368F0EE480A1868B0EE481AF0EE481AF1
:10C41000B0EE480AB0F0D8FF04F5227084EDC88A67
:10C4200084EDC98A84EDCA8A84F80C5332F028FF5F
:10C43000144805F015FA96F8CA3713486FF3C3038A
:10C4400086F8CA37AEF04AFD11E096F9C837002BDE
:10C45000C9DA04F13C0034F0EDFF05460028C2D1F2
:10C460002046FFF7D9FA094A022167F071FA2846F7
:10C4700004B0BDEC028B70BDB082003024B7003038
:10C480000000000028B1003098A8003074B51608EC
:10C4900038B5094D044695F87038012B03D105F6DF
:10C4A0006C0032F057FF95F83D14044873F07EFE9F
:10C4B000002384F80D3338BDB0A2003074A60030DC
:10C4C0000A4B10B504462DED028BB0EE408AD3F82E
:10C4D0003003B0F0DFFA9FED060A012028EE008A53
:10C4E00084EDC98ABDEC028B10BD00BFB0A2003044
:10C4F0000AD7233C0A4B10B504462DED028BB0EE53
:10C50000408AD3F83003B0F0D5FA9FED060A012037
:10C5100028EE008A84EDCA8ABDEC028B10BD00BFF4
:10C52000B0A200300AD7233C0A4B10B504462DEDCB
:10C53000028BB0EE408AD3F83003B0F0C9FA9FED19
:10C54000060A012028EE008A84EDC88ABDEC028B21
:10C5500010BD00BFB0A200300AD7233CC3681B68DF
:10C560001869ADF0ADB8000038B5D0F8E83204462F
:10C570000D461BB9BCF06EF8C4F8E802BCF06AF8CE
:10C58000D4F8E832C01A4FF47A73B0FBF3F0B4F881
:10C59000E632984209D32046FFF73EFA2B88044A38
:10C5A000062167F0D5F9012038BD0020FCE700BF67
:10C5B00090B5160890F8E432052B05D1054BD3F859
:10C5C0003833D868ACF0ECBFC36818680368DB6820
:10C5D000184700BFB0A2003008B590F8E432052B30
:10C5E0000BD1094BD3F83833D868243031F0FAF93D
:10C5F000BCEEC00A10EE100A08BDC36818680368D4
:10C600009B689847F4E700BFB0A2003090F8E4328E
:10C610008B4206D00B2B80F8E41202D10148FCF7C4
:10C6200069BD7047B032003073B501231E4E054618
:10C630000A4680F87530D6F8D437834214D10124E5
:10C64000019285F80D43D6F8D40703681B68984714
:10C65000019A0146154864F0C1F896F8C9379A0660
:10C660001BD4204602B070BD01910321FEF730FFBC
:10C67000019A04460028E2D185F8750064F09AFD1D
:10C680001B220A2164F0F2FC96F8C9379B06E8D514
:10C69000074A137843F0040303E0054A137843F094
:10C6A00002031370DDE700BFB0820030F8440030B1
:10C6B0002CB9003030B585B004460D4601466846B9
:10C6C000FFF7B4F9694604F13C0035F065FCC8B9E0
:10C6D00064F070FD1B220A2164F0C8FC0D4B93F836
:10C6E000C9379B0604D50C4A137843F00403137032
:10C6F0002046FFF791F9094A042167F029F9002043
:10C7000005B030BD2946204605B0BDE83040FFF7F2
:10C710008BBF00BFB08200302CB90030A4B5160822
:10C7200030B585B004460D4601466846FFF77EF9F0
:10C73000694604F13C0035F053FCC8B964F03AFD99
:10C740001B220A2164F092FC0D4B93F8C9379B061B
:10C7500004D50C4A137843F0040313702046FFF706
:10C760005BF9094A042167F0F3F8002005B030BDF9
:10C770002946204605B0BDE83040FFF755BF00BF51
:10C78000B08200302CB90030E0B516087FB5054600
:10C790000E460146684605F13C04FFF747F9694635
:10C7A000204635F01DFCC0B92046694635F0F4FB43
:10C7B000044690B964F0FEFC1B220A2164F056FC8A
:10C7C0000D4B93F8C9379B060FD42846FFF724F981
:10C7D0000A4A042167F0BCF804E031462846FFF716
:10C7E00023FF0446204604B070BD054A137843F089
:10C7F00004031370E9E700BFB082003018B61608D2
:10C800002CB9003030B5044685B00F480BF044FA1F
:10C810000546B0B1072301A984F8E432002301934F
:10C8200002930393E3681868B0F0C0F8E36801A9C5
:10C830000022186803685B68984700210348FAF7EC
:10C840003FFD284605B030BDB032003024B700307F
:10C85000F0B5404F05460C46D7E9C0322DED028BAE
:10C860001343D7F8FC2287B013430CD162F084FE47
:10C8700040F275124FF4801107B0BDEC028BBDE899
:10C88000F04062F031BE8069B1F0E6FD2046B0EEC6
:10C89000408A15F0B7FD032839D1EB6801A9186863
:10C8A000B0F08AF9064690B3DDED017A636838EEA0
:10C8B000678A0093284B0021DFED287A93F9C83767
:10C8C0009FED270A002B009B264827FE800A38EEA2
:10C8D000008ABDEEC88A18EE102A9342ACBF0093BE
:10C8E0000092FAF7EDFC6B691868ADF09DFEDDED86
:10C8F000007A31461C48B8EEE70A0CF061F80021D6
:10C900002846FFF783FE07B0BDEC028BF0BD94E82C
:10C910000F0002AE86E80F00D7F800336A46022106
:10C9200030460493D7F80433059315F077FD78B9B2
:10C9300064F040FC0222152164F098FBDDED037ADF
:10C94000F8EEE77A77EE887AFDEEE77ACDED007AB9
:10C950000026AFE7B0A20030B08200300000000037
:10C960000000C84224B7003040B8003030B52DED8B
:10C97000028BC3688BB004460D461868B0F0F2F81D
:10C9800000285CD1002301930293039394F8E432CE
:10C99000F3B90022002304A93848CDE90423CDE9E6
:10C9A0000623CDE908230CF03DF888B19DED067B08
:10C9B0009DED045BF7EEC76BB7EEC55B9DED087BA5
:10C9C0008DED015ACDED026AB7EEC77B8DED037A8E
:10C9D00094EDC80A9FED2A8AE368B4EEC80ADDED3B
:10C9E000010A9DED021ADDED031AF1EE10FA186846
:10C9F000AABFDFED247A9FED240A20EE270AB0F0CB
:10CA0000E3FCD4EDC97AF4EEC87AF1EE10FA07DB54
:10CA1000E3689FED1C0A186827EE800AB0F03AF828
:10CA2000D4EDCA7AF4EEC87AF1EE10FA07DBE368C7
:10CA30009FED140A186827EE800AB0F03BF8E3680F
:10CA400029461868B0F0EAFB054688B10F4B1B6811
:10CA5000022B09D0032B03D10D4B93F9A5361BB143
:10CA600000210A48FAF74CFC01212046FFF7CEFDD1
:10CA700028460BB0BDEC028B30BD00BF40B8003083
:10CA8000000000340000C8420000000024B700305D
:10CA9000B062003010B52DED028BC3680446DFEDA7
:10CAA000338A1B684269D3ED0A0A9FED318AF4EE9E
:10CAB000E80A93ED060A1068F1EE10FA60FE880AA3
:10CAC000ACF044F8E36862691B681068D3ED0A0AA9
:10CAD00093ED060AF4EEE80AF1EE10FA60FE880A19
:10CAE000ACF0AAF863691868ACF04EFA18B963693B
:10CAF0001868ADF001FBE36862691B68106893ED8C
:10CB0000080A93ED0C1AD3ED070AB0EEC00AACF098
:10CB100049FAE36862691B68106893ED080A93EDAF
:10CB20000C1AD3ED070AB0EEC00AACF0B1FA636993
:10CB30001868ACF053FB18B963691868ADF074FD60
:10CB400000210C48FAF7BCFB0B488CF0A5F90B4A06
:10CB500020460221B2F8CA3723F48163A2F8CA370B
:10CB6000BDEC028BBDE81040FFF750BD0000003463
:10CB700000007A4324B7003084A70030B082003030
:10CB80000C4B10B50446D3F8380390ED0F0A00F1B2
:10CB9000200190F86020AFF02BFC07480368022BBF
:10CBA00002D00821FAF78CFB20460521BDE8104091
:10CBB000FFF72CBDB0A2003024B70030F0B5504DC7
:10CBC00004460E461746D5F838032DED028BB0EE1D
:10CBD000408A93B0AFF038FADFED4A8AF0EEC87AB7
:10CBE000F4EEE87AF1EE10FA07D49FED470AD5F893
:10CBF000380328EE000AAFF089FAD5F8380390ED33
:10CC00000F0AB0EEC00A0FB1B1EE400AAFF06EFAF3
:10CC1000002302AA03A9D5F83803039304930593CC
:10CC2000AFF090FADFED397A9DED027AB4EEE77A53
:10CC3000F1EE10FA5FDD022203A90EA815F052FFF3
:10CC400071683046019115F0DDFB019902460EA88E
:10CC500015F0AEFBE3680EA91868B0F0DFFA10B962
:10CC60002B48FCF741FEA069B1F0F4FB90ED017A8E
:10CC700090ED006A06A9B7EEC77AD5F83803B7EE8B
:10CC8000C66A20308DED066B8DED087B31F0C6F95C
:10CC90000AA88DED0A0B8DED0C1B31F009FA1D4B26
:10CCA0001B68022B1CD0D5F83833B7EEC00B00211F
:10CCB0001848D3ED0E7AF4EEE87AF1EE10FAB8BF28
:10CCC000D3ED047AF4EEC07AF1EE10FA10D5DFED70
:10CCD000127AB4EEE70AF1EE10FA09DDFAF710FB6A
:10CCE00004212046FFF792FC13B0BDEC028BF0BD8F
:10CCF000FAF7E6FAF4E72046FFF742FFF4E700BF51
:10CD0000B0A20030000000340000C842000096438A
:10CD1000B032003024B700300000FA43284B70B521
:10CD20002DED028BD3E9CB54DFED268A0646D4EDF8
:10CD30000A0A28469FED248AF4EEE80A94ED060AD2
:10CD4000F1EE10FA60FE880AABF000FFD4ED0A0A9B
:10CD5000284694ED060AF4EEE80AF1EE10FA60FEB9
:10CD6000880AABF069FF2846ACF00EF910B92846E6
:10CD7000ADF0C2F994ED080A284694ED0C1AB0EE15
:10CD8000C00AD4ED070AACF00DF994ED080A284664
:10CD900094ED0C1AB0EEC00AD4ED070AACF078F9A5
:10CDA0002846ACF01BFA10B92846ADF03DFC002136
:10CDB0000648FAF785FA0123BDEC028B337070BD8B
:10CDC000B0A200300000003400007A4324B70030E5
:10CDD000074808B5D0F800339B0704D50121A0F51A
:10CDE000A040F5F7B1FD0348BDE808400BF046BC94
:10CDF000B082003040B8003030B589B00446FDF74D
:10CE000059FF30B10021204609B0BDE83040FDF7A0
:10CE100089BF636A02211868B2F0CEFAE368186825
:10CE200003685B69984701461048FCF747FC636953
:10CE30001868ADF05DFD236A1D68636905AC18686C
:10CE4000ACF0ECFA20460A498DED020ACDED030A5A
:10CE50008DED041AFAF792FC079B02A9284600936D
:10CE600094E80C00A9F0FAFA09B030BDB0320030F5
:10CE700024B7003038B50446FDF71CFF054628B13D
:10CE800020460021BDE83840FDF74CBF636A02210F
:10CE90001868B2F091FA29462046BDE83840FEF7FE
:10CEA000A3BD00000021014807F02EB988B2003070
:10CEB00030B5174D89B09FED170A044605F5E043DC
:10CEC000D3F83803AFF002FB01462846FCF7F6FB27
:10CED00063691868ADF00CFD236A1D68636905ACD1
:10CEE0001868ACF09BFA20460B498DED020ACDED97
:10CEF000030A8DED041AFAF741FC079B02A92846A4
:10CF0000009394E80C00A9F0A9FA09B030BD00BF65
:10CF1000B03200300000000024B7003030B589B0D6
:10CF20000446FDF7C7FE30B10021204609B0BDE838
:10CF30003040FDF7F7BE636A02211868B2F03CFA90
:10CF4000E368186803685B69984701461048FCF776
:10CF5000B5FB63691868ADF0CBFC236A1D68636993
:10CF600005AC1868ACF05AFA20460A498DED020A61
:10CF7000CDED030A8DED041AFAF700FC079B02A918
:10CF80002846009394E80C00A9F068FA09B030BD77
:10CF9000B032003024B7003030B52DED028B83B0B5
:10CFA0000446FDF787FE20B9636A1B6893F8CC300E
:10CFB00043B90021204603B0BDEC028BBDE83040F0
:10CFC000FDF7B0BE94F8EC32DA071DD4E3681D68B3
:10CFD0002B6828469B689847D5ED097A94F8EC327F
:10CFE000B4EEE70AF1EE10FA4CBF0122002262F320
:10CFF000000384F8EC3207D4204603B0BDEC028B6A
:10D00000BDE83040FFF7F8BE94F8EC329B0732D40D
:10D01000E368DFED448A1B686269D3ED0A0A9FED7D
:10D02000428AF4EEE80A93ED060A1068F1EE10FA6F
:10D0300060FE880AABF08AFDE36862691B681068CD
:10D04000D3ED0A0A93ED060AF4EEE80AF1EE10FABF
:10D0500060FE880AABF0F0FD63691868ABF094FFDE
:10D0600018B963691868ADF047F894F8EC3243F0EA
:10D07000020384F8EC322D4BD4F8F422D3F8FC32BE
:10D080009B1A07EE903AB8EEE78AF1EE047AB0EE1A
:10D09000C87AB4EEE77AF1EE10FA38D594F8EC32AB
:10D0A00043F0040384F8EC32204684EDBC8AFEF79A
:10D0B000E3FA6369A26BB1EE480A1B68D2ED001A6D
:10D0C00093EDC91AD3ED0E0A2CF052F9636940F2C0
:10D0D000AA401B6893EDC61AD3EDC70A2BF0A6FC35
:10D0E0002046FEF755F912488DED010A0AF06CFC56
:10D0F00063699DED010A1868ABF0D6FF6369186893
:10D1000003B0BDEC028BBDE83040ADF0F1BBD4ED17
:10D11000BC7A68EE277AF5EEC07AF1EE10FAC3D544
:10D12000BCE700BF0000003400007A43B0A200302A
:10D13000D886003030B52DED028B83B00446FDF764
:10D14000B9FD20B9636A1B6893F8CC3043B900215C
:10D15000204603B0BDEC028BBDE83040FDF7E2BDD8
:10D16000636940F2C440DFED327A64251B6894EDB8
:10D17000C60A93EDC61AD3EDC70A20EE270A2BF094
:10D1800055FC2046FEF704F9236AB0EE408A186881
:10D1900003689B6E9847274B6846B3F9743607EED1
:10D1A000903AB4F81033F8EEE77A13FB05F307EE84
:10D1B000103A94F91233B4EEE70A13FB05F3F8EED4
:10D1C000C76AF1EE10FA07EE103ACDED006AB8EE3C
:10D1D000C77A77FE807A9FED180AF4EE407A8DEDDB
:10D1E000017AF1EE10FA58BFB0EE670A30F054FC45
:10D1F000236A0121DDED010A1868B4F814330268CE
:10D2000013FB05F39DED000A126B01EE103AB8EE28
:10D21000C11A90476369B0EE480A1868ABF044FF42
:10D2200063691868ADF064FB03B0BDEC028B30BDE0
:10D230000000C842B062003000007A44F0B5B34D3F
:10D2400004462DED028BD5F8D40785B0FDF732FDED
:10D2500048B10021D5F8D40705B0BDEC028BBDE87C
:10D26000F040FDF75FBD05F500570221D5F8F8073E
:10D27000B2F0A2F8D7F8243393ED378ABBF0EAF97D
:10D28000B5F8C837064603F481437BB1D7F82C03C1
:10D29000ABF0DAFC2378022B08D16DF0F5FD9C4B46
:10D2A0009C4A062166F054FB0323237084F08EFF12
:10D2B00084F078FF48B184F089FF84F07DFF20B1CD
:10D2C0002378012B10D9022B20D02378082B00F2D1
:10D2D0008581DFE813F024003C00660002013D0177
:10D2E000440158015A012D006DF0CEFD884B8A4A49
:10D2F000062166F02DFBD7F82C3393EDDA7B08235B
:10D30000B7EEC77B84ED057A2370DEE76DF0BCFDD8
:10D310007F4B824A062166F01BFB0323F4E7D7F814
:10D32000300303681B69984710B12046FFF7F6FCED
:10D330002378082B00F27081DFE813F059016101B6
:10D34000610177017701770177017F017F01A66095
:10D35000D7F82C3393EDDA7BB7EEC77B84ED057AF3
:10D360009FED6F7AD5EDDC7AF4EEC77AF1EE10FA24
:10D370004FDB9FED6C7A67EE877AD7F8303393ED09
:10D38000087A4FF07E53B0EEC77A23610223F4EEA1
:10D39000477A2370F1EE10FA48BFB0EE677A84ED59
:10D3A000067A94ED016ADFED5E6AF0EEC67AD7F890
:10D3B0002C33F4EEE67AF1EE10FA0CD493EDDA7B2E
:10D3C000B7EEC77BD4ED057A77EEC77AB4EEE76A9D
:10D3D000F1EE10FA29D49FED547AD4ED067A67EE77
:10D3E000877A93EDE47AB4EEE77AF1EE10FA26DC70
:10D3F000A368D4ED047AF31AB3F5FA6F21D2B4EE30
:10D40000678AF1EE10FA37FE888A84ED048AE660B6
:10D410008EE7464BB3F9AA36002BB8BF5B429BB2EE
:10D4200007EE903AF8EEE77AA7E7062323706DF04F
:10D430002BFD374B3E4A042166F08AFA78E7A66056
:10D4400076E795EDD97A67EE877AF4EEC87AF1EE51
:10D4500010FADCD4D5EDDA7AF4EEE67AF1EE10FAD1
:10D4600021DB95F8983333B9062323706DF00CFD5A
:10D47000274B304ADFE730480AF008FA98B195F9AF
:10D48000AE3383B9B5F99A33D5EDDA7A07EE103AAF
:10D49000DFED246AB8EEC77A67EEA67AB4EEE77AD3
:10D4A000F1EE10FAB3DCE068301AB0F5FA7F7FF6DF
:10D4B0003FAF032323706DF0E7FCD4ED047A95EDC4
:10D4C000D97A0621124B27EE277A1C4AB7EEC77A83
:10D4D0008DED007B66F03CFA2AE7D7F82C03ADF01F
:10D4E00027F984F073FE84F05DFE68B16DF0CCFC2A
:10D4F000074B134A062166F02BFA84F067FE84F08E
:10D500003FFE0423237013E70523FBE7B0820030BE
:10D5100064B6160872B616087CB6160893B61608D6
:10D52000000000340000C842333373BFB0620030E3
:10D53000A5B61608C0B61608B0320030F0B6160808
:10D5400018B7160800007A440000FA43CDCCCC3D51
:10D5500084F03CFE84F026FEC8BB05232370E068FF
:10D560005FED087AD5EDDB6A361A1FED097AA6EE73
:10D57000A77A07EE906AF8EE677AF4EEC77AF1EED2
:10D5800010FA3FF5D5AE07232370D7F82C331FEDE3
:10D59000117AD3EDC67AD3EDC96A67EE877AB6EE13
:10D5A000007A67EEA77A67EE877A87EEA67AD4EDDF
:10D5B000056A76EEC76A93EDDA7BB7EEC77BF4EEC9
:10D5C000C76AF1EE10FA3FF6B3AE08239AE784F08B
:10D5D000FDFD84F0F1FD0028BFD1A9E661F0CCFF8C
:10D5E00040F29C524FF4801161F07EFFA0E61C488F
:10D5F00005B0BDEC028BBDE8F040FFF7FDBBD5F8F0
:10D60000D407FEF739F894ED060A0121B1EE400A7D
:10D61000D7F82C03ABF058FDD7F82C0305B0BDECC0
:10D62000028BBDE8F040ADF063B9D5F8D407FEF742
:10D6300023F800219FED0B0AEAE79FED0A8AD5F84F
:10D64000D4078DED038AFEF717F8B0EE480A0123E0
:10D6500003AA04F11401D7F82C03ACF0C1FBDBE7FB
:10D66000E0AA0030000000002DE9F041074608461E
:10D670000E462DED028B84B014F0C4FE03288046C4
:10D680006D462CD1FB681868AFF0C8F8012826D188
:10D69000294625480AF07CF90446D0B17B69424608
:10D6A000DDED007A1B68F8EEE77A03F5806393ED11
:10D6B000006BB7EEC66B77EEC67AFDEEE77A17EE33
:10D6C000901ACDED007AC829B8BFC821304614F0B1
:10D6D0006FFE204604B0BDEC028BBDE8F081134B19
:10D6E0000FCB85E80F00304614F08CFE014628462B
:10D6F00014F0F0FE04460028EBD07B692846DDEDEF
:10D70000017A1B68B8EEE78A03F5806393ED007B2E
:10D71000B7EEC77B38EE478A14F074FE0246BDEEC2
:10D72000C88A18EE101AD1E7B0320030A8A5003030
:10D7300010B543698CB00C461B68684693EDFC5BE2
:10D7400093EDFE6B03F580639FED0F4B93ED007B34
:10D7500025EE045B26EE046B27EE447B8DED005B2B
:10D760008DED026B8DED047B31F066FC06A9204641
:10D770008DED060B8DED081B8DED0A2B15F056FA7D
:10D780000CB010BDAFF3008000000040E17A843F90
:10D79000083230B504461D4685B00FCA84E80F0034
:10D7A000134301BFAB68A360EB68E360636893B9A0
:10D7B000204614F027FE03AA0146284614F02EFE48
:10D7C00060B103992046019114F01CFE01990246B4
:10D7D000204614F0EDFD204605B030BD69682846AE
:10D7E0000191F1E730B50B6985B004460BB94B697F
:10D7F00053B3002308316D46C4F808330FC985E8D8
:10D800000F0029462046FFF72FFF98B9124B01223F
:10D810002846D3F8FC1214F0CBFD63F0CBFC0222B7
:10D82000152163F023FC2046FEF7F6F80B4A02218F
:10D8300066F08EF829462046FFF798F810B9084898
:10D84000FCF752F805B030BD0123C0F8083305B02D
:10D85000BDE83040FFF71EB9B0A2003034B716085B
:10D86000B032003070B51A4B88B004460E466D4693
:10D870000FCB85E80F0020462946FFF759FFE368E4
:10D880001868AFF06FF998B1E368186803681B690E
:10D89000984768B1E36829461868AEF0CBFF38B9FD
:10D8A00061F06AFE40F295624FF4801161F01CFE57
:10D8B000214604A82B463246FFF76AFF04A92046FA
:10D8C000FFF754F810B90348FCF70EF808B070BD24
:10D8D000A8A50030B032003070B5154B88B00C46AA
:10D8E00006466D460FCB85E80F0029463046FFF708
:10D8F0001FFF2B462246314604A8FFF749FF6288E6
:10D90000A388122A4FEA132305D1227ED20744BFEF
:10D9100003EB83035B0007EE903A227A04A93046BA
:10D92000B8EE670AC2F34002FFF748F908B070BDCD
:10D93000A8A5003038B504460D46FFF793FF002335
:10D94000C4F8E832AB88A4F8E63238BD7FB50D469E
:10D950000446FFF787FF6E4605F108010FC986E808
:10D960000F00134306D1234BD3F80023D3F804331D
:10D970000292039304F53D720121304614F04EFDEE
:10D9800094F8EC3270B923F00503204643F0050308
:10D9900084F8EC32FEF740F8174A062165F0D8FF0C
:10D9A00004B070BD23F00703626984F8EC320023F1
:10D9B000C4F8F032E36810681B6893ED080A93ED31
:10D9C0000C1AD3ED070AB0EEC00AABF0EBFAE3682D
:10D9D00062691B68106893ED080A93ED0C1AB0EEAB
:10D9E000C00AD3ED070AABF053FB08212046FEF72F
:10D9F0000DFED5E7B0A2003060B716082DE9F04360
:10DA00008DB088461C4607466D4613460A460146B9
:10DA10002846DDE91469FFF7BBFE95E80F0084E8AE
:10DA20000F0007A814F0BEFCB8F80430F3B9B8F83A
:10DA3000001005AA07F13C00013189B233F0B2FCB5
:10DA4000A0B1234605AA39462846FFF7A1FE95E86E
:10DA50000F0086E80F00BDF81630A3F152025342C2
:10DA6000534189F800300DB0BDE8F08394E80F0011
:10DA700086E80F000023F4E770B58B8892B0044667
:10DA80000D461646002B47D10DA814F08BFC2988B3
:10DA90000BAA04F13C00013189B233F083FC002869
:10DAA0003AD0BDF82E1052291CD019D8112913D8FC
:10DAB0000F2913D933462A46214603A8FFF768FEEB
:10DAC00003AB214607A80BAAFFF762FEE36807A98C
:10DAD0001868AFF0E3FB01E01329EBD012B070BD82
:10DAE0005E29FAE707AD03A814F05CFC284614F0A1
:10DAF00059FC0DF10B0332460BA92046CDE900532A
:10DB000003ABFFF77BFFE0689DF80B302A4603A9C3
:10DB10000068AFF099FBE1E70120DFE770B5214B2A
:10DB200088B004460E466D460FCB85E80F002046B0
:10DB30002946FFF7FDFDE3681868AFF013F898B1C8
:10DB4000E368186803681B69984768B1E368294669
:10DB50001868AEF06FFE38B961F00EFD40F2166243
:10DB60004FF4801161F0C0FC214604A82B463246D8
:10DB7000FFF70EFE04A92046FEF7F8FE20B90A487A
:10DB8000FBF7B2FE08B070BD002304AA3146204660
:10DB9000C4F8E832B388A4F8E632FFF76DFF002836
:10DBA000F0D1ECE7A8A50030B0320030F0B5324B30
:10DBB00091B004460E4604AD0FCB85E80F00204619
:10DBC0002946FFF7B5FDE3681868AEF0CBFF98B1C2
:10DBD000E368186803681B69984768B1E3682946D9
:10DBE0001868AEF027FE38B961F0C6FC4FF4DF626A
:10DBF0004FF4801161F078FC0CAF08A814F0D2FB50
:10DC0000384614F0CFFB0DF10F032A46314620466B
:10DC1000CDE9007308ABFFF7F1FEE0689DF80F3027
:10DC20003A4608A90068AFF04FFE20B91348FBF749
:10DC30005BFE11B0F0BD002308AA31462046C4F8AF
:10DC4000E832B388A4F8E632FFF716FF0028EDD0DB
:10DC50000B4B1B68022B09D0032B03D1094B93F903
:10DC6000A5361BB100210648F9F74AFB01212046E1
:10DC7000FEF7CCFCDDE700BFA8A50030B0320030D5
:10DC800024B70030B0620030DFED0A7A91ED041A5B
:10DC9000D1ED030A91ED020A21EE271A8B884FF489
:10DCA0007A7160EEA70A044820EE270A594303F070
:10DCB000E1BD00BF0000C84228B1003037B50446BE
:10DCC0000D46BAF0C7FCC4F8FC02D5ED027AF5EEB9
:10DCD000C07AF1EE10FA17DD9FED137A67EE877ABE
:10DCE000FCEEE77AC4EDBE7A2046FDF795FED4F847
:10DCF000F8224FF47A730621B2FBF3F30B4A03B018
:10DD0000BDE8304065F024BE84F098FD002395F90D
:10DD10000D20009395F90C1095F90E3084F0E2FC7B
:10DD2000C4F8F802E0E700BF00007A4478B71608AC
:10DD300010B5B1F90A300446A0F8103391F90C304F
:10DD400080F81233B1F90D30A0F81433B1F90F3067
:10DD500007EE903AF8EEE77AC0EDC67ABAF07AFCB0
:10DD60000B21C4F81C032046BDE81040FEF74EBC52
:10DD700038B504460D46BAF06DFC9FED067AC4F83E
:10DD80000403D5ED027A67EE877AFDEEE77AC4EDFB
:10DD9000C07A38BD00007A444A7C0B460548003AF8
:10DDA00091F91010D3ED030A18BF012293ED020A76
:10DDB000F9F7B0BA24B7003070B51B4E044686B0F0
:10DDC0000D46D6F8D40703681B689847042806D187
:10DDD0006B88102B0FD0732B20D000201CE0D6F8BE
:10DDE000D40703681B6898470328F6D194F8E432F7
:10DDF000062BF2D1ECE705F1080102ACDFED0B0ACE
